 MFCD42D

 Timestamp is 3588714a (Wed Jun 17 18:45:46 1998)

 Preferred load address is 5f700000

 Start         Length     Name                   Class
 0001:00000000 0002b66eH .text                   CODE
 0001:0002b670 00000242H .text$AFX_CORE2         CODE
 0001:0002b8c0 00000516H .text$AFX_INIT          CODE
 0001:0002bde0 00000583H .text$AFX_VDEL          CODE
 0001:0002c370 00001bf0H .text$x                 CODE
 0002:00000000 00000518H .idata$5                DATA
 0002:00000520 0000745cH .rdata                  DATA
 0002:00007980 000007acH .rdata$r                DATA
 0002:00008130 000032d8H .xdata$x                DATA
 0002:0000b408 00000060H .didat$2                DATA
 0002:0000b468 00000020H .didat$3                DATA
 0002:0000b488 0000009cH .didat$4                DATA
 0002:0000b524 00000036H .didat$6                DATA
 0002:0000b55c 0000009cH .didat$7                DATA
 0002:0000b5f8 00000064H .idata$2                DATA
 0002:0000b65c 00000014H .idata$3                DATA
 0002:0000b670 00000518H .idata$4                DATA
 0002:0000bb88 0000032aH .idata$6                DATA
 0002:0000bec0 00000b38H .edata                  DATA
 0003:00000000 00000004H .CRT$XCA                DATA
 0003:00000004 00000004H .CRT$XCL                DATA
 0003:00000008 00000004H .CRT$XCZ                DATA
 0003:0000000c 00000004H .CRT$XIA                DATA
 0003:00000010 00000004H .CRT$XIZ                DATA
 0003:00000020 00000538H .data                   DATA
 0003:00000558 0000009cH .didat$5                DATA
 0003:000005f8 00000064H .bss                    DATA
 0004:00000000 00000100H .rsrc$01                DATA
 0004:00000100 00001030H .rsrc$02                DATA

  Address         Publics by Value              Rva+Base     Lib:Object

 0001:00000000       ?GetHead@CSimpleList@@QBEPAXXZ 5f701000 f i dlldb.obj
 0001:00000010       ?AfxThrowDBException@@YGXFPAVCDatabase@@PAX@Z 5f701010 f   dbcore.obj
 0001:00000121       ??0CDBException@@QAE@F@Z   5f701121 f   dbcore.obj
 0001:00000194       ??1CDBException@@UAE@XZ    5f701194 f   dbcore.obj
 0001:000001f7       ?BuildErrorString@CDBException@@UAEXPAVCDatabase@@PAXH@Z 5f7011f7 f   dbcore.obj
 0001:000005cb       ?GetErrorMessage@CDBException@@UAEHPADIPAI@Z 5f7015cb f   dbcore.obj
 0001:0000064a       ?TraceErrorMessage@CDBException@@QBEXPBD@Z 5f70164a f   dbcore.obj
 0001:00000757       ?Empty@CDBException@@QAEXXZ 5f701757 f   dbcore.obj
 0001:00000778       ?AfxGetHENV@@YGPAXXZ       5f701778 f   dbcore.obj
 0001:00000793       ??0CDatabase@@QAE@XZ       5f701793 f   dbcore.obj
 0001:0000085f       ??1CDatabase@@UAE@XZ       5f70185f f   dbcore.obj
 0001:000008e1       ?Open@CDatabase@@UAEHPBDHH0H@Z 5f7018e1 f   dbcore.obj
 0001:00000ac0       ?OpenEx@CDatabase@@UAEHPBDK@Z 5f701ac0 f   dbcore.obj
 0001:00000c34       ?ExecuteSQL@CDatabase@@QAEXPBD@Z 5f701c34 f   dbcore.obj
 0001:00000e93       ?Cancel@CDatabase@@QAEXXZ  5f701e93 f   dbcore.obj
 0001:00000ee6       ?Close@CDatabase@@UAEXXZ   5f701ee6 f   dbcore.obj
 0001:0000105b       ?Free@CDatabase@@IAEXXZ    5f70205b f   dbcore.obj
 0001:00001196       ?OnSetOptions@CDatabase@@UAEXPAX@Z 5f702196 f   dbcore.obj
 0001:00001224       ?GetDatabaseName@CDatabase@@QBE?AVCString@@XZ 5f702224 f   dbcore.obj
 0001:000012c8       ?BeginTrans@CDatabase@@QAEHXZ 5f7022c8 f   dbcore.obj
 0001:00001375       ?CommitTrans@CDatabase@@QAEHXZ 5f702375 f   dbcore.obj
 0001:00001457       ?Rollback@CDatabase@@QAEHXZ 5f702457 f   dbcore.obj
 0001:00001539       ?Check@CDatabase@@UBEHF@Z  5f702539 f   dbcore.obj
 0001:00001556       ?CheckHstmt@CDatabase@@QBGHFPAX@Z 5f702556 f   dbcore.obj
 0001:0000160e       ?ReplaceBrackets@CDatabase@@QAEXPAD@Z 5f70260e f   dbcore.obj
 0001:00001763       ?AllocConnect@CDatabase@@IAEXK@Z 5f702763 f   dbcore.obj
 0001:0000198f       ?Connect@CDatabase@@IAEHK@Z 5f70298f f   dbcore.obj
 0001:00001af9       ?VerifyConnect@CDatabase@@IAEXXZ 5f702af9 f   dbcore.obj
 0001:00001bc3       ?GetConnectInfo@CDatabase@@IAEXXZ 5f702bc3 f   dbcore.obj
 0001:00001fe8       ?BindParameters@CDatabase@@UAEXPAX@Z 5f702fe8 f   dbcore.obj
 0001:00001ff5       ?AssertValid@CDatabase@@UBEXXZ 5f702ff5 f   dbcore.obj
 0001:00002008       ?Dump@CDatabase@@UBEXAAVCDumpContext@@@Z 5f703008 f   dbcore.obj
 0001:00002148       ??0CRecordset@@QAE@PAVCDatabase@@@Z 5f703148 f   dbcore.obj
 0001:000025a0       ??1CRecordset@@UAE@XZ      5f7035a0 f   dbcore.obj
 0001:000027d1       ?Open@CRecordset@@UAEHIPBDK@Z 5f7037d1 f   dbcore.obj
 0001:00002aa2       ?Close@CRecordset@@UAEXXZ  5f703aa2 f   dbcore.obj
 0001:00002e9e       ?IsOpen@CRecordset@@QBEHXZ 5f703e9e f   dbcore.obj
 0001:00003014       ?IsFieldDirty@CRecordset@@QAEHPAX@Z 5f704014 f   dbcore.obj
 0001:0000315e       ?IsFieldNull@CRecordset@@QAEHPAX@Z 5f70415e f   dbcore.obj
 0001:00003232       ?IsFieldNullable@CRecordset@@QAEHPAX@Z 5f704232 f   dbcore.obj
 0001:000032bd       ?CanBookmark@CRecordset@@QBEHXZ 5f7042bd f   dbcore.obj
 0001:00003348       ?Move@CRecordset@@UAEXJG@Z 5f704348 f   dbcore.obj
 0001:000034e1       ?CheckRowsetError@CRecordset@@UAEXF@Z 5f7044e1 f   dbcore.obj
 0001:0000366d       ?GetBookmark@CRecordset@@QAEXAAVCDBVariant@@@Z 5f70466d f   dbcore.obj
 0001:00003758       ?SetBookmark@CRecordset@@QAEXABVCDBVariant@@@Z 5f704758 f   dbcore.obj
 0001:000037f7       ?SetRowsetSize@CRecordset@@UAEXK@Z 5f7047f7 f   dbcore.obj
 0001:00003984       ?AddNew@CRecordset@@UAEXXZ 5f704984 f   dbcore.obj
 0001:00003a9e       ?Edit@CRecordset@@UAEXXZ   5f704a9e f   dbcore.obj
 0001:00003c68       ?Update@CRecordset@@UAEHXZ 5f704c68 f   dbcore.obj
 0001:00003d2a       ?Delete@CRecordset@@UAEXXZ 5f704d2a f   dbcore.obj
 0001:00003dde       ?CancelUpdate@CRecordset@@QAEXXZ 5f704dde f   dbcore.obj
 0001:00003e5d       ?FlushResultSet@CRecordset@@QBEHXZ 5f704e5d f   dbcore.obj
 0001:00003ed5       ?GetODBCFieldInfo@CRecordset@@QAEXPBDAAUCODBCFieldInfo@@@Z 5f704ed5 f   dbcore.obj
 0001:00003f98       ?GetODBCFieldInfo@CRecordset@@QAEXFAAUCODBCFieldInfo@@@Z 5f704f98 f   dbcore.obj
 0001:0000406e       ?GetFieldValue@CRecordset@@QAEXPBDAAVCDBVariant@@F@Z 5f70506e f   dbcore.obj
 0001:0000413e       ?GetFieldValue@CRecordset@@QAEXFAAVCDBVariant@@F@Z 5f70513e f   dbcore.obj
 0001:0000435e       ?GetFieldValue@CRecordset@@QAEXPBDAAVCString@@@Z 5f70535e f   dbcore.obj
 0001:00004421       ?GetFieldValue@CRecordset@@QAEXFAAVCString@@@Z 5f705421 f   dbcore.obj
 0001:000045b1       ?SetFieldDirty@CRecordset@@QAEXPAXH@Z 5f7055b1 f   dbcore.obj
 0001:0000466a       ?SetFieldNull@CRecordset@@QAEXPAXH@Z 5f70566a f   dbcore.obj
 0001:0000479d       ?SetParamNull@CRecordset@@QAEXHH@Z 5f70579d f   dbcore.obj
 0001:0000481c       ?SetLockingMode@CRecordset@@QAEXI@Z 5f70581c f   dbcore.obj
 0001:00004892       ?Requery@CRecordset@@UAEHXZ 5f705892 f   dbcore.obj
 0001:00004b25       ?Cancel@CRecordset@@QAEXXZ 5f705b25 f   dbcore.obj
 0001:00004b93       ?GetDefaultConnect@CRecordset@@UAE?AVCString@@XZ 5f705b93 f   dbcore.obj
 0001:00004bd5       ?GetDefaultSQL@CRecordset@@UAE?AVCString@@XZ 5f705bd5 f   dbcore.obj
 0001:00004c17       ?DoFieldExchange@CRecordset@@UAEXPAVCFieldExchange@@@Z 5f705c17 f   dbcore.obj
 0001:00004c37       ?DoBulkFieldExchange@CRecordset@@UAEXPAVCFieldExchange@@@Z 5f705c37 f   dbcore.obj
 0001:00004c80       ?OnSetOptions@CRecordset@@UAEXPAX@Z 5f705c80 f   dbcore.obj
 0001:00004d3c       ?Check@CRecordset@@UBEHF@Z 5f705d3c f   dbcore.obj
 0001:00004e72       ?PreBindFields@CRecordset@@UAEXXZ 5f705e72 f   dbcore.obj
 0001:00004e7d       ?SetState@CRecordset@@IAEXHPBDK@Z 5f705e7d f   dbcore.obj
 0001:00004fcc       ?AllocHstmt@CRecordset@@IAEHXZ 5f705fcc f   dbcore.obj
 0001:000053d9       ?BuildSQL@CRecordset@@IAEXPBD@Z 5f7063d9 f   dbcore.obj
 0001:00005555       ?PrepareAndExecute@CRecordset@@IAEXXZ 5f706555 f   dbcore.obj
 0001:00005912       ?VerifyDriverBehavior@CRecordset@@IAEXXZ 5f706912 f   dbcore.obj
 0001:00005a6a       ?VerifyCursorSupport@CRecordset@@IAEKXZ 5f706a6a f   dbcore.obj
 0001:00005b63       ?AllocAndCacheFieldInfo@CRecordset@@IAEXXZ 5f706b63 f   dbcore.obj
 0001:00005e17       ?AllocRowset@CRecordset@@IAEXXZ 5f706e17 f   dbcore.obj
 0001:00005e7b       ?FreeRowset@CRecordset@@IAEXXZ 5f706e7b f   dbcore.obj
 0001:00005f05       ?EnableBookmarks@CRecordset@@IAEXXZ 5f706f05 f   dbcore.obj
 0001:00005f86       ?SetUpdateMethod@CRecordset@@IAEXXZ 5f706f86 f   dbcore.obj
 0001:00005fd6       ?SetConcurrencyAndCursorType@CRecordset@@IAEXPAXK@Z 5f706fd6 f   dbcore.obj
 0001:000061d1       ?IsSQLUpdatable@CRecordset@@QAEHPBD@Z 5f7071d1 f   dbcore.obj
 0001:00006236       ?IsSelectQueryUpdatable@CRecordset@@QAEHPBD@Z 5f707236 f   dbcore.obj
 0001:000064d2       ?IsJoin@CRecordset@@SGHPBD@Z 5f7074d2 f   dbcore.obj
 0001:0000650d       ?FindSQLToken@CRecordset@@SGPBDPBD0@Z 5f70750d f   dbcore.obj
 0001:0000673f       ?InitRecord@CRecordset@@QAEXXZ 5f70773f f   dbcore.obj
 0001:000067be       ?ResetCursor@CRecordset@@QAEXXZ 5f7077be f   dbcore.obj
 0001:00006817       ?CheckRowsetCurrencyStatus@CRecordset@@QAEXGJ@Z 5f707817 f   dbcore.obj
 0001:00006953       ?FetchData@CRecordset@@QAEFGJPAK@Z 5f707953 f   dbcore.obj
 0001:00006a40       ?SkipDeletedRecords@CRecordset@@QAEXGJPAKPAF@Z 5f707a40 f   dbcore.obj
 0001:00006c4d       ?SetRowsetCurrencyStatus@CRecordset@@UAEXFGJK@Z 5f707c4d f   dbcore.obj
 0001:00006f7e       ?RefreshRowset@CRecordset@@QAEXGG@Z 5f707f7e f   dbcore.obj
 0001:00007041       ?SetRowsetCursorPosition@CRecordset@@QAEXGG@Z 5f708041 f   dbcore.obj
 0001:000070cb       ?BuildSelectSQL@CRecordset@@IAEXXZ 5f7080cb f   dbcore.obj
 0001:00007313       ?AppendFilterAndSortSQL@CRecordset@@IAEXXZ 5f708313 f   dbcore.obj
 0001:0000738c       ?IsRecordsetUpdatable@CRecordset@@IAEHXZ 5f70838c f   dbcore.obj
 0001:00007465       ?ExecuteSetPosUpdate@CRecordset@@IAEXXZ 5f708465 f   dbcore.obj
 0001:00007571       ?PrepareUpdateHstmt@CRecordset@@IAEXXZ 5f708571 f   dbcore.obj
 0001:00007701       ?BuildUpdateSQL@CRecordset@@IAEXXZ 5f708701 f   dbcore.obj
 0001:00007af9       ?ExecuteUpdateSQL@CRecordset@@IAEXXZ 5f708af9 f   dbcore.obj
 0001:00007c9a       ?SendLongBinaryData@CRecordset@@IAEXPAX@Z 5f708c9a f   dbcore.obj
 0001:00007ef7       ?AllocStatusArrays@CRecordset@@QAEXXZ 5f708ef7 f   dbcore.obj
 0001:000080ee       ?GetBoundFieldIndex@CRecordset@@QAEHPAX@Z 5f7090ee f   dbcore.obj
 0001:0000811c       ?GetBoundParamIndex@CRecordset@@QAEHPAX@Z 5f70911c f   dbcore.obj
 0001:0000814a       ?GetFieldIndexByName@CRecordset@@QAEFPBD@Z 5f70914a f   dbcore.obj
 0001:000081d1       ?GetFieldLengthBuffer@CRecordset@@QAEPAJKH@Z 5f7091d1 f   dbcore.obj
 0001:00008255       ?GetFieldStatus@CRecordset@@QAEEK@Z 5f709255 f   dbcore.obj
 0001:0000829c       ?SetFieldStatus@CRecordset@@QAEXKE@Z 5f70929c f   dbcore.obj
 0001:000082f5       ?ClearFieldStatus@CRecordset@@QAEXXZ 5f7092f5 f   dbcore.obj
 0001:0000831b       ?IsFieldStatusDirty@CRecordset@@QBEHK@Z 5f70931b f   dbcore.obj
 0001:00008367       ?SetDirtyFieldStatus@CRecordset@@QAEXK@Z 5f709367 f   dbcore.obj
 0001:000083bf       ?ClearDirtyFieldStatus@CRecordset@@QAEXK@Z 5f7093bf f   dbcore.obj
 0001:00008417       ?IsFieldStatusNull@CRecordset@@QBEHK@Z 5f709417 f   dbcore.obj
 0001:00008463       ?SetNullFieldStatus@CRecordset@@QAEXK@Z 5f709463 f   dbcore.obj
 0001:000084bb       ?ClearNullFieldStatus@CRecordset@@QAEXK@Z 5f7094bb f   dbcore.obj
 0001:00008513       ?IsParamStatusNull@CRecordset@@QBEHK@Z 5f709513 f   dbcore.obj
 0001:0000855f       ?SetNullParamStatus@CRecordset@@QAEXK@Z 5f70955f f   dbcore.obj
 0001:000085b7       ?ClearNullParamStatus@CRecordset@@QAEXK@Z 5f7095b7 f   dbcore.obj
 0001:0000860f       ?IsFieldNullable@CRecordset@@QBEHK@Z 5f70960f f   dbcore.obj
 0001:00008686       ?BindParams@CRecordset@@QAEIPAX@Z 5f709686 f   dbcore.obj
 0001:000086f9       ?RebindParams@CRecordset@@QAEXPAX@Z 5f7096f9 f   dbcore.obj
 0001:00008772       ?BindFieldsToColumns@CRecordset@@QAEIXZ 5f709772 f   dbcore.obj
 0001:0000885b       ?BindFieldsForUpdate@CRecordset@@QAEXXZ 5f70985b f   dbcore.obj
 0001:000088bb       ?UnbindFieldsForUpdate@CRecordset@@QAEXXZ 5f7098bb f   dbcore.obj
 0001:0000891b       ?Fixups@CRecordset@@QAEXXZ 5f70991b f   dbcore.obj
 0001:000089b2       ?AppendNames@CRecordset@@QAEIPAVCString@@PBD@Z 5f7099b2 f   dbcore.obj
 0001:00008aa0       ?AppendNamesValues@CRecordset@@QAEIPAXPAVCString@@PBD@Z 5f709aa0 f   dbcore.obj
 0001:00008b93       ?AppendValues@CRecordset@@QAEIPAXPAVCString@@PBD@Z 5f709b93 f   dbcore.obj
 0001:00008c86       ?StoreFields@CRecordset@@QAEXXZ 5f709c86 f   dbcore.obj
 0001:00008cf1       ?LoadFields@CRecordset@@QAEXXZ 5f709cf1 f   dbcore.obj
 0001:00008d64       ?MarkForUpdate@CRecordset@@QAEXXZ 5f709d64 f   dbcore.obj
 0001:00008da3       ?MarkForAddNew@CRecordset@@QAEXXZ 5f709da3 f   dbcore.obj
 0001:00008de2       ?AllocDataCache@CRecordset@@QAEXXZ 5f709de2 f   dbcore.obj
 0001:00008e21       ?FreeDataCache@CRecordset@@QAEXXZ 5f709e21 f   dbcore.obj
 0001:0000901e       ?DumpFields@CRecordset@@QBEXAAVCDumpContext@@@Z 5f70a01e f   dbcore.obj
 0001:00009052       ?UpdateInsertDelete@CRecordset@@IAEHXZ 5f70a052 f   dbcore.obj
 0001:000093ea       ?GetLBFetchSize@CRecordset@@MAEJJ@Z 5f70a3ea f   dbcore.obj
 0001:000093fc       ?GetLBReallocSize@CRecordset@@MAEJJ@Z 5f70a3fc f   dbcore.obj
 0001:0000940e       ?GetDefaultFieldType@CRecordset@@SGFF@Z 5f70a40e f   dbcore.obj
 0001:00009505       ?GetDataBuffer@CRecordset@@SGPAXAAVCDBVariant@@FPAHFK@Z 5f70a505 f   dbcore.obj
 0001:00009832       ?GetTextLen@CRecordset@@SGHFK@Z 5f70a832 f   dbcore.obj
 0001:000098a4       ?GetData@CRecordset@@SGJPAVCDatabase@@PAXFF1HF@Z 5f70a8a4 f   dbcore.obj
 0001:00009a3e       ?GetLongCharDataAndCleanup@CRecordset@@SGXPAVCDatabase@@PAXFJPAPAXHAAVCString@@F@Z 5f70aa3e f   dbcore.obj
 0001:00009bb0       ?GetLongBinaryDataAndCleanup@CRecordset@@SGXPAVCDatabase@@PAXFJPAPAXHAAVCDBVariant@@F@Z 5f70abb0 f   dbcore.obj
 0001:00009d78       ?AssertValid@CRecordset@@UBEXXZ 5f70ad78 f   dbcore.obj
 0001:00009da5       ?Dump@CRecordset@@UBEXAAVCDumpContext@@@Z 5f70ada5 f   dbcore.obj
 0001:0000a026       ?AfxSetCurrentRecord@@YGXPAJJF@Z 5f70b026 f   dbcore.obj
 0001:0000a04b       ?AfxSetRecordCount@@YGXPAJJJHF@Z 5f70b04b f   dbcore.obj
 0001:0000a08e       ?AfxSetRecordCount@@YGXPAJJHF@Z 5f70b08e f   dbcore.obj
 0001:0000a0d5       ?IsOpen@CDatabase@@QBEHXZ  5f70b0d5 f   dbcore.obj
 0001:0000a0fc       ?CanUpdate@CDatabase@@QBEHXZ 5f70b0fc f   dbcore.obj
 0001:0000a136       ?CanTransact@CDatabase@@QBEHXZ 5f70b136 f   dbcore.obj
 0001:0000a170       ?SetLoginTimeout@CDatabase@@QAEXK@Z 5f70b170 f   dbcore.obj
 0001:0000a196       ?SetQueryTimeout@CDatabase@@QAEXK@Z 5f70b196 f   dbcore.obj
 0001:0000a1bc       ?GetConnect@CDatabase@@QBEABVCString@@XZ 5f70b1bc f   dbcore.obj
 0001:0000a1dd       ?GetBookmarkPersistence@CDatabase@@QBEKXZ 5f70b1dd f   dbcore.obj
 0001:0000a1fe       ?GetCursorCommitBehavior@CDatabase@@QBEHXZ 5f70b1fe f   dbcore.obj
 0001:0000a220       ?GetCursorRollbackBehavior@CDatabase@@QBEHXZ 5f70b220 f   dbcore.obj
 0001:0000a242       ?ThrowDBException@CDatabase@@MAEXF@Z 5f70b242 f   dbcore.obj
 0001:0000a274       ?SetSynchronousMode@CDatabase@@QAEXH@Z 5f70b274 f   dbcore.obj
 0001:0000a2a3       ?GetSQL@CRecordset@@QBEABVCString@@XZ 5f70b2a3 f   dbcore.obj
 0001:0000a2df       ?GetTableName@CRecordset@@QBEABVCString@@XZ 5f70b2df f   dbcore.obj
 0001:0000a31b       ?IsBOF@CRecordset@@QBEHXZ  5f70b31b f   dbcore.obj
 0001:0000a358       ?IsEOF@CRecordset@@QBEHXZ  5f70b358 f   dbcore.obj
 0001:0000a395       ?IsDeleted@CRecordset@@QBEHXZ 5f70b395 f   dbcore.obj
 0001:0000a3d2       ?CanUpdate@CRecordset@@QBEHXZ 5f70b3d2 f   dbcore.obj
 0001:0000a40f       ?CanScroll@CRecordset@@QBEHXZ 5f70b40f f   dbcore.obj
 0001:0000a44c       ?CanAppend@CRecordset@@QBEHXZ 5f70b44c f   dbcore.obj
 0001:0000a489       ?CanRestart@CRecordset@@QBEHXZ 5f70b489 f   dbcore.obj
 0001:0000a4cd       ?CanTransact@CRecordset@@QBEHXZ 5f70b4cd f   dbcore.obj
 0001:0000a50d       ?GetODBCFieldCount@CRecordset@@QBEFXZ 5f70b50d f   dbcore.obj
 0001:0000a548       ?GetRowsetSize@CRecordset@@QBEKXZ 5f70b548 f   dbcore.obj
 0001:0000a585       ?GetRowsFetched@CRecordset@@QBEKXZ 5f70b585 f   dbcore.obj
 0001:0000a5c2       ?GetRowStatus@CRecordset@@QBEGG@Z 5f70b5c2 f   dbcore.obj
 0001:0000a632       ?GetRecordCount@CRecordset@@QBEJXZ 5f70b632 f   dbcore.obj
 0001:0000a66f       ?GetStatus@CRecordset@@QBEXAAUCRecordsetStatus@@@Z 5f70b66f f   dbcore.obj
 0001:0000a6c2       ?ThrowDBException@CRecordset@@UAEXFPAX@Z 5f70b6c2 f   dbcore.obj
 0001:0000a70d       ?MoveNext@CRecordset@@QAEXXZ 5f70b70d f   dbcore.obj
 0001:0000a750       ?MovePrev@CRecordset@@QAEXXZ 5f70b750 f   dbcore.obj
 0001:0000a793       ?MoveFirst@CRecordset@@QAEXXZ 5f70b793 f   dbcore.obj
 0001:0000a7d6       ?MoveLast@CRecordset@@QAEXXZ 5f70b7d6 f   dbcore.obj
 0001:0000a819       ?SetAbsolutePosition@CRecordset@@QAEXJ@Z 5f70b819 f   dbcore.obj
 0001:0000a860       ??_ECDBException@@UAEPAXI@Z 5f70b860 f i dbcore.obj
 0001:0000a860       ??_GCDBException@@UAEPAXI@Z 5f70b860 f i dbcore.obj
 0001:0000a890       ??_GCDatabase@@UAEPAXI@Z   5f70b890 f i dbcore.obj
 0001:0000a8c0       __tcsnicmp                 5f70b8c0 f i dbcore.obj
 0001:0000a8e0       ?T2CA@@YAPBDPBD@Z          5f70b8e0 f i dbcore.obj
 0001:0000a8e0       ?T2A@@YAPADPAD@Z           5f70b8e0 f i dbcore.obj
 0001:0000a8f0       __tcsinc                   5f70b8f0 f i dbcore.obj
 0001:0000a910       ??_GCRecordset@@UAEPAXI@Z  5f70b910 f i dbcore.obj
 0001:0000a910       ??_ECRecordset@@UAEPAXI@Z  5f70b910 f i dbcore.obj
 0001:0000a940       ??_ECODBCFieldInfo@@QAEPAXI@Z 5f70b940 f i dbcore.obj
 0001:0000a9b0       ??1CODBCFieldInfo@@QAE@XZ  5f70b9b0 f i dbcore.obj
 0001:0000a9d0       ??0CODBCFieldInfo@@QAE@XZ  5f70b9d0 f i dbcore.obj
 0001:0000a9f0       __tcsstr                   5f70b9f0 f i dbcore.obj
 0001:0000aa10       ??_GCString@@QAEPAXI@Z     5f70ba10 f i dbcore.obj
 0001:0000aa40       ??_GCNoTrackObject@@UAEPAXI@Z 5f70ba40 f i dbcore.obj
 0001:0000aa40       ??_ECNoTrackObject@@UAEPAXI@Z 5f70ba40 f i dbcore.obj
 0001:0000aa70       ??1CNoTrackObject@@UAE@XZ  5f70ba70 f i dbcore.obj
 0001:0000aa90       ??0CFieldExchange@@QAE@IPAVCRecordset@@PAX@Z 5f70ba90 f   dbrfx.obj
 0001:0000ab6d       ?IsFieldType@CFieldExchange@@QAEHPAI@Z 5f70bb6d f   dbrfx.obj
 0001:0000ac6d       ?Default@CFieldExchange@@QAEXPBDPAXPAJHII@Z 5f70bc6d f   dbrfx.obj
 0001:0000b289       ?RFX_Text@@YGXPAVCFieldExchange@@PBDPADHHF@Z 5f70c289 f   dbrfx.obj
 0001:0000b8be       ?RFX_Text@@YGXPAVCFieldExchange@@PBDAAVCString@@HHF@Z 5f70c8be f   dbrfx.obj
 0001:0000bfce       ?RFX_Int@@YGXPAVCFieldExchange@@PBDAAH@Z 5f70cfce f   dbrfx.obj
 0001:0000c26b       ?RFX_Long@@YGXPAVCFieldExchange@@PBDAAJ@Z 5f70d26b f   dbrfx.obj
 0001:0000c508       ?RFX_Byte@@YGXPAVCFieldExchange@@PBDAAE@Z 5f70d508 f   dbrfx.obj
 0001:0000c7a7       ?RFX_Bool@@YGXPAVCFieldExchange@@PBDAAH@Z 5f70d7a7 f   dbrfx.obj
 0001:0000ca4c       ?RFX_Binary@@YGXPAVCFieldExchange@@PBDAAVCByteArray@@H@Z 5f70da4c f   dbrfx.obj
 0001:0000cf27       ?RFX_Date@@YGXPAVCFieldExchange@@PBDAAVCTime@@@Z 5f70df27 f   dbrfx.obj
 0001:0000dad7       ?RFX_Date@@YGXPAVCFieldExchange@@PBDAAUtagTIMESTAMP_STRUCT@@@Z 5f70ead7 f   dbrfx.obj
 0001:0000e002       ?RFX_Date@@YGXPAVCFieldExchange@@PBDAAVCOleDateTime@@@Z 5f70f002 f   dbrfx.obj
 0001:0000eb1d       ?RFX_LongBinary@@YGXPAVCFieldExchange@@PBDAAVCLongBinary@@@Z 5f70fb1d f   dbrfx.obj
 0001:0000f0e4       ?GetLongBinarySize@CFieldExchange@@QAEJH@Z 5f7100e4 f   dbrfx.obj
 0001:0000f250       ?GetLongBinaryData@CFieldExchange@@QAEXHAAVCLongBinary@@PAJ@Z 5f710250 f   dbrfx.obj
 0001:0000f4db       ?ReallocLongBinary@CFieldExchange@@QAEPAEAAVCLongBinary@@JJ@Z 5f7104db f   dbrfx.obj
 0001:0000f5e0       ?AfxStoreField@@YGXAAVCRecordset@@IPAX@Z 5f7105e0 f   dbrfx.obj
 0001:0000f728       ?AfxLoadField@@YGXAAVCRecordset@@IPAXPAJ@Z 5f710728 f   dbrfx.obj
 0001:0000f834       ?AfxCompareValueByRef@@YGHPAX0H@Z 5f710834 f   dbrfx.obj
 0001:0000fb26       ?AfxCopyValueByRef@@YGXPAX0PAJH@Z 5f710b26 f   dbrfx.obj
 0001:0000fdbb       ?RFX_Text_Bulk@@YGXPAVCFieldExchange@@PBDPAPADPAPAJH@Z 5f710dbb f   dbrfx.obj
 0001:0000ff4b       ?RFX_Bool_Bulk@@YGXPAVCFieldExchange@@PBDPAPAHPAPAJ@Z 5f710f4b f   dbrfx.obj
 0001:000100d8       ?RFX_Int_Bulk@@YGXPAVCFieldExchange@@PBDPAPAHPAPAJ@Z 5f7110d8 f   dbrfx.obj
 0001:00010265       ?RFX_Long_Bulk@@YGXPAVCFieldExchange@@PBDPAPAJ2@Z 5f711265 f   dbrfx.obj
 0001:000103f2       ?RFX_Date_Bulk@@YGXPAVCFieldExchange@@PBDPAPAUtagTIMESTAMP_STRUCT@@PAPAJ@Z 5f7113f2 f   dbrfx.obj
 0001:0001057f       ?RFX_Byte_Bulk@@YGXPAVCFieldExchange@@PBDPAPAEPAPAJ@Z 5f71157f f   dbrfx.obj
 0001:00010709       ?RFX_Binary_Bulk@@YGXPAVCFieldExchange@@PBDPAPAEPAPAJH@Z 5f711709 f   dbrfx.obj
 0001:00010899       ?AfxRFXBulkDefault@@YGXPAVCFieldExchange@@PBDPAXPAJHI@Z 5f711899 f   dbrfx.obj
 0001:00010996       ?SetFieldType@CFieldExchange@@QAEXI@Z 5f711996 f   dbrfx.obj
 0001:000109f0       ?SetLength@CDBByteArray@@QAEXH@Z 5f7119f0 f i dbrfx.obj
 0001:00010a30       ?_GetBaseMessageMap@CRecordView@@KGPBUAFX_MSGMAP@@XZ 5f711a30 f   dbview.obj
 0001:00010a3a       ?GetMessageMap@CRecordView@@MBEPBUAFX_MSGMAP@@XZ 5f711a3a f   dbview.obj
 0001:00010a4a       ??0CRecordView@@IAE@PBD@Z  5f711a4a f   dbview.obj
 0001:00010a6f       ??0CRecordView@@IAE@I@Z    5f711a6f f   dbview.obj
 0001:00010a94       ??1CRecordView@@UAE@XZ     5f711a94 f   dbview.obj
 0001:00010ab0       ?OnInitialUpdate@CRecordView@@UAEXXZ 5f711ab0 f   dbview.obj
 0001:00010b53       ?IsOnFirstRecord@CRecordView@@QAEHXZ 5f711b53 f   dbview.obj
 0001:00010b92       ?IsOnLastRecord@CRecordView@@QAEHXZ 5f711b92 f   dbview.obj
 0001:00010bef       ?OnMove@CRecordView@@UAEHI@Z 5f711bef f   dbview.obj
 0001:00010d19       ?OnUpdateRecordFirst@CRecordView@@IAEXPAVCCmdUI@@@Z 5f711d19 f   dbview.obj
 0001:00010d93       ?OnUpdateRecordPrev@CRecordView@@IAEXPAVCCmdUI@@@Z 5f711d93 f   dbview.obj
 0001:00010dac       ?OnUpdateRecordNext@CRecordView@@IAEXPAVCCmdUI@@@Z 5f711dac f   dbview.obj
 0001:00010e1a       ?OnUpdateRecordLast@CRecordView@@IAEXPAVCCmdUI@@@Z 5f711e1a f   dbview.obj
 0001:00010e94       ?AfxFieldText@@YGHPAVCDataExchange@@HPAXPAVCRecordset@@@Z 5f711e94 f   dbview.obj
 0001:00010fc1       ?DDX_FieldText@@YGXPAVCDataExchange@@HAAHPAVCRecordset@@@Z 5f711fc1 f   dbview.obj
 0001:00010ff2       ?DDX_FieldText@@YGXPAVCDataExchange@@HAAEPAVCRecordset@@@Z 5f711ff2 f   dbview.obj
 0001:00011023       ?DDX_FieldText@@YGXPAVCDataExchange@@HAAIPAVCRecordset@@@Z 5f712023 f   dbview.obj
 0001:00011054       ?DDX_FieldText@@YGXPAVCDataExchange@@HAAJPAVCRecordset@@@Z 5f712054 f   dbview.obj
 0001:00011085       ?DDX_FieldText@@YGXPAVCDataExchange@@HAAKPAVCRecordset@@@Z 5f712085 f   dbview.obj
 0001:000110b6       ?DDX_FieldText@@YGXPAVCDataExchange@@HAAVCString@@PAVCRecordset@@@Z 5f7120b6 f   dbview.obj
 0001:0001126b       ?DDX_FieldText@@YGXPAVCDataExchange@@HPADHPAVCRecordset@@@Z 5f71226b f   dbview.obj
 0001:0001135b       ?DDX_FieldLBString@@YGXPAVCDataExchange@@HAAVCString@@PAVCRecordset@@@Z 5f71235b f   dbview.obj
 0001:000114d6       ?DDX_FieldLBStringExact@@YGXPAVCDataExchange@@HAAVCString@@PAVCRecordset@@@Z 5f7124d6 f   dbview.obj
 0001:000115a0       ?DDX_FieldLBIndex@@YGXPAVCDataExchange@@HAAHPAVCRecordset@@@Z 5f7125a0 f   dbview.obj
 0001:0001160c       ?DDX_FieldCBString@@YGXPAVCDataExchange@@HAAVCString@@PAVCRecordset@@@Z 5f71260c f   dbview.obj
 0001:000117d3       ?DDX_FieldCBStringExact@@YGXPAVCDataExchange@@HAAVCString@@PAVCRecordset@@@Z 5f7127d3 f   dbview.obj
 0001:0001189d       ?DDX_FieldCBIndex@@YGXPAVCDataExchange@@HAAHPAVCRecordset@@@Z 5f71289d f   dbview.obj
 0001:00011909       ?DDX_FieldScroll@@YGXPAVCDataExchange@@HAAHPAVCRecordset@@@Z 5f712909 f   dbview.obj
 0001:00011975       ?DDX_FieldCheck@@YGXPAVCDataExchange@@HAAHPAVCRecordset@@@Z 5f712975 f   dbview.obj
 0001:00011ae2       ?DDX_FieldRadio@@YGXPAVCDataExchange@@HAAHPAVCRecordset@@@Z 5f712ae2 f   dbview.obj
 0001:00011b7d       ?AssertValid@CRecordView@@UBEXXZ 5f712b7d f   dbview.obj
 0001:00011b90       ?Dump@CRecordView@@UBEXAAVCDumpContext@@@Z 5f712b90 f   dbview.obj
 0001:00011bf2       ?OnMove@CRecordView@@IAEXHH@Z 5f712bf2 f   dbview.obj
 0001:00011c10       ??_GCRecordView@@UAEPAXI@Z 5f712c10 f i dbview.obj
 0001:00011c10       ??_ECRecordView@@UAEPAXI@Z 5f712c10 f i dbview.obj
 0001:00011c40       ??1CFormView@@UAE@XZ       5f712c40 f i dbview.obj
 0001:00011c60       ??_9@$BBBE@AE              5f712c60 f i dbview.obj
 0001:00011c70       ?RFX_Single@@YGXPAVCFieldExchange@@PBDAAM@Z 5f712c70 f   dbflt.obj
 0001:00011f1c       ?RFX_Double@@YGXPAVCFieldExchange@@PBDAAN@Z 5f712f1c f   dbflt.obj
 0001:00012204       ?RFX_Single_Bulk@@YGXPAVCFieldExchange@@PBDPAPAMPAPAJ@Z 5f713204 f   dbflt.obj
 0001:0001237d       ?RFX_Double_Bulk@@YGXPAVCFieldExchange@@PBDPAPANPAPAJ@Z 5f71337d f   dbflt.obj
 0001:000124f6       ?DDX_FieldText@@YGXPAVCDataExchange@@HAAMPAVCRecordset@@@Z 5f7134f6 f   dbflt.obj
 0001:00012534       ?DDX_FieldText@@YGXPAVCDataExchange@@HAANPAVCRecordset@@@Z 5f713534 f   dbflt.obj
 0001:00012580       ??0CLongBinary@@QAE@XZ     5f713580 f   dblong.obj
 0001:000125a9       ??1CLongBinary@@UAE@XZ     5f7135a9 f   dblong.obj
 0001:000125e5       ?AssertValid@CLongBinary@@UBEXXZ 5f7135e5 f   dblong.obj
 0001:000125f8       ?Dump@CLongBinary@@UBEXAAVCDumpContext@@@Z 5f7135f8 f   dblong.obj
 0001:00012660       ??_GCLongBinary@@UAEPAXI@Z 5f713660 f i dblong.obj
 0001:00012690       ??0CDBVariant@@QAE@XZ      5f713690 f   dbvar.obj
 0001:000126b1       ?Clear@CDBVariant@@QAEXXZ  5f7136b1 f   dbvar.obj
 0001:00012755       ??1CDBVariant@@UAE@XZ      5f713755 f   dbvar.obj
 0001:00012780       ??_GCDBVariant@@UAEPAXI@Z  5f713780 f i dbvar.obj
 0001:00012780       ??_ECDBVariant@@UAEPAXI@Z  5f713780 f i dbvar.obj
 0001:000127b0       ??0_AFX_DAO_STATE@@QAE@XZ  5f7137b0 f   daocore.obj
 0001:0001281d       ??1_AFX_DAO_STATE@@UAE@XZ  5f71381d f   daocore.obj
 0001:000128e1       ?AfxDaoCheck@@YGXJPBD0HHH@Z 5f7138e1 f   daocore.obj
 0001:00012968       ?AfxDaoTrace@@YGXJPBD0H@Z  5f713968 f   daocore.obj
 0001:000129cc       ?Dump@CDaoErrorInfo@@UBEXAAVCDumpContext@@@Z 5f7139cc f   daocore.obj
 0001:00012a82       ?Dump@CDaoWorkspaceInfo@@UBEXAAVCDumpContext@@@Z 5f713a82 f   daocore.obj
 0001:00012b03       ?Dump@CDaoDatabaseInfo@@UBEXAAVCDumpContext@@@Z 5f713b03 f   daocore.obj
 0001:00012bf0       ?Dump@CDaoTableDefInfo@@UBEXAAVCDumpContext@@@Z 5f713bf0 f   daocore.obj
 0001:00012d41       ?Dump@CDaoFieldInfo@@UBEXAAVCDumpContext@@@Z 5f713d41 f   daocore.obj
 0001:00012ee8       ?Dump@CDaoIndexFieldInfo@@UBEXAAVCDumpContext@@@Z 5f713ee8 f   daocore.obj
 0001:00012f42       ??0CDaoIndexInfo@@QAE@XZ   5f713f42 f   daocore.obj
 0001:00012f81       ??1CDaoIndexInfo@@UAE@XZ   5f713f81 f   daocore.obj
 0001:00013016       ?Dump@CDaoIndexInfo@@UBEXAAVCDumpContext@@@Z 5f714016 f   daocore.obj
 0001:00013180       ?Dump@CDaoRelationFieldInfo@@UBEXAAVCDumpContext@@@Z 5f714180 f   daocore.obj
 0001:000131d9       ??0CDaoRelationInfo@@QAE@XZ 5f7141d9 f   daocore.obj
 0001:0001325f       ??1CDaoRelationInfo@@UAE@XZ 5f71425f f   daocore.obj
 0001:00013312       ?Dump@CDaoRelationInfo@@UBEXAAVCDumpContext@@@Z 5f714312 f   daocore.obj
 0001:0001340e       ?Dump@CDaoQueryDefInfo@@UBEXAAVCDumpContext@@@Z 5f71440e f   daocore.obj
 0001:00013548       ?Dump@CDaoParameterInfo@@UBEXAAVCDumpContext@@@Z 5f714548 f   daocore.obj
 0001:00013611       ?_GetBaseClass@CDaoException@@KGPAUCRuntimeClass@@XZ 5f714611 f   daocore.obj
 0001:0001361b       ?GetRuntimeClass@CDaoException@@UBEPAUCRuntimeClass@@XZ 5f71461b f   daocore.obj
 0001:0001362b       ??0CDaoException@@QAE@XZ   5f71462b f   daocore.obj
 0001:00013668       ??1CDaoException@@UAE@XZ   5f714668 f   daocore.obj
 0001:00013732       ?GetErrorCount@CDaoException@@QAEFXZ 5f714732 f   daocore.obj
 0001:00013795       ?GetErrorInfo@CDaoException@@QAEXH@Z 5f714795 f   daocore.obj
 0001:000138c6       ?GetErrorMessage@CDaoException@@UAEHPADIPAI@Z 5f7148c6 f   daocore.obj
 0001:00013a02       ?InitErrorsCollection@CDaoException@@IAEXXZ 5f714a02 f   daocore.obj
 0001:00013a5e       ?FillErrorInfo@CDaoException@@IAEXXZ 5f714a5e f   daocore.obj
 0001:00013c7f       ?AfxThrowDaoException@@YGXHJ@Z 5f714c7f f   daocore.obj
 0001:00013e21       ?_GetBaseClass@CDaoWorkspace@@KGPAUCRuntimeClass@@XZ 5f714e21 f   daocore.obj
 0001:00013e2b       ?GetRuntimeClass@CDaoWorkspace@@UBEPAUCRuntimeClass@@XZ 5f714e2b f   daocore.obj
 0001:00013e3b       ??0CDaoWorkspace@@QAE@XZ   5f714e3b f   daocore.obj
 0001:00013ed0       ??1CDaoWorkspace@@UAE@XZ   5f714ed0 f   daocore.obj
 0001:00013f6f       ?Create@CDaoWorkspace@@UAEXPBD00@Z 5f714f6f f   daocore.obj
 0001:000140ed       ?Append@CDaoWorkspace@@UAEXXZ 5f7150ed f   daocore.obj
 0001:00014264       ?Open@CDaoWorkspace@@UAEXPBD@Z 5f715264 f   daocore.obj
 0001:0001444e       ?Close@CDaoWorkspace@@UAEXXZ 5f71544e f   daocore.obj
 0001:00014590       ?GetVersion@CDaoWorkspace@@SG?AVCString@@XZ 5f715590 f   daocore.obj
 0001:0001463f       ?GetIniPath@CDaoWorkspace@@SG?AVCString@@XZ 5f71563f f   daocore.obj
 0001:000146ee       ?SetIniPath@CDaoWorkspace@@SGXPBD@Z 5f7156ee f   daocore.obj
 0001:00014782       ?SetDefaultUser@CDaoWorkspace@@SGXPBD@Z 5f715782 f   daocore.obj
 0001:00014816       ?SetDefaultPassword@CDaoWorkspace@@SGXPBD@Z 5f715816 f   daocore.obj
 0001:000148aa       ?GetLoginTimeout@CDaoWorkspace@@SGFXZ 5f7158aa f   daocore.obj
 0001:000148fd       ?SetLoginTimeout@CDaoWorkspace@@SGXF@Z 5f7158fd f   daocore.obj
 0001:0001494d       ?GetName@CDaoWorkspace@@QAE?AVCString@@XZ 5f71594d f   daocore.obj
 0001:00014a26       ?GetUserNameA@CDaoWorkspace@@QAE?AVCString@@XZ 5f715a26 f   daocore.obj
 0001:00014aff       ?SetIsolateODBCTrans@CDaoWorkspace@@QAEXH@Z 5f715aff f   daocore.obj
 0001:00014b7b       ?GetIsolateODBCTrans@CDaoWorkspace@@QAEHXZ 5f715b7b f   daocore.obj
 0001:00014bff       ?CompactDatabase@CDaoWorkspace@@SGXPBD00H0@Z 5f715bff f   daocore.obj
 0001:00014e4c       ?CompactDatabase@CDaoWorkspace@@SGXPBD00H@Z 5f715e4c f   daocore.obj
 0001:00014e6a       ?RepairDatabase@CDaoWorkspace@@SGXPBD@Z 5f715e6a f   daocore.obj
 0001:00014efe       ?Idle@CDaoWorkspace@@SGXH@Z 5f715efe f   daocore.obj
 0001:00014fcd       ?GetWorkspaceCount@CDaoWorkspace@@QAEFXZ 5f715fcd f   daocore.obj
 0001:00015031       ?GetWorkspaceInfo@CDaoWorkspace@@QAEXHAAUCDaoWorkspaceInfo@@K@Z 5f716031 f   daocore.obj
 0001:00015135       ?GetWorkspaceInfo@CDaoWorkspace@@QAEXPBDAAUCDaoWorkspaceInfo@@K@Z 5f716135 f   daocore.obj
 0001:00015239       ?GetDatabaseCount@CDaoWorkspace@@QAEFXZ 5f716239 f   daocore.obj
 0001:0001529d       ?GetDatabaseInfo@CDaoWorkspace@@QAEXHAAUCDaoDatabaseInfo@@K@Z 5f71629d f   daocore.obj
 0001:000153a1       ?GetDatabaseInfo@CDaoWorkspace@@QAEXPBDAAUCDaoDatabaseInfo@@K@Z 5f7163a1 f   daocore.obj
 0001:000154a5       ?BeginTrans@CDaoWorkspace@@QAEXXZ 5f7164a5 f   daocore.obj
 0001:0001553d       ?CommitTrans@CDaoWorkspace@@QAEXXZ 5f71653d f   daocore.obj
 0001:0001566a       ?Rollback@CDaoWorkspace@@QAEXXZ 5f71666a f   daocore.obj
 0001:00015702       ?InitializeEngine@CDaoWorkspace@@KAXXZ 5f716702 f   daocore.obj
 0001:0001570c       ?InitWorkspacesCollection@CDaoWorkspace@@IAEXXZ 5f71670c f   daocore.obj
 0001:00015774       ?FillWorkspaceInfo@CDaoWorkspace@@IAEXPAUDAOWorkspace@@AAUCDaoWorkspaceInfo@@K@Z 5f716774 f   daocore.obj
 0001:000158fe       ?InitDatabasesCollection@CDaoWorkspace@@IAEXXZ 5f7168fe f   daocore.obj
 0001:0001594e       ?FillDatabaseInfo@CDaoWorkspace@@IAEXPAUDAODatabase@@AAUCDaoDatabaseInfo@@K@Z 5f71694e f   daocore.obj
 0001:00015bb9       ?ThrowDaoException@CDaoWorkspace@@MAEXH@Z 5f716bb9 f   daocore.obj
 0001:00015be4       ?AssertValid@CDaoWorkspace@@UBEXXZ 5f716be4 f   daocore.obj
 0001:00015bf7       ?Dump@CDaoWorkspace@@UBEXAAVCDumpContext@@@Z 5f716bf7 f   daocore.obj
 0001:00015c81       ?_GetBaseClass@CDaoDatabase@@KGPAUCRuntimeClass@@XZ 5f716c81 f   daocore.obj
 0001:00015c8b       ?GetRuntimeClass@CDaoDatabase@@UBEPAUCRuntimeClass@@XZ 5f716c8b f   daocore.obj
 0001:00015c9b       ??0CDaoDatabase@@QAE@PAVCDaoWorkspace@@@Z 5f716c9b f   daocore.obj
 0001:00015d67       ??1CDaoDatabase@@UAE@XZ    5f716d67 f   daocore.obj
 0001:00015e52       ?Create@CDaoDatabase@@UAEXPBD0H@Z 5f716e52 f   daocore.obj
 0001:00015fc6       ?Open@CDaoDatabase@@UAEXPBDHH0@Z 5f716fc6 f   daocore.obj
 0001:00016207       ?Close@CDaoDatabase@@UAEXXZ 5f717207 f   daocore.obj
 0001:000163f9       ?CanUpdate@CDaoDatabase@@QAEHXZ 5f7173f9 f   daocore.obj
 0001:000164a3       ?CanTransact@CDaoDatabase@@QAEHXZ 5f7174a3 f   daocore.obj
 0001:0001654d       ?GetName@CDaoDatabase@@QAE?AVCString@@XZ 5f71754d f   daocore.obj
 0001:0001664b       ?GetConnect@CDaoDatabase@@QAE?AVCString@@XZ 5f71764b f   daocore.obj
 0001:00016749       ?GetVersion@CDaoDatabase@@QAE?AVCString@@XZ 5f717749 f   daocore.obj
 0001:00016847       ?GetQueryTimeout@CDaoDatabase@@QAEFXZ 5f717847 f   daocore.obj
 0001:000168e9       ?SetQueryTimeout@CDaoDatabase@@QAEXF@Z 5f7178e9 f   daocore.obj
 0001:00016988       ?GetRecordsAffected@CDaoDatabase@@QAEJXZ 5f717988 f   daocore.obj
 0001:00016a29       ?DeleteTableDef@CDaoDatabase@@QAEXPBD@Z 5f717a29 f   daocore.obj
 0001:00016afa       ?DeleteQueryDef@CDaoDatabase@@QAEXPBD@Z 5f717afa f   daocore.obj
 0001:00016bcb       ?CreateRelation@CDaoDatabase@@QAEXPBD00J00@Z 5f717bcb f   daocore.obj
 0001:00016ca2       ?CreateRelation@CDaoDatabase@@QAEXAAUCDaoRelationInfo@@@Z 5f717ca2 f   daocore.obj
 0001:000172b1       ?DeleteRelation@CDaoDatabase@@QAEXPBD@Z 5f7182b1 f   daocore.obj
 0001:00017382       ?Execute@CDaoDatabase@@QAEXPBDH@Z 5f718382 f   daocore.obj
 0001:0001749c       ?GetTableDefCount@CDaoDatabase@@QAEFXZ 5f71849c f   daocore.obj
 0001:00017500       ?GetTableDefInfo@CDaoDatabase@@QAEXHAAUCDaoTableDefInfo@@K@Z 5f718500 f   daocore.obj
 0001:00017604       ?GetTableDefInfo@CDaoDatabase@@QAEXPBDAAUCDaoTableDefInfo@@K@Z 5f718604 f   daocore.obj
 0001:00017708       ?GetRelationCount@CDaoDatabase@@QAEFXZ 5f718708 f   daocore.obj
 0001:0001776c       ?GetRelationInfo@CDaoDatabase@@QAEXHAAUCDaoRelationInfo@@K@Z 5f71876c f   daocore.obj
 0001:00017870       ?GetRelationInfo@CDaoDatabase@@QAEXPBDAAUCDaoRelationInfo@@K@Z 5f718870 f   daocore.obj
 0001:00017974       ?GetQueryDefCount@CDaoDatabase@@QAEFXZ 5f718974 f   daocore.obj
 0001:000179d8       ?GetQueryDefInfo@CDaoDatabase@@QAEXHAAUCDaoQueryDefInfo@@K@Z 5f7189d8 f   daocore.obj
 0001:00017adc       ?GetQueryDefInfo@CDaoDatabase@@QAEXPBDAAUCDaoQueryDefInfo@@K@Z 5f718adc f   daocore.obj
 0001:00017be0       ?InitWorkspace@CDaoDatabase@@IAEXXZ 5f718be0 f   daocore.obj
 0001:00017cc8       ?InitTableDefsCollection@CDaoDatabase@@IAEXXZ 5f718cc8 f   daocore.obj
 0001:00017d18       ?FillTableDefInfo@CDaoDatabase@@IAEXPAU_DAOTableDef@@AAUCDaoTableDefInfo@@K@Z 5f718d18 f   daocore.obj
 0001:00018044       ?InitRelationsCollection@CDaoDatabase@@IAEXXZ 5f719044 f   daocore.obj
 0001:00018094       ?FillRelationInfo@CDaoDatabase@@IAEXPAU_DAORelation@@AAUCDaoRelationInfo@@K@Z 5f719094 f   daocore.obj
 0001:000185e9       ?InitQueryDefsCollection@CDaoDatabase@@IAEXXZ 5f7195e9 f   daocore.obj
 0001:00018639       ?FillQueryDefInfo@CDaoDatabase@@IAEXPAU_DAOQueryDef@@AAUCDaoQueryDefInfo@@K@Z 5f719639 f   daocore.obj
 0001:000188f9       ?ThrowDaoException@CDaoDatabase@@MAEXH@Z 5f7198f9 f   daocore.obj
 0001:00018924       ?AssertValid@CDaoDatabase@@UBEXXZ 5f719924 f   daocore.obj
 0001:00018937       ?Dump@CDaoDatabase@@UBEXAAVCDumpContext@@@Z 5f719937 f   daocore.obj
 0001:000189a6       ?_GetBaseClass@CDaoTableDef@@KGPAUCRuntimeClass@@XZ 5f7199a6 f   daocore.obj
 0001:000189b0       ?GetRuntimeClass@CDaoTableDef@@UBEPAUCRuntimeClass@@XZ 5f7199b0 f   daocore.obj
 0001:000189c0       ??0CDaoTableDef@@QAE@PAVCDaoDatabase@@@Z 5f7199c0 f   daocore.obj
 0001:00018a1c       ??1CDaoTableDef@@UAE@XZ    5f719a1c f   daocore.obj
 0001:00018a96       ?Create@CDaoTableDef@@UAEXPBDJ00@Z 5f719a96 f   daocore.obj
 0001:00018d2c       ?Append@CDaoTableDef@@UAEXXZ 5f719d2c f   daocore.obj
 0001:00018e94       ?Open@CDaoTableDef@@UAEXPBD@Z 5f719e94 f   daocore.obj
 0001:00019088       ?Close@CDaoTableDef@@UAEXXZ 5f71a088 f   daocore.obj
 0001:0001913b       ?CanUpdate@CDaoTableDef@@QAEHXZ 5f71a13b f   daocore.obj
 0001:000191e5       ?SetName@CDaoTableDef@@QAEXPBD@Z 5f71a1e5 f   daocore.obj
 0001:000192d1       ?GetName@CDaoTableDef@@QAE?AVCString@@XZ 5f71a2d1 f   daocore.obj
 0001:000193cf       ?SetSourceTableName@CDaoTableDef@@QAEXPBD@Z 5f71a3cf f   daocore.obj
 0001:000194bb       ?GetSourceTableName@CDaoTableDef@@QAE?AVCString@@XZ 5f71a4bb f   daocore.obj
 0001:000195b9       ?SetConnect@CDaoTableDef@@QAEXPBD@Z 5f71a5b9 f   daocore.obj
 0001:000196a5       ?GetConnect@CDaoTableDef@@QAE?AVCString@@XZ 5f71a6a5 f   daocore.obj
 0001:000197a3       ?SetAttributes@CDaoTableDef@@QAEXJ@Z 5f71a7a3 f   daocore.obj
 0001:0001984a       ?GetAttributes@CDaoTableDef@@QAEJXZ 5f71a84a f   daocore.obj
 0001:000198eb       ?GetDateCreated@CDaoTableDef@@QAE?AVCOleDateTime@@XZ 5f71a8eb f   daocore.obj
 0001:000199db       ?GetDateLastUpdated@CDaoTableDef@@QAE?AVCOleDateTime@@XZ 5f71a9db f   daocore.obj
 0001:00019acb       ?SetValidationRule@CDaoTableDef@@QAEXPBD@Z 5f71aacb f   daocore.obj
 0001:00019bb7       ?GetValidationRule@CDaoTableDef@@QAE?AVCString@@XZ 5f71abb7 f   daocore.obj
 0001:00019cb5       ?SetValidationText@CDaoTableDef@@QAEXPBD@Z 5f71acb5 f   daocore.obj
 0001:00019da1       ?GetValidationText@CDaoTableDef@@QAE?AVCString@@XZ 5f71ada1 f   daocore.obj
 0001:00019e9f       ?GetRecordCount@CDaoTableDef@@QAEJXZ 5f71ae9f f   daocore.obj
 0001:00019f40       ?CreateField@CDaoTableDef@@QAEXPBDFJJ@Z 5f71af40 f   daocore.obj
 0001:00019fe6       ?CreateField@CDaoTableDef@@QAEXAAUCDaoFieldInfo@@@Z 5f71afe6 f   daocore.obj
 0001:0001a266       ?DeleteField@CDaoTableDef@@QAEXPBD@Z 5f71b266 f   daocore.obj
 0001:0001a331       ?DeleteField@CDaoTableDef@@QAEXH@Z 5f71b331 f   daocore.obj
 0001:0001a3b3       ?CreateIndex@CDaoTableDef@@QAEXAAUCDaoIndexInfo@@@Z 5f71b3b3 f   daocore.obj
 0001:0001a54b       ?DeleteIndex@CDaoTableDef@@QAEXPBD@Z 5f71b54b f   daocore.obj
 0001:0001a616       ?DeleteIndex@CDaoTableDef@@QAEXH@Z 5f71b616 f   daocore.obj
 0001:0001a698       ?GetFieldCount@CDaoTableDef@@QAEFXZ 5f71b698 f   daocore.obj
 0001:0001a6fc       ?GetFieldInfo@CDaoTableDef@@QAEXHAAUCDaoFieldInfo@@K@Z 5f71b6fc f   daocore.obj
 0001:0001a800       ?GetFieldInfo@CDaoTableDef@@QAEXPBDAAUCDaoFieldInfo@@K@Z 5f71b800 f   daocore.obj
 0001:0001a904       ?GetIndexCount@CDaoTableDef@@QAEFXZ 5f71b904 f   daocore.obj
 0001:0001a968       ?GetIndexInfo@CDaoTableDef@@QAEXHAAUCDaoIndexInfo@@K@Z 5f71b968 f   daocore.obj
 0001:0001aa6c       ?GetIndexInfo@CDaoTableDef@@QAEXPBDAAUCDaoIndexInfo@@K@Z 5f71ba6c f   daocore.obj
 0001:0001ab70       ?RefreshLink@CDaoTableDef@@QAEXXZ 5f71bb70 f   daocore.obj
 0001:0001ac08       ?InitFieldsCollection@CDaoTableDef@@IAEXXZ 5f71bc08 f   daocore.obj
 0001:0001ac58       ?InitIndexesCollection@CDaoTableDef@@IAEXXZ 5f71bc58 f   daocore.obj
 0001:0001aca8       ?ThrowDaoException@CDaoTableDef@@MAEXH@Z 5f71bca8 f   daocore.obj
 0001:0001acd3       ?AssertValid@CDaoTableDef@@UBEXXZ 5f71bcd3 f   daocore.obj
 0001:0001ace6       ?Dump@CDaoTableDef@@UBEXAAVCDumpContext@@@Z 5f71bce6 f   daocore.obj
 0001:0001ad55       ?_GetBaseClass@CDaoQueryDef@@KGPAUCRuntimeClass@@XZ 5f71bd55 f   daocore.obj
 0001:0001ad5f       ?GetRuntimeClass@CDaoQueryDef@@UBEPAUCRuntimeClass@@XZ 5f71bd5f f   daocore.obj
 0001:0001ad6f       ??0CDaoQueryDef@@QAE@PAVCDaoDatabase@@@Z 5f71bd6f f   daocore.obj
 0001:0001adcb       ??1CDaoQueryDef@@UAE@XZ    5f71bdcb f   daocore.obj
 0001:0001ae45       ?Create@CDaoQueryDef@@UAEXPBD0@Z 5f71be45 f   daocore.obj
 0001:0001b09a       ?Append@CDaoQueryDef@@UAEXXZ 5f71c09a f   daocore.obj
 0001:0001b202       ?Open@CDaoQueryDef@@UAEXPBD@Z 5f71c202 f   daocore.obj
 0001:0001b3f6       ?Close@CDaoQueryDef@@UAEXXZ 5f71c3f6 f   daocore.obj
 0001:0001b4d0       ?CanUpdate@CDaoQueryDef@@QAEHXZ 5f71c4d0 f   daocore.obj
 0001:0001b559       ?GetName@CDaoQueryDef@@QAE?AVCString@@XZ 5f71c559 f   daocore.obj
 0001:0001b635       ?SetName@CDaoQueryDef@@QAEXPBD@Z 5f71c635 f   daocore.obj
 0001:0001b6fe       ?GetSQL@CDaoQueryDef@@QAE?AVCString@@XZ 5f71c6fe f   daocore.obj
 0001:0001b7da       ?SetSQL@CDaoQueryDef@@QAEXPBD@Z 5f71c7da f   daocore.obj
 0001:0001b8a3       ?GetType@CDaoQueryDef@@QAEFXZ 5f71c8a3 f   daocore.obj
 0001:0001b922       ?GetDateCreated@CDaoQueryDef@@QAE?AVCOleDateTime@@XZ 5f71c922 f   daocore.obj
 0001:0001b9ef       ?GetDateLastUpdated@CDaoQueryDef@@QAE?AVCOleDateTime@@XZ 5f71c9ef f   daocore.obj
 0001:0001babc       ?GetConnect@CDaoQueryDef@@QAE?AVCString@@XZ 5f71cabc f   daocore.obj
 0001:0001bb98       ?SetConnect@CDaoQueryDef@@QAEXPBD@Z 5f71cb98 f   daocore.obj
 0001:0001bc61       ?GetODBCTimeout@CDaoQueryDef@@QAEFXZ 5f71cc61 f   daocore.obj
 0001:0001bce0       ?SetODBCTimeout@CDaoQueryDef@@QAEXF@Z 5f71cce0 f   daocore.obj
 0001:0001bd65       ?GetReturnsRecords@CDaoQueryDef@@QAEHXZ 5f71cd65 f   daocore.obj
 0001:0001bdee       ?SetReturnsRecords@CDaoQueryDef@@QAEXH@Z 5f71cdee f   daocore.obj
 0001:0001be76       ?GetRecordsAffected@CDaoQueryDef@@QAEJXZ 5f71ce76 f   daocore.obj
 0001:0001bef4       ?Execute@CDaoQueryDef@@UAEXH@Z 5f71cef4 f   daocore.obj
 0001:0001bfec       ?GetParamValue@CDaoQueryDef@@UAE?AVCOleVariant@@PBD@Z 5f71cfec f   daocore.obj
 0001:0001c1f4       ?GetParamValue@CDaoQueryDef@@UAE?AVCOleVariant@@H@Z 5f71d1f4 f   daocore.obj
 0001:0001c3fc       ?SetParamValue@CDaoQueryDef@@UAEXPBDABVCOleVariant@@@Z 5f71d3fc f   daocore.obj
 0001:0001c608       ?SetParamValue@CDaoQueryDef@@UAEXHABVCOleVariant@@@Z 5f71d608 f   daocore.obj
 0001:0001c814       ?SetParamValueNull@CDaoQueryDef@@QAEXPBD@Z 5f71d814 f   daocore.obj
 0001:0001c88b       ?SetParamValueNull@CDaoQueryDef@@QAEXH@Z 5f71d88b f   daocore.obj
 0001:0001c902       ?GetFieldCount@CDaoQueryDef@@QAEFXZ 5f71d902 f   daocore.obj
 0001:0001c966       ?GetFieldInfo@CDaoQueryDef@@QAEXHAAUCDaoFieldInfo@@K@Z 5f71d966 f   daocore.obj
 0001:0001ca6a       ?GetFieldInfo@CDaoQueryDef@@QAEXPBDAAUCDaoFieldInfo@@K@Z 5f71da6a f   daocore.obj
 0001:0001cb6e       ?GetParameterCount@CDaoQueryDef@@QAEFXZ 5f71db6e f   daocore.obj
 0001:0001cbd2       ?GetParameterInfo@CDaoQueryDef@@QAEXHAAUCDaoParameterInfo@@K@Z 5f71dbd2 f   daocore.obj
 0001:0001ccd6       ?GetParameterInfo@CDaoQueryDef@@QAEXPBDAAUCDaoParameterInfo@@K@Z 5f71dcd6 f   daocore.obj
 0001:0001cdda       ?InitFieldsCollection@CDaoQueryDef@@IAEXXZ 5f71ddda f   daocore.obj
 0001:0001ce2a       ?InitParametersCollection@CDaoQueryDef@@IAEXXZ 5f71de2a f   daocore.obj
 0001:0001ce7a       ?FillParameterInfo@CDaoQueryDef@@IAEXPAUDAOParameter@@AAUCDaoParameterInfo@@K@Z 5f71de7a f   daocore.obj
 0001:0001d030       ?ThrowDaoException@CDaoQueryDef@@MAEXH@Z 5f71e030 f   daocore.obj
 0001:0001d05b       ?AssertValid@CDaoQueryDef@@UBEXXZ 5f71e05b f   daocore.obj
 0001:0001d06e       ?Dump@CDaoQueryDef@@UBEXAAVCDumpContext@@@Z 5f71e06e f   daocore.obj
 0001:0001d0dd       ?_GetBaseClass@CDaoRecordset@@KGPAUCRuntimeClass@@XZ 5f71e0dd f   daocore.obj
 0001:0001d0e7       ?GetRuntimeClass@CDaoRecordset@@UBEPAUCRuntimeClass@@XZ 5f71e0e7 f   daocore.obj
 0001:0001d0f7       ??0CDaoRecordset@@QAE@PAVCDaoDatabase@@@Z 5f71e0f7 f   daocore.obj
 0001:0001d264       ??1CDaoRecordset@@UAE@XZ   5f71e264 f   daocore.obj
 0001:0001d385       ?Open@CDaoRecordset@@UAEXHPBDH@Z 5f71e385 f   daocore.obj
 0001:0001dd8b       ?Open@CDaoRecordset@@UAEXPAVCDaoQueryDef@@HH@Z 5f71ed8b f   daocore.obj
 0001:0001e075       ?Open@CDaoRecordset@@UAEXPAVCDaoTableDef@@HH@Z 5f71f075 f   daocore.obj
 0001:0001e311       ?Close@CDaoRecordset@@UAEXXZ 5f71f311 f   daocore.obj
 0001:0001e608       ?Requery@CDaoRecordset@@UAEXXZ 5f71f608 f   daocore.obj
 0001:0001e88b       ?GetDefaultDBName@CDaoRecordset@@UAE?AVCString@@XZ 5f71f88b f   daocore.obj
 0001:0001e8cd       ?GetDefaultSQL@CDaoRecordset@@UAE?AVCString@@XZ 5f71f8cd f   daocore.obj
 0001:0001e90f       ?DoFieldExchange@CDaoRecordset@@UAEXPAVCDaoFieldExchange@@@Z 5f71f90f f   daocore.obj
 0001:0001e92f       ?IsBOF@CDaoRecordset@@QBEHXZ 5f71f92f f   daocore.obj
 0001:0001e9b8       ?IsEOF@CDaoRecordset@@QBEHXZ 5f71f9b8 f   daocore.obj
 0001:0001ea41       ?IsDeleted@CDaoRecordset@@QBEHXZ 5f71fa41 f   daocore.obj
 0001:0001ea91       ?CanScroll@CDaoRecordset@@QBEHXZ 5f71fa91 f   daocore.obj
 0001:0001eae1       ?CanUpdate@CDaoRecordset@@QBEHXZ 5f71fae1 f   daocore.obj
 0001:0001eb6a       ?CanAppend@CDaoRecordset@@QBEHXZ 5f71fb6a f   daocore.obj
 0001:0001ebba       ?CanRestart@CDaoRecordset@@QAEHXZ 5f71fbba f   daocore.obj
 0001:0001ec64       ?CanTransact@CDaoRecordset@@QAEHXZ 5f71fc64 f   daocore.obj
 0001:0001eced       ?CanBookmark@CDaoRecordset@@QAEHXZ 5f71fced f   daocore.obj
 0001:0001ed76       ?GetName@CDaoRecordset@@QAE?AVCString@@XZ 5f71fd76 f   daocore.obj
 0001:0001ee74       ?GetType@CDaoRecordset@@QAEFXZ 5f71fe74 f   daocore.obj
 0001:0001ef16       ?GetEditMode@CDaoRecordset@@QAEFXZ 5f71ff16 f   daocore.obj
 0001:0001efbb       ?GetSQL@CDaoRecordset@@QBE?AVCString@@XZ 5f71ffbb f   daocore.obj
 0001:0001f04e       ?GetDateCreated@CDaoRecordset@@QAE?AVCOleDateTime@@XZ 5f72004e f   daocore.obj
 0001:0001f13e       ?GetDateLastUpdated@CDaoRecordset@@QAE?AVCOleDateTime@@XZ 5f72013e f   daocore.obj
 0001:0001f22e       ?GetLastModifiedBookmark@CDaoRecordset@@QAE?AVCOleVariant@@XZ 5f72022e f   daocore.obj
 0001:0001f32c       ?GetValidationRule@CDaoRecordset@@QAE?AVCString@@XZ 5f72032c f   daocore.obj
 0001:0001f42d       ?GetValidationText@CDaoRecordset@@QAE?AVCString@@XZ 5f72042d f   daocore.obj
 0001:0001f52b       ?GetCurrentIndex@CDaoRecordset@@QAE?AVCString@@XZ 5f72052b f   daocore.obj
 0001:0001f629       ?SetCurrentIndex@CDaoRecordset@@QAEXPBD@Z 5f720629 f   daocore.obj
 0001:0001f714       ?GetRecordCount@CDaoRecordset@@QAEJXZ 5f720714 f   daocore.obj
 0001:0001f7b5       ?SetFieldDirty@CDaoRecordset@@QAEXPAXH@Z 5f7207b5 f   daocore.obj
 0001:0001f891       ?IsFieldDirty@CDaoRecordset@@QAEHPAX@Z 5f720891 f   daocore.obj
 0001:0001f989       ?SetFieldNull@CDaoRecordset@@QAEXPAXH@Z 5f720989 f   daocore.obj
 0001:0001faa1       ?IsFieldNull@CDaoRecordset@@QAEHPAX@Z 5f720aa1 f   daocore.obj
 0001:0001fb84       ?IsFieldNullable@CDaoRecordset@@QAEHPAX@Z 5f720b84 f   daocore.obj
 0001:0001fcf7       ?GetFieldCount@CDaoRecordset@@QAEFXZ 5f720cf7 f   daocore.obj
 0001:0001fd5b       ?GetFieldInfo@CDaoRecordset@@QAEXHAAUCDaoFieldInfo@@K@Z 5f720d5b f   daocore.obj
 0001:0001fe5f       ?GetFieldInfo@CDaoRecordset@@QAEXPBDAAUCDaoFieldInfo@@K@Z 5f720e5f f   daocore.obj
 0001:0001ff63       ?GetIndexCount@CDaoRecordset@@QAEFXZ 5f720f63 f   daocore.obj
 0001:0001ffc7       ?GetIndexInfo@CDaoRecordset@@QAEXHAAUCDaoIndexInfo@@K@Z 5f720fc7 f   daocore.obj
 0001:000200cb       ?GetIndexInfo@CDaoRecordset@@QAEXPBDAAUCDaoIndexInfo@@K@Z 5f7210cb f   daocore.obj
 0001:000201cf       ?GetBookmark@CDaoRecordset@@QAE?AVCOleVariant@@XZ 5f7211cf f   daocore.obj
 0001:000202cd       ?SetBookmark@CDaoRecordset@@QAEXVCOleVariant@@@Z 5f7212cd f   daocore.obj
 0001:000203a8       ?GetAbsolutePosition@CDaoRecordset@@QAEJXZ 5f7213a8 f   daocore.obj
 0001:0002044c       ?SetAbsolutePosition@CDaoRecordset@@QAEXJ@Z 5f72144c f   daocore.obj
 0001:000204f5       ?GetPercentPosition@CDaoRecordset@@QAEMXZ 5f7214f5 f   daocore.obj
 0001:00020599       ?SetPercentPosition@CDaoRecordset@@QAEXM@Z 5f721599 f   daocore.obj
 0001:00020642       ?MoveNext@CDaoRecordset@@QAEXXZ 5f721642 f   daocore.obj
 0001:0002066d       ?MovePrev@CDaoRecordset@@QAEXXZ 5f72166d f   daocore.obj
 0001:00020698       ?MoveFirst@CDaoRecordset@@QAEXXZ 5f721698 f   daocore.obj
 0001:000206c6       ?MoveLast@CDaoRecordset@@QAEXXZ 5f7216c6 f   daocore.obj
 0001:000206f4       ?Move@CDaoRecordset@@UAEXJ@Z 5f7216f4 f   daocore.obj
 0001:00020923       ?FindNext@CDaoRecordset@@QAEHPBD@Z 5f721923 f   daocore.obj
 0001:00020954       ?FindPrev@CDaoRecordset@@QAEHPBD@Z 5f721954 f   daocore.obj
 0001:00020985       ?FindFirst@CDaoRecordset@@QAEHPBD@Z 5f721985 f   daocore.obj
 0001:000209b9       ?FindLast@CDaoRecordset@@QAEHPBD@Z 5f7219b9 f   daocore.obj
 0001:000209ed       ?Find@CDaoRecordset@@UAEHJPBD@Z 5f7219ed f   daocore.obj
 0001:00020beb       ?Seek@CDaoRecordset@@QAEHPBDPAVCOleVariant@@11@Z 5f721beb f   daocore.obj
 0001:00020f9c       ?Seek@CDaoRecordset@@QAEHPBDPAVCOleVariant@@G@Z 5f721f9c f   daocore.obj
 0001:00021315       ?CancelUpdate@CDaoRecordset@@UAEXXZ 5f722315 f   daocore.obj
 0001:000213ca       ?SetLockingMode@CDaoRecordset@@QAEXH@Z 5f7223ca f   daocore.obj
 0001:0002146c       ?GetLockingMode@CDaoRecordset@@QAEHXZ 5f72246c f   daocore.obj
 0001:00021516       ?SetCacheStart@CDaoRecordset@@QAEXVCOleVariant@@@Z 5f722516 f   daocore.obj
 0001:000215ec       ?GetCacheStart@CDaoRecordset@@QAE?AVCOleVariant@@XZ 5f7225ec f   daocore.obj
 0001:000216ed       ?SetCacheSize@CDaoRecordset@@QAEXJ@Z 5f7226ed f   daocore.obj
 0001:0002178e       ?GetCacheSize@CDaoRecordset@@QAEJXZ 5f72278e f   daocore.obj
 0001:00021832       ?FillCache@CDaoRecordset@@QAEXPAJPAVCOleVariant@@@Z 5f722832 f   daocore.obj
 0001:000219d7       ?AddNew@CDaoRecordset@@UAEXXZ 5f7229d7 f   daocore.obj
 0001:00021acc       ?Edit@CDaoRecordset@@UAEXXZ 5f722acc f   daocore.obj
 0001:00021bbe       ?Update@CDaoRecordset@@UAEXXZ 5f722bbe f   daocore.obj
 0001:00021cb7       ?Delete@CDaoRecordset@@UAEXXZ 5f722cb7 f   daocore.obj
 0001:00021d86       ?GetFieldValue@CDaoRecordset@@UAE?AVCOleVariant@@PBD@Z 5f722d86 f   daocore.obj
 0001:00021e01       ?GetFieldValue@CDaoRecordset@@UAE?AVCOleVariant@@H@Z 5f722e01 f   daocore.obj
 0001:00021e7c       ?GetFieldValue@CDaoRecordset@@UAEXPBDAAVCOleVariant@@@Z 5f722e7c f   daocore.obj
 0001:00021fa9       ?GetFieldValue@CDaoRecordset@@UAEXHAAVCOleVariant@@@Z 5f722fa9 f   daocore.obj
 0001:000220d6       ?SetFieldValue@CDaoRecordset@@UAEXPBDABVCOleVariant@@@Z 5f7230d6 f   daocore.obj
 0001:0002222d       ?SetFieldValue@CDaoRecordset@@UAEXHABVCOleVariant@@@Z 5f72322d f   daocore.obj
 0001:00022384       ?SetFieldValue@CDaoRecordset@@QAEXHPBD@Z 5f723384 f   daocore.obj
 0001:000223e9       ?SetFieldValue@CDaoRecordset@@QAEXPBD0@Z 5f7233e9 f   daocore.obj
 0001:0002244e       ?SetFieldValueNull@CDaoRecordset@@QAEXPBD@Z 5f72344e f   daocore.obj
 0001:000224c5       ?SetFieldValueNull@CDaoRecordset@@QAEXH@Z 5f7234c5 f   daocore.obj
 0001:0002253c       ?GetParamValue@CDaoRecordset@@UAE?AVCOleVariant@@PBD@Z 5f72353c f   daocore.obj
 0001:000225d8       ?GetParamValue@CDaoRecordset@@UAE?AVCOleVariant@@H@Z 5f7235d8 f   daocore.obj
 0001:00022674       ?SetParamValue@CDaoRecordset@@UAEXPBDABVCOleVariant@@@Z 5f723674 f   daocore.obj
 0001:000226fc       ?SetParamValue@CDaoRecordset@@UAEXHABVCOleVariant@@@Z 5f7236fc f   daocore.obj
 0001:00022784       ?SetParamValueNull@CDaoRecordset@@QAEXPBD@Z 5f723784 f   daocore.obj
 0001:000227fb       ?SetParamValueNull@CDaoRecordset@@QAEXH@Z 5f7237fb f   daocore.obj
 0001:00022872       ?GetFieldLength@CDaoRecordset@@QAEKH@Z 5f723872 f   daocore.obj
 0001:000228ca       ?InitFieldsCollection@CDaoRecordset@@IAEXXZ 5f7238ca f   daocore.obj
 0001:00022949       ?InitIndexesCollection@CDaoRecordset@@IAEXXZ 5f723949 f   daocore.obj
 0001:000229cb       ?BuildSQL@CDaoRecordset@@IAEXXZ 5f7239cb f   daocore.obj
 0001:00022aef       ?AllocDatabase@CDaoRecordset@@IAEXXZ 5f723aef f   daocore.obj
 0001:00022c05       ?BuildSelectList@CDaoRecordset@@IAEXXZ 5f723c05 f   daocore.obj
 0001:00022c7d       ?BuildParameterList@CDaoRecordset@@IAEXXZ 5f723c7d f   daocore.obj
 0001:00022d18       ?BindFields@CDaoRecordset@@IAEXXZ 5f723d18 f   daocore.obj
 0001:00022efd       ?BindParameters@CDaoRecordset@@IAEXXZ 5f723efd f   daocore.obj
 0001:00022f7b       ?Fixup@CDaoRecordset@@IAEXXZ 5f723f7b f   daocore.obj
 0001:00022fba       ?AllocCache@CDaoRecordset@@IAEXXZ 5f723fba f   daocore.obj
 0001:00023080       ?StoreFields@CDaoRecordset@@IAEXXZ 5f724080 f   daocore.obj
 0001:000230fa       ?LoadFields@CDaoRecordset@@IAEXXZ 5f7240fa f   daocore.obj
 0001:00023157       ?FreeCache@CDaoRecordset@@IAEXXZ 5f724157 f   daocore.obj
 0001:00023230       ?MarkForAddNew@CDaoRecordset@@IAEXXZ 5f724230 f   daocore.obj
 0001:0002326f       ?MarkForEdit@CDaoRecordset@@IAEXXZ 5f72426f f   daocore.obj
 0001:000232ae       ?GetFieldIndex@CDaoRecordset@@IAEHPAX@Z 5f7242ae f   daocore.obj
 0001:0002331b       ?SetDirtyFields@CDaoRecordset@@MAEXXZ 5f72431b f   daocore.obj
 0001:0002336b       ?SetCursorAttributes@CDaoRecordset@@QAEXXZ 5f72436b f   daocore.obj
 0001:000233ea       ?GetDataAndFixupNulls@CDaoRecordset@@QAEXXZ 5f7243ea f   daocore.obj
 0001:000234ef       ?IsFieldStatusDirty@CDaoRecordset@@QAEHI@Z 5f7244ef f   daocore.obj
 0001:0002352a       ?SetDirtyFieldStatus@CDaoRecordset@@QAEXI@Z 5f72452a f   daocore.obj
 0001:00023565       ?ClearDirtyFieldStatus@CDaoRecordset@@QAEXI@Z 5f724565 f   daocore.obj
 0001:000235a0       ?IsFieldStatusNull@CDaoRecordset@@QAEHI@Z 5f7245a0 f   daocore.obj
 0001:000235d9       ?SetNullFieldStatus@CDaoRecordset@@QAEXI@Z 5f7245d9 f   daocore.obj
 0001:00023614       ?ClearNullFieldStatus@CDaoRecordset@@QAEXI@Z 5f724614 f   daocore.obj
 0001:0002364f       ?IsFieldStatusNullable@CDaoRecordset@@QAEHI@Z 5f72464f f   daocore.obj
 0001:00023688       ?SetNullableFieldStatus@CDaoRecordset@@QAEXI@Z 5f724688 f   daocore.obj
 0001:000236c3       ?IsFieldStatusNullableKnown@CDaoRecordset@@QAEHI@Z 5f7246c3 f   daocore.obj
 0001:000236fc       ?SetNullableKnownFieldStatus@CDaoRecordset@@QAEXI@Z 5f7246fc f   daocore.obj
 0001:00023737       ?ClearFieldStatusFlags@CDaoRecordset@@QAEXXZ 5f724737 f   daocore.obj
 0001:0002376d       ?IsMatch@CDaoRecordset@@QAEHXZ 5f72476d f   daocore.obj
 0001:000237f1       ?StripBrackets@CDaoRecordset@@SAXPBDPAD@Z 5f7247f1 f   daocore.obj
 0001:00023894       ?ThrowDaoException@CDaoRecordset@@MAEXH@Z 5f724894 f   daocore.obj
 0001:000238bf       ?AssertValid@CDaoRecordset@@UBEXXZ 5f7248bf f   daocore.obj
 0001:000238d2       ?Dump@CDaoRecordset@@UBEXAAVCDumpContext@@@Z 5f7248d2 f   daocore.obj
 0001:00023ae1       ?AfxGetFieldInfo@@YAXPAU_DAOField@@AAUCDaoFieldInfo@@K@Z 5f724ae1 f   daocore.obj
 0001:00023f17       ?AfxSetFieldInfo@@YAXPAU_DAOField@@AAUCDaoFieldInfo@@@Z 5f724f17 f   daocore.obj
 0001:0002418a       ?AfxGetDefaultValue@@YAXPAU_DAOField@@AAVCString@@@Z 5f72518a f   daocore.obj
 0001:00024264       ?AfxSetDefaultValue@@YAXPAU_DAOField@@AAVCString@@@Z 5f725264 f   daocore.obj
 0001:0002435f       ?AfxGetIndexInfo@@YAXPAU_DAOIndex@@AAUCDaoIndexInfo@@K@Z 5f72535f f   daocore.obj
 0001:000245f2       ?AfxSetIndexInfo@@YAXPAU_DAOIndex@@AAUCDaoIndexInfo@@@Z 5f7255f2 f   daocore.obj
 0001:0002471d       ?AfxGetIndexFields@@YAXPAU_DAOIndex@@PAPAUDAOIndexFields@@@Z 5f72571d f   daocore.obj
 0001:00024823       ?AfxGetIndexFieldInfo@@YAXPAU_DAOIndex@@AAUCDaoIndexInfo@@@Z 5f725823 f   daocore.obj
 0001:00024cb3       ?AfxSetIndexFieldInfo@@YAXPAU_DAOIndex@@AAUCDaoIndexInfo@@@Z 5f725cb3 f   daocore.obj
 0001:00024f13       ?ThrowGetRowsDaoException@@YAXJ@Z 5f725f13 f   daocore.obj
 0001:00025119       ?AfxGetDaoState@@YAPAV_AFX_DAO_STATE@@XZ 5f726119 f   daocore.obj
 0001:000251b3       ?AfxDaoInit@@YGXXZ         5f7261b3 f   daocore.obj
 0001:00025441       ?AfxDaoGetEngine@@YGPAU_DAODBEngine@@XZ 5f726441 f   daocore.obj
 0001:0002544e       ?AfxDaoTerm@@YGXXZ         5f72644e f   daocore.obj
 0001:000254fc       ?IsOpen@CDaoWorkspace@@QBEHXZ 5f7264fc f   daocore.obj
 0001:0002551d       ?IsNew@CDaoWorkspace@@QBEHXZ 5f72651d f   daocore.obj
 0001:0002553e       ?IsOpen@CDaoDatabase@@QBEHXZ 5f72653e f   daocore.obj
 0001:0002555f       ?IsOpen@CDaoTableDef@@QBEHXZ 5f72655f f   daocore.obj
 0001:00025580       ?IsOpen@CDaoQueryDef@@QBEHXZ 5f726580 f   daocore.obj
 0001:000255a1       ?IsOpen@CDaoRecordset@@QBEHXZ 5f7265a1 f   daocore.obj
 0001:000255d0       ??_G_AFX_DAO_STATE@@UAEPAXI@Z 5f7265d0 f i daocore.obj
 0001:000255d0       ??_E_AFX_DAO_STATE@@UAEPAXI@Z 5f7265d0 f i daocore.obj
 0001:00025600       ??_ECDaoIndexInfo@@UAEPAXI@Z 5f726600 f i daocore.obj
 0001:00025600       ??_GCDaoIndexInfo@@UAEPAXI@Z 5f726600 f i daocore.obj
 0001:00025630       ??_ECDaoIndexFieldInfo@@QAEPAXI@Z 5f726630 f i daocore.obj
 0001:000256a0       ??1CDaoIndexFieldInfo@@QAE@XZ 5f7266a0 f i daocore.obj
 0001:000256c0       ??_ECDaoRelationInfo@@UAEPAXI@Z 5f7266c0 f i daocore.obj
 0001:000256c0       ??_GCDaoRelationInfo@@UAEPAXI@Z 5f7266c0 f i daocore.obj
 0001:000256f0       ??_ECDaoRelationFieldInfo@@QAEPAXI@Z 5f7266f0 f i daocore.obj
 0001:00025760       ??1CDaoRelationFieldInfo@@QAE@XZ 5f726760 f i daocore.obj
 0001:000257b0       ??_GCDaoException@@UAEPAXI@Z 5f7267b0 f i daocore.obj
 0001:000257e0       ??_GCDaoErrorInfo@@QAEPAXI@Z 5f7267e0 f i daocore.obj
 0001:00025810       ??1CDaoErrorInfo@@QAE@XZ   5f726810 f i daocore.obj
 0001:00025870       ??0CDaoErrorInfo@@QAE@XZ   5f726870 f i daocore.obj
 0001:000258e0       ??_GCDaoWorkspace@@UAEPAXI@Z 5f7268e0 f i daocore.obj
 0001:00025910       ??_GCDaoDatabase@@UAEPAXI@Z 5f726910 f i daocore.obj
 0001:00025940       ??0CDaoRelationFieldInfo@@QAE@XZ 5f726940 f i daocore.obj
 0001:000259a0       ??_ECDaoTableDef@@UAEPAXI@Z 5f7269a0 f i daocore.obj
 0001:000259a0       ??_GCDaoTableDef@@UAEPAXI@Z 5f7269a0 f i daocore.obj
 0001:000259d0       ??0CDaoFieldInfo@@QAE@XZ   5f7269d0 f i daocore.obj
 0001:00025a80       ??1CDaoFieldInfo@@QAE@XZ   5f726a80 f i daocore.obj
 0001:00025b20       ??_ECDaoQueryDef@@UAEPAXI@Z 5f726b20 f i daocore.obj
 0001:00025b20       ??_GCDaoQueryDef@@UAEPAXI@Z 5f726b20 f i daocore.obj
 0001:00025b50       ??_GCDaoRecordset@@UAEPAXI@Z 5f726b50 f i daocore.obj
 0001:00025b80       ??0CDaoIndexFieldInfo@@QAE@XZ 5f726b80 f i daocore.obj
 0001:00025bb0       ??_9@$BEM@AG               5f726bb0 f i daocore.obj
 0001:00025bc0       ??_9@$BHE@AG               5f726bc0 f i daocore.obj
 0001:00025bd0       ??_9@$BHI@AG               5f726bd0 f i daocore.obj
 0001:00025be0       ??0CDaoFieldExchange@@QAE@IPAVCDaoRecordset@@PAX@Z 5f726be0 f   daodfx.obj
 0001:00025c4b       ?IsValidOperation@CDaoFieldExchange@@QAEHXZ 5f726c4b f   daodfx.obj
 0001:00025cc9       ?AppendParamType@CDaoFieldExchange@@SGXAAVCString@@K@Z 5f726cc9 f   daodfx.obj
 0001:00025dfa       ?GetCacheValue@CDaoFieldExchange@@SGPAUCDaoFieldCache@@PAVCDaoRecordset@@PAX@Z 5f726dfa f   daodfx.obj
 0001:00025e2a       ?SetNullValue@CDaoFieldExchange@@SGXPAXK@Z 5f726e2a f   daodfx.obj
 0001:00025f3a       ?IsNullValue@CDaoFieldExchange@@SGHPAXK@Z 5f726f3a f   daodfx.obj
 0001:000260d0       ?AllocCacheValue@CDaoFieldExchange@@SGXAAPAUCDaoFieldCache@@K@Z 5f7270d0 f   daodfx.obj
 0001:000263dc       ?DeleteCacheValue@CDaoFieldExchange@@SGXPAUCDaoFieldCache@@K@Z 5f7273dc f   daodfx.obj
 0001:00026551       ?CopyValue@CDaoFieldExchange@@SGXPAX0K@Z 5f727551 f   daodfx.obj
 0001:000266e8       ?CompareValue@CDaoFieldExchange@@SGHPAX0K@Z 5f7276e8 f   daodfx.obj
 0001:0002693e       ?FillVariant@CDaoFieldExchange@@SGXPAXKPAPAVCOleVariant@@@Z 5f72793e f   daodfx.obj
 0001:00026b83       ?Default@CDaoFieldExchange@@QAEXPBDPAXKK@Z 5f727b83 f   daodfx.obj
 0001:000273a8       ?DFX_Text@@YGXPAVCDaoFieldExchange@@PBDAAVCString@@HK@Z 5f7283a8 f   daodfx.obj
 0001:00027546       ?DFX_Binary@@YGXPAVCDaoFieldExchange@@PBDAAVCByteArray@@HK@Z 5f728546 f   daodfx.obj
 0001:00027657       ?DFX_LongBinary@@YGXPAVCDaoFieldExchange@@PBDAAVCLongBinary@@KK@Z 5f728657 f   daodfx.obj
 0001:000277a2       ?DFX_Bool@@YGXPAVCDaoFieldExchange@@PBDAAHK@Z 5f7287a2 f   daodfx.obj
 0001:000278fe       ?DFX_Byte@@YGXPAVCDaoFieldExchange@@PBDAAEK@Z 5f7288fe f   daodfx.obj
 0001:00027a24       ?DFX_Short@@YGXPAVCDaoFieldExchange@@PBDAAFK@Z 5f728a24 f   daodfx.obj
 0001:00027b4b       ?DFX_Long@@YGXPAVCDaoFieldExchange@@PBDAAJK@Z 5f728b4b f   daodfx.obj
 0001:00027c71       ?DFX_Currency@@YGXPAVCDaoFieldExchange@@PBDAAVCOleCurrency@@K@Z 5f728c71 f   daodfx.obj
 0001:00027df1       ?DFX_Single@@YGXPAVCDaoFieldExchange@@PBDAAMK@Z 5f728df1 f   daodfx.obj
 0001:00027f17       ?DFX_Double@@YGXPAVCDaoFieldExchange@@PBDAANK@Z 5f728f17 f   daodfx.obj
 0001:00028038       ?DFX_DateTime@@YGXPAVCDaoFieldExchange@@PBDAAVCOleDateTime@@K@Z 5f729038 f   daodfx.obj
 0001:000281b8       _DaoStringAllocCallback@12 5f7291b8 f   daodfx.obj
 0001:00028279       _DaoBinaryAllocCallback@12 5f729279 f   daodfx.obj
 0001:00028345       _DaoLongBinaryAllocCallback@12 5f729345 f   daodfx.obj
 0001:0002843e       ?AllocLongBinary@@YAXAAVCLongBinary@@K@Z 5f72943e f   daodfx.obj
 0001:000284c8       ?SetFieldType@CDaoFieldExchange@@QAEXI@Z 5f7294c8 f   daodfx.obj
 0001:00028510       ??_GCOleVariant@@QAEPAXI@Z 5f729510 f i daodfx.obj
 0001:00028540       ?_GetBaseClass@CDaoRecordView@@KGPAUCRuntimeClass@@XZ 5f729540 f   daoview.obj
 0001:0002854a       ?GetRuntimeClass@CDaoRecordView@@UBEPAUCRuntimeClass@@XZ 5f72954a f   daoview.obj
 0001:0002855a       ?_GetBaseMessageMap@CDaoRecordView@@KGPBUAFX_MSGMAP@@XZ 5f72955a f   daoview.obj
 0001:00028564       ?GetMessageMap@CDaoRecordView@@MBEPBUAFX_MSGMAP@@XZ 5f729564 f   daoview.obj
 0001:00028574       ??0CDaoRecordView@@IAE@PBD@Z 5f729574 f   daoview.obj
 0001:00028638       ??0CDaoRecordView@@IAE@I@Z 5f729638 f   daoview.obj
 0001:000286fc       ??1CDaoRecordView@@UAE@XZ  5f7296fc f   daoview.obj
 0001:00028777       ?OnInitialUpdate@CDaoRecordView@@UAEXXZ 5f729777 f   daoview.obj
 0001:00028952       ?OnMove@CDaoRecordView@@UAEHI@Z 5f729952 f   daoview.obj
 0001:00028ea4       ?IsOnFirstRecord@CDaoRecordView@@QAEHXZ 5f729ea4 f   daoview.obj
 0001:00028eda       ?IsOnLastRecord@CDaoRecordView@@QAEHXZ 5f729eda f   daoview.obj
 0001:00028f10       ?AfxFieldText@@YGHPAVCDataExchange@@HPAXPAVCDaoRecordset@@@Z 5f729f10 f   daoview.obj
 0001:00028ff5       ?DDX_FieldText@@YGXPAVCDataExchange@@HAAHPAVCDaoRecordset@@@Z 5f729ff5 f   daoview.obj
 0001:00029026       ?DDX_FieldText@@YGXPAVCDataExchange@@HAAEPAVCDaoRecordset@@@Z 5f72a026 f   daoview.obj
 0001:00029057       ?DDX_FieldText@@YGXPAVCDataExchange@@HAAFPAVCDaoRecordset@@@Z 5f72a057 f   daoview.obj
 0001:00029088       ?DDX_FieldText@@YGXPAVCDataExchange@@HAAJPAVCDaoRecordset@@@Z 5f72a088 f   daoview.obj
 0001:000290b9       ?DDX_FieldText@@YGXPAVCDataExchange@@HAAKPAVCDaoRecordset@@@Z 5f72a0b9 f   daoview.obj
 0001:000290ea       ?DDX_FieldText@@YGXPAVCDataExchange@@HAAVCOleCurrency@@PAVCDaoRecordset@@@Z 5f72a0ea f   daoview.obj
 0001:0002911b       ?DDX_FieldText@@YGXPAVCDataExchange@@HAAMPAVCDaoRecordset@@@Z 5f72a11b f   daoview.obj
 0001:0002914c       ?DDX_FieldText@@YGXPAVCDataExchange@@HAANPAVCDaoRecordset@@@Z 5f72a14c f   daoview.obj
 0001:0002917d       ?DDX_FieldText@@YGXPAVCDataExchange@@HAAVCOleDateTime@@PAVCDaoRecordset@@@Z 5f72a17d f   daoview.obj
 0001:000291ae       ?DDX_FieldText@@YGXPAVCDataExchange@@HAAVCString@@PAVCDaoRecordset@@@Z 5f72a1ae f   daoview.obj
 0001:000291df       ?DDX_FieldText@@YGXPAVCDataExchange@@HPADHPAVCDaoRecordset@@@Z 5f72a1df f   daoview.obj
 0001:00029214       ?DDX_FieldLBString@@YGXPAVCDataExchange@@HAAVCString@@PAVCDaoRecordset@@@Z 5f72a214 f   daoview.obj
 0001:0002936e       ?DDX_FieldLBStringExact@@YGXPAVCDataExchange@@HAAVCString@@PAVCDaoRecordset@@@Z 5f72a36e f   daoview.obj
 0001:00029438       ?DDX_FieldCBString@@YGXPAVCDataExchange@@HAAVCString@@PAVCDaoRecordset@@@Z 5f72a438 f   daoview.obj
 0001:00029586       ?DDX_FieldCBStringExact@@YGXPAVCDataExchange@@HAAVCString@@PAVCDaoRecordset@@@Z 5f72a586 f   daoview.obj
 0001:00029650       ?DDX_FieldLBIndex@@YGXPAVCDataExchange@@HAAHPAVCDaoRecordset@@@Z 5f72a650 f   daoview.obj
 0001:000296bc       ?DDX_FieldCBIndex@@YGXPAVCDataExchange@@HAAHPAVCDaoRecordset@@@Z 5f72a6bc f   daoview.obj
 0001:00029728       ?DDX_FieldScroll@@YGXPAVCDataExchange@@HAAHPAVCDaoRecordset@@@Z 5f72a728 f   daoview.obj
 0001:00029794       ?DDX_FieldSlider@@YGXPAVCDataExchange@@HAAHPAVCDaoRecordset@@@Z 5f72a794 f   daoview.obj
 0001:00029800       ?DDX_FieldCheck@@YGXPAVCDataExchange@@HAAHPAVCDaoRecordset@@@Z 5f72a800 f   daoview.obj
 0001:0002996d       ?DDX_FieldRadio@@YGXPAVCDataExchange@@HAAHPAVCDaoRecordset@@@Z 5f72a96d f   daoview.obj
 0001:00029a08       ?AssertValid@CDaoRecordView@@UBEXXZ 5f72aa08 f   daoview.obj
 0001:00029a1b       ?Dump@CDaoRecordView@@UBEXAAVCDumpContext@@@Z 5f72aa1b f   daoview.obj
 0001:00029b5c       ?OnUpdateRecordFirst@CDaoRecordView@@IAEXPAVCCmdUI@@@Z 5f72ab5c f   daoview.obj
 0001:00029b90       ?OnUpdateRecordNext@CDaoRecordView@@IAEXPAVCCmdUI@@@Z 5f72ab90 f   daoview.obj
 0001:00029bc4       ?OnUpdateRecordPrev@CDaoRecordView@@IAEXPAVCCmdUI@@@Z 5f72abc4 f   daoview.obj
 0001:00029bf8       ?OnUpdateRecordLast@CDaoRecordView@@IAEXPAVCCmdUI@@@Z 5f72abf8 f   daoview.obj
 0001:00029c2c       ?OnMove@CDaoRecordView@@IAEXHH@Z 5f72ac2c f   daoview.obj
 0001:00029c50       ??_ECDaoRecordView@@UAEPAXI@Z 5f72ac50 f i daoview.obj
 0001:00029c50       ??_GCDaoRecordView@@UAEPAXI@Z 5f72ac50 f i daoview.obj
 0001:00029c80       ??_Estringdispid@CComTypeInfoHolder@ATL@@QAEPAXI@Z 5f72ac80 f i viewoled.obj
 0001:00029cf0       ??1stringdispid@CComTypeInfoHolder@ATL@@QAE@XZ 5f72acf0 f i viewoled.obj
 0001:00029d10       ??1CComBSTR@ATL@@QAE@XZ    5f72ad10 f i viewoled.obj
 0001:00029d30       ?MovePrev@CRowset@ATL@@QAEJXZ 5f72ad30 f i viewoled.obj
 0001:00029d50       ?MoveNext@CRowset@ATL@@QAEJXZ 5f72ad50 f i viewoled.obj
 0001:00029d70       ?MoveNext@CRowset@ATL@@QAEJJ_N@Z 5f72ad70 f i viewoled.obj
 0001:00029e80       ?AtlTrace2@ATL@@YAXKIPBDZZ 5f72ae80 f i viewoled.obj
 0001:00029f30       ?ReleaseRows@CRowset@ATL@@QAEJXZ 5f72af30 f i viewoled.obj
 0001:00029fc0       ?MoveFirst@CRowset@ATL@@QAEJXZ 5f72afc0 f i viewoled.obj
 0001:0002a070       ?MoveLast@CRowset@ATL@@QAEJXZ 5f72b070 f i viewoled.obj
 0001:0002a180       ?GetData@CRowset@ATL@@QAEJXZ 5f72b180 f i viewoled.obj
 0001:0002a230       ?GetNumAccessors@CAccessorBase@ATL@@QBEKXZ 5f72b230 f i viewoled.obj
 0001:0002a250       ?IsAutoAccessor@CAccessorBase@ATL@@QBE_NK@Z 5f72b250 f i viewoled.obj
 0001:0002a2e0       ?GetData@CRowset@ATL@@QAEJH@Z 5f72b2e0 f i viewoled.obj
 0001:0002a3d0       ?GetHAccessor@CAccessorBase@ATL@@QBEKK@Z 5f72b3d0 f i viewoled.obj
 0001:0002a430       ?GetBuffer@CAccessorBase@ATL@@QBEPAEXZ 5f72b430 f i viewoled.obj
 0001:0002a450       ?SetData@CRowset@ATL@@QBEJH@Z 5f72b450 f i viewoled.obj
 0001:0002a4f2       ?AfxGetModuleState@@YGPAVAFX_MODULE_STATE@@XZ 5f72b4f2 f   MFC42D:MFC42D.DLL
 0001:0002a4f8       ?AfxTermThread@@YGXPAUHINSTANCE__@@@Z 5f72b4f8 f   MFC42D:MFC42D.DLL
 0001:0002a4fe       ?AfxTermExtensionModule@@YGXAAUAFX_EXTENSION_MODULE@@H@Z 5f72b4fe f   MFC42D:MFC42D.DLL
 0001:0002a504       ??0CDynLinkLibrary@@QAE@AAUAFX_EXTENSION_MODULE@@H@Z 5f72b504 f   MFC42D:MFC42D.DLL
 0001:0002a50a       ??2CObject@@SGPAXI@Z       5f72b50a f   MFC42D:MFC42D.DLL
 0001:0002a510       ?AfxAssertFailedLine@@YGHPBDH@Z 5f72b510 f   MFC42D:MFC42D.DLL
 0001:0002a516       ?AfxInitExtensionModule@@YGHAAUAFX_EXTENSION_MODULE@@PAUHINSTANCE__@@@Z 5f72b516 f   MFC42D:MFC42D.DLL
 0001:0002a51c       ??3CObject@@SGXPAX@Z       5f72b51c f   MFC42D:MFC42D.DLL
 0001:0002a522       ?AfxGetAppModuleState@@YGPAVAFX_MODULE_STATE@@XZ 5f72b522 f   MFC42D:MFC42D.DLL
 0001:0002a528       ??3@YAXPAX@Z               5f72b528 f   MFC42D:MFC42D.DLL
 0001:0002a52e       ??2@YAPAXI@Z               5f72b52e f   MFC42D:MFC42D.DLL
 0001:0002a534       ??3CException@@SGXPAX@Z    5f72b534 f   MFC42D:MFC42D.DLL
 0001:0002a53a       ??3CException@@SGXPAXPBDH@Z 5f72b53a f   MFC42D:MFC42D.DLL
 0001:0002a540       ?AfxTrace@@YAXPBDZZ        5f72b540 f   MFC42D:MFC42D.DLL
 0001:0002a546       ?LoadStringA@CString@@QAEHI@Z 5f72b546 f   MFC42D:MFC42D.DLL
 0001:0002a54c       ??2CObject@@SGPAXIPBDH@Z   5f72b54c f   MFC42D:MFC42D.DLL
 0001:0002a552       ?ReportError@CException@@UAEHII@Z 5f72b552 f   MFC42D:MFC42D.DLL
 0001:0002a558       ?Dump@CObject@@UBEXAAVCDumpContext@@@Z 5f72b558 f   MFC42D:MFC42D.DLL
 0001:0002a55e       ?AssertValid@CObject@@UBEXXZ 5f72b55e f   MFC42D:MFC42D.DLL
 0001:0002a564       ?Serialize@CObject@@UAEXAAVCArchive@@@Z 5f72b564 f   MFC42D:MFC42D.DLL
 0001:0002a56a       ??1CString@@QAE@XZ         5f72b56a f   MFC42D:MFC42D.DLL
 0001:0002a570       ??1CException@@UAE@XZ      5f72b570 f   MFC42D:MFC42D.DLL
 0001:0002a576       ??0CString@@QAE@XZ         5f72b576 f   MFC42D:MFC42D.DLL
 0001:0002a57c       ??0CException@@QAE@XZ      5f72b57c f   MFC42D:MFC42D.DLL
 0001:0002a582       ??H@YG?AVCString@@ABV0@PBD@Z 5f72b582 f   MFC42D:MFC42D.DLL
 0001:0002a588       ??H@YG?AVCString@@PBDABV0@@Z 5f72b588 f   MFC42D:MFC42D.DLL
 0001:0002a58e       ??4CString@@QAEABV0@ABV0@@Z 5f72b58e f   MFC42D:MFC42D.DLL
 0001:0002a594       ?Right@CString@@QBE?AV1@H@Z 5f72b594 f   MFC42D:MFC42D.DLL
 0001:0002a59a       ?GetLength@CString@@QBEHXZ 5f72b59a f   MFC42D:MFC42D.DLL
 0001:0002a5a0       ??YCString@@QAEABV0@ABV0@@Z 5f72b5a0 f   MFC42D:MFC42D.DLL
 0001:0002a5a6       ?Left@CString@@QBE?AV1@H@Z 5f72b5a6 f   MFC42D:MFC42D.DLL
 0001:0002a5ac       ?Find@CString@@QBEHD@Z     5f72b5ac f   MFC42D:MFC42D.DLL
 0001:0002a5b2       ??ACString@@QBEDH@Z        5f72b5b2 f   MFC42D:MFC42D.DLL
 0001:0002a5b8       ?IsEmpty@CString@@QBEHXZ   5f72b5b8 f   MFC42D:MFC42D.DLL
 0001:0002a5be       ??YCString@@QAEABV0@PBD@Z  5f72b5be f   MFC42D:MFC42D.DLL
 0001:0002a5c4       ??BCString@@QBEPBDXZ       5f72b5c4 f   MFC42D:MFC42D.DLL
 0001:0002a5ca       ??4CString@@QAEABV0@PBE@Z  5f72b5ca f   MFC42D:MFC42D.DLL
 0001:0002a5d0       ?AfxAssertValidObject@@YGXPBVCObject@@PBDH@Z 5f72b5d0 f   MFC42D:MFC42D.DLL
 0001:0002a5d6       ?AfxIsValidString@@YGHPBDH@Z 5f72b5d6 f   MFC42D:MFC42D.DLL
 0001:0002a5dc       ??0CString@@QAE@PBD@Z      5f72b5dc f   MFC42D:MFC42D.DLL
 0001:0002a5e2       ?Empty@CString@@QAEXXZ     5f72b5e2 f   MFC42D:MFC42D.DLL
 0001:0002a5e8       ??1CObject@@UAE@XZ         5f72b5e8 f   MFC42D:MFC42D.DLL
 0001:0002a5ee       ??0CPtrList@@QAE@H@Z       5f72b5ee f   MFC42D:MFC42D.DLL
 0001:0002a5f4       ??0CObject@@IAE@XZ         5f72b5f4 f   MFC42D:MFC42D.DLL
 0001:0002a5fa       ??1CPtrList@@UAE@XZ        5f72b5fa f   MFC42D:MFC42D.DLL
 0001:0002a600       ??4CString@@QAEABV0@PBD@Z  5f72b600 f   MFC42D:MFC42D.DLL
 0001:0002a606       ?IsKindOf@CObject@@QBEHPBUCRuntimeClass@@@Z 5f72b606 f   MFC42D:MFC42D.DLL
 0001:0002a60c       ?AfxUnlockGlobals@@YGXH@Z  5f72b60c f   MFC42D:MFC42D.DLL
 0001:0002a612       ?GetHead@CPtrList@@QAEAAPAXXZ 5f72b612 f   MFC42D:MFC42D.DLL
 0001:0002a618       ?IsEmpty@CPtrList@@QBEHXZ  5f72b618 f   MFC42D:MFC42D.DLL
 0001:0002a61e       ?AfxLockGlobals@@YGXH@Z    5f72b61e f   MFC42D:MFC42D.DLL
 0001:0002a624       ?Delete@CException@@QAEXXZ 5f72b624 f   MFC42D:MFC42D.DLL
 0001:0002a62a       ?AfxThrowMemoryException@@YGXXZ 5f72b62a f   MFC42D:MFC42D.DLL
 0001:0002a630       ?GetSafeOwner_@CWnd@@SGPAUHWND__@@PAU2@PAPAU2@@Z 5f72b630 f   MFC42D:MFC42D.DLL
 0001:0002a636       ?GetDepth@CDumpContext@@QBEHXZ 5f72b636 f   MFC42D:MFC42D.DLL
 0001:0002a63c       ??6CDumpContext@@QAEAAV0@K@Z 5f72b63c f   MFC42D:MFC42D.DLL
 0001:0002a642       ??6CDumpContext@@QAEAAV0@H@Z 5f72b642 f   MFC42D:MFC42D.DLL
 0001:0002a648       ??6@YGAAVCDumpContext@@AAV0@ABVCString@@@Z 5f72b648 f   MFC42D:MFC42D.DLL
 0001:0002a64e       ??6CDumpContext@@QAEAAV0@PBX@Z 5f72b64e f   MFC42D:MFC42D.DLL
 0001:0002a654       ??6CDumpContext@@QAEAAV0@PBD@Z 5f72b654 f   MFC42D:MFC42D.DLL
 0001:0002a65a       ??1CMapPtrToPtr@@UAE@XZ    5f72b65a f   MFC42D:MFC42D.DLL
 0001:0002a660       ?AddHead@CPtrList@@QAEPAU__POSITION@@PAX@Z 5f72b660 f   MFC42D:MFC42D.DLL
 0001:0002a666       ?AfxIsValidAddress@@YGHPBXIH@Z 5f72b666 f   MFC42D:MFC42D.DLL
 0001:0002a66c       ??0CMapPtrToPtr@@QAE@H@Z   5f72b66c f   MFC42D:MFC42D.DLL
 0001:0002a672       ?RemoveAt@CPtrList@@QAEXPAU__POSITION@@@Z 5f72b672 f   MFC42D:MFC42D.DLL
 0001:0002a678       ?Find@CPtrList@@QBEPAU__POSITION@@PAXPAU2@@Z 5f72b678 f   MFC42D:MFC42D.DLL
 0001:0002a67e       ?Find@CString@@QBEHPBD@Z   5f72b67e f   MFC42D:MFC42D.DLL
 0001:0002a684       ??2@YAPAXIPBDH@Z           5f72b684 f   MFC42D:MFC42D.DLL
 0001:0002a68a       ?GetBufferSetLength@CString@@QAEPADH@Z 5f72b68a f   MFC42D:MFC42D.DLL
 0001:0002a690       ??9@YG_NABVCString@@0@Z    5f72b690 f   MFC42D:MFC42D.DLL
 0001:0002a696       ??3CObject@@SGXPAXPBDH@Z   5f72b696 f   MFC42D:MFC42D.DLL
 0001:0002a69c       ?ReleaseBuffer@CString@@QAEXH@Z 5f72b69c f   MFC42D:MFC42D.DLL
 0001:0002a6a2       ?GetBuffer@CString@@QAEPADH@Z 5f72b6a2 f   MFC42D:MFC42D.DLL
 0001:0002a6a8       ??3@YAXPAXPBDH@Z           5f72b6a8 f   MFC42D:MFC42D.DLL
 0001:0002a6ae       ?MakeUpper@CString@@QAEXXZ 5f72b6ae f   MFC42D:MFC42D.DLL
 0001:0002a6b4       ?SetAt@CString@@QAEXHD@Z   5f72b6b4 f   MFC42D:MFC42D.DLL
 0001:0002a6ba       ?Lookup@CMapPtrToPtr@@QBEHPAXAAPAX@Z 5f72b6ba f   MFC42D:MFC42D.DLL
 0001:0002a6c0       ??8@YG_NABVCString@@PBD@Z  5f72b6c0 f   MFC42D:MFC42D.DLL
 0001:0002a6c6       ??6CDumpContext@@QAEAAV0@PBVCObject@@@Z 5f72b6c6 f   MFC42D:MFC42D.DLL
 0001:0002a6cc       ??6CDumpContext@@QAEAAV0@J@Z 5f72b6cc f   MFC42D:MFC42D.DLL
 0001:0002a6d2       ??6CDumpContext@@QAEAAV0@I@Z 5f72b6d2 f   MFC42D:MFC42D.DLL
 0001:0002a6d8       ??1CProcessLocalObject@@QAE@XZ 5f72b6d8 f   MFC42D:MFC42D.DLL
 0001:0002a6de       ?GetData@CProcessLocalObject@@QAEPAVCNoTrackObject@@P6GPAV2@XZ@Z 5f72b6de f   MFC42D:MFC42D.DLL
 0001:0002a6e4       ??3CNoTrackObject@@SGXPAX@Z 5f72b6e4 f   MFC42D:MFC42D.DLL
 0001:0002a6ea       ??2CNoTrackObject@@SGPAXI@Z 5f72b6ea f   MFC42D:MFC42D.DLL
 0001:0002a6f0       ?GetData@CByteArray@@QAEPAEXZ 5f72b6f0 f   MFC42D:MFC42D.DLL
 0001:0002a6f6       ??YCString@@QAEABV0@D@Z    5f72b6f6 f   MFC42D:MFC42D.DLL
 0001:0002a6fc       ?SetAt@CMapPtrToPtr@@QAEXPAX0@Z 5f72b6fc f   MFC42D:MFC42D.DLL
 0001:0002a702       ?LockBuffer@CString@@QAEPADXZ 5f72b702 f   MFC42D:MFC42D.DLL
 0001:0002a708       ??6CDumpContext@@QAEAAV0@E@Z 5f72b708 f   MFC42D:MFC42D.DLL
 0001:0002a70e       ??0CByteArray@@QAE@XZ      5f72b70e f   MFC42D:MFC42D.DLL
 0001:0002a714       ?SetSize@CByteArray@@QAEXHH@Z 5f72b714 f   MFC42D:MFC42D.DLL
 0001:0002a71a       ??ACByteArray@@QAEAAEH@Z   5f72b71a f   MFC42D:MFC42D.DLL
 0001:0002a720       ?GetSize@CByteArray@@QBEHXZ 5f72b720 f   MFC42D:MFC42D.DLL
 0001:0002a726       ??6@YGAAVCDumpContext@@AAV0@VCTime@@@Z 5f72b726 f   MFC42D:MFC42D.DLL
 0001:0002a72c       ??0CTime@@QAE@XZ           5f72b72c f   MFC42D:MFC42D.DLL
 0001:0002a732       ??9CTime@@QBEHV0@@Z        5f72b732 f   MFC42D:MFC42D.DLL
 0001:0002a738       ??0CTime@@QAE@ABV0@@Z      5f72b738 f   MFC42D:MFC42D.DLL
 0001:0002a73e       ??0CTime@@QAE@HHHHHHH@Z    5f72b73e f   MFC42D:MFC42D.DLL
 0001:0002a744       ??4CTime@@QAEABV0@ABV0@@Z  5f72b744 f   MFC42D:MFC42D.DLL
 0001:0002a74a       ??0CTime@@QAE@J@Z          5f72b74a f   MFC42D:MFC42D.DLL
 0001:0002a750       ?GetSecond@CTime@@QBEHXZ   5f72b750 f   MFC42D:MFC42D.DLL
 0001:0002a756       ?GetMinute@CTime@@QBEHXZ   5f72b756 f   MFC42D:MFC42D.DLL
 0001:0002a75c       ?GetHour@CTime@@QBEHXZ     5f72b75c f   MFC42D:MFC42D.DLL
 0001:0002a762       ?GetDay@CTime@@QBEHXZ      5f72b762 f   MFC42D:MFC42D.DLL
 0001:0002a768       ?GetMonth@CTime@@QBEHXZ    5f72b768 f   MFC42D:MFC42D.DLL
 0001:0002a76e       ?GetYear@CTime@@QBEHXZ     5f72b76e f   MFC42D:MFC42D.DLL
 0001:0002a774       ??6CDumpContext@@QAEAAV0@G@Z 5f72b774 f   MFC42D:MFC42D.DLL
 0001:0002a77a       ??8CTime@@QBEHV0@@Z        5f72b77a f   MFC42D:MFC42D.DLL
 0001:0002a780       ??8@YG_NABVCString@@0@Z    5f72b780 f   MFC42D:MFC42D.DLL
 0001:0002a786       ?Copy@CByteArray@@QAEXABV1@@Z 5f72b786 f   MFC42D:MFC42D.DLL
 0001:0002a78c       ?OnEndPrintPreview@CView@@MAEXPAVCDC@@PAUCPrintInfo@@UtagPOINT@@PAVCPreviewView@@@Z 5f72b78c f   MFC42D:MFC42D.DLL
 0001:0002a792       ?OnEndPrinting@CView@@MAEXPAVCDC@@PAUCPrintInfo@@@Z 5f72b792 f   MFC42D:MFC42D.DLL
 0001:0002a798       ?OnPrint@CView@@MAEXPAVCDC@@PAUCPrintInfo@@@Z 5f72b798 f   MFC42D:MFC42D.DLL
 0001:0002a79e       ?OnBeginPrinting@CView@@MAEXPAVCDC@@PAUCPrintInfo@@@Z 5f72b79e f   MFC42D:MFC42D.DLL
 0001:0002a7a4       ?OnPreparePrinting@CView@@MAEHPAUCPrintInfo@@@Z 5f72b7a4 f   MFC42D:MFC42D.DLL
 0001:0002a7aa       ?OnDraw@CFormView@@MAEXPAVCDC@@@Z 5f72b7aa f   MFC42D:MFC42D.DLL
 0001:0002a7b0       ?OnUpdate@CView@@MAEXPAV1@JPAVCObject@@@Z 5f72b7b0 f   MFC42D:MFC42D.DLL
 0001:0002a7b6       ?OnActivateFrame@CFormView@@MAEXIPAVCFrameWnd@@@Z 5f72b7b6 f   MFC42D:MFC42D.DLL
 0001:0002a7bc       ?OnActivateView@CFormView@@MAEXHPAVCView@@0@Z 5f72b7bc f   MFC42D:MFC42D.DLL
 0001:0002a7c2       ?OnPrepareDC@CScrollView@@UAEXPAVCDC@@PAUCPrintInfo@@@Z 5f72b7c2 f   MFC42D:MFC42D.DLL
 0001:0002a7c8       ?OnDragScroll@CView@@UAEKKVCPoint@@@Z 5f72b7c8 f   MFC42D:MFC42D.DLL
 0001:0002a7ce       ?OnDropEx@CView@@UAEKPAVCOleDataObject@@KKVCPoint@@@Z 5f72b7ce f   MFC42D:MFC42D.DLL
 0001:0002a7d4       ?OnDrop@CView@@UAEHPAVCOleDataObject@@KVCPoint@@@Z 5f72b7d4 f   MFC42D:MFC42D.DLL
 0001:0002a7da       ?OnDragLeave@CView@@UAEXXZ 5f72b7da f   MFC42D:MFC42D.DLL
 0001:0002a7e0       ?OnDragOver@CView@@UAEKPAVCOleDataObject@@KVCPoint@@@Z 5f72b7e0 f   MFC42D:MFC42D.DLL
 0001:0002a7e6       ?OnDragEnter@CView@@UAEKPAVCOleDataObject@@KVCPoint@@@Z 5f72b7e6 f   MFC42D:MFC42D.DLL
 0001:0002a7ec       ?OnScrollBy@CScrollView@@UAEHVCSize@@H@Z 5f72b7ec f   MFC42D:MFC42D.DLL
 0001:0002a7f2       ?OnScroll@CScrollView@@UAEHIIH@Z 5f72b7f2 f   MFC42D:MFC42D.DLL
 0001:0002a7f8       ?IsSelected@CView@@UBEHPBVCObject@@@Z 5f72b7f8 f   MFC42D:MFC42D.DLL
 0001:0002a7fe       ?SetOccDialogInfo@CFormView@@MAEHPAU_AFX_OCC_DIALOG_INFO@@@Z 5f72b7fe f   MFC42D:MFC42D.DLL
 0001:0002a804       ?IsFrameWnd@CWnd@@UBEHXZ   5f72b804 f   MFC42D:MFC42D.DLL
 0001:0002a80a       ?CheckAutoCenter@CWnd@@UAEHXZ 5f72b80a f   MFC42D:MFC42D.DLL
 0001:0002a810       ?OnChildNotify@CWnd@@MAEHIIJPAJ@Z 5f72b810 f   MFC42D:MFC42D.DLL
 0001:0002a816       ?PostNcDestroy@CView@@MAEXXZ 5f72b816 f   MFC42D:MFC42D.DLL
 0001:0002a81c       ?DefWindowProcA@CWnd@@MAEJIIJ@Z 5f72b81c f   MFC42D:MFC42D.DLL
 0001:0002a822       ?OnWndMsg@CWnd@@MAEHIIJPAJ@Z 5f72b822 f   MFC42D:MFC42D.DLL
 0001:0002a828       ?WindowProc@CWnd@@MAEJIIJ@Z 5f72b828 f   MFC42D:MFC42D.DLL
 0001:0002a82e       ?OnAmbientProperty@CWnd@@UAEHPAVCOleControlSite@@JPAUtagVARIANT@@@Z 5f72b82e f   MFC42D:MFC42D.DLL
 0001:0002a834       ?PreTranslateMessage@CFormView@@MAEHPAUtagMSG@@@Z 5f72b834 f   MFC42D:MFC42D.DLL
 0001:0002a83a       ?EndModalState@CWnd@@UAEXXZ 5f72b83a f   MFC42D:MFC42D.DLL
 0001:0002a840       ?BeginModalState@CWnd@@UAEXXZ 5f72b840 f   MFC42D:MFC42D.DLL
 0001:0002a846       ?DoDataExchange@CWnd@@MAEXPAVCDataExchange@@@Z 5f72b846 f   MFC42D:MFC42D.DLL
 0001:0002a84c       ?GetSuperWndProcAddr@CWnd@@MAEPAP6GJPAUHWND__@@IIJ@ZXZ 5f72b84c f   MFC42D:MFC42D.DLL
 0001:0002a852       ?OnNotify@CWnd@@MAEHIJPAJ@Z 5f72b852 f   MFC42D:MFC42D.DLL
 0001:0002a858       ?OnCommand@CWnd@@MAEHIJ@Z  5f72b858 f   MFC42D:MFC42D.DLL
 0001:0002a85e       ?EndModalLoop@CWnd@@UAEXH@Z 5f72b85e f   MFC42D:MFC42D.DLL
 0001:0002a864       ?ContinueModal@CWnd@@UAEHXZ 5f72b864 f   MFC42D:MFC42D.DLL
 0001:0002a86a       ?WinHelpA@CWnd@@UAEXKI@Z   5f72b86a f   MFC42D:MFC42D.DLL
 0001:0002a870       ?GetScrollBarCtrl@CView@@UBEPAVCScrollBar@@H@Z 5f72b870 f   MFC42D:MFC42D.DLL
 0001:0002a876       ?OnToolHitTest@CWnd@@UBEHVCPoint@@PAUtagTOOLINFOA@@@Z 5f72b876 f   MFC42D:MFC42D.DLL
 0001:0002a87c       ?CalcWindowRect@CScrollView@@UAEXPAUtagRECT@@I@Z 5f72b87c f   MFC42D:MFC42D.DLL
 0001:0002a882       ?PreCreateWindow@CView@@MAEHAAUtagCREATESTRUCTA@@@Z 5f72b882 f   MFC42D:MFC42D.DLL
 0001:0002a888       ?DestroyWindow@CWnd@@UAEHXZ 5f72b888 f   MFC42D:MFC42D.DLL
 0001:0002a88e       ?Create@CFormView@@MAEHPBD0KABUtagRECT@@PAVCWnd@@IPAUCCreateContext@@@Z 5f72b88e f   MFC42D:MFC42D.DLL
 0001:0002a894       ?PreSubclassWindow@CWnd@@UAEXXZ 5f72b894 f   MFC42D:MFC42D.DLL
 0001:0002a89a       ?GetConnectionHook@CCmdTarget@@MAEPAUIConnectionPoint@@ABU_GUID@@@Z 5f72b89a f   MFC42D:MFC42D.DLL
 0001:0002a8a0       ?GetExtraConnectionPoints@CCmdTarget@@MAEHPAVCPtrArray@@@Z 5f72b8a0 f   MFC42D:MFC42D.DLL
 0001:0002a8a6       ?GetInterfaceHook@CCmdTarget@@UAEPAUIUnknown@@PBX@Z 5f72b8a6 f   MFC42D:MFC42D.DLL
 0001:0002a8ac       ?OnCreateAggregates@CCmdTarget@@UAEHXZ 5f72b8ac f   MFC42D:MFC42D.DLL
 0001:0002a8b2       ?GetEventSinkMap@CCmdTarget@@MBEPBUAFX_EVENTSINKMAP@@XZ 5f72b8b2 f   MFC42D:MFC42D.DLL
 0001:0002a8b8       ?GetInterfaceMap@CCmdTarget@@MBEPBUAFX_INTERFACEMAP@@XZ 5f72b8b8 f   MFC42D:MFC42D.DLL
 0001:0002a8be       ?GetConnectionMap@CCmdTarget@@MBEPBUAFX_CONNECTIONMAP@@XZ 5f72b8be f   MFC42D:MFC42D.DLL
 0001:0002a8c4       ?GetDispatchMap@CCmdTarget@@MBEPBUAFX_DISPMAP@@XZ 5f72b8c4 f   MFC42D:MFC42D.DLL
 0001:0002a8ca       ?GetCommandMap@CCmdTarget@@MBEPBUAFX_OLECMDMAP@@XZ 5f72b8ca f   MFC42D:MFC42D.DLL
 0001:0002a8d0       ?GetTypeLib@CCmdTarget@@UAEJKPAPAUITypeLib@@@Z 5f72b8d0 f   MFC42D:MFC42D.DLL
 0001:0002a8d6       ?GetTypeLibCache@CCmdTarget@@UAEPAVCTypeLibCache@@XZ 5f72b8d6 f   MFC42D:MFC42D.DLL
 0001:0002a8dc       ?GetTypeInfoCount@CCmdTarget@@UAEIXZ 5f72b8dc f   MFC42D:MFC42D.DLL
 0001:0002a8e2       ?GetDispatchIID@CCmdTarget@@UAEHPAU_GUID@@@Z 5f72b8e2 f   MFC42D:MFC42D.DLL
 0001:0002a8e8       ?IsInvokeAllowed@CCmdTarget@@UAEHJ@Z 5f72b8e8 f   MFC42D:MFC42D.DLL
 0001:0002a8ee       ?OnFinalRelease@CWnd@@UAEXXZ 5f72b8ee f   MFC42D:MFC42D.DLL
 0001:0002a8f4       ?OnCmdMsg@CView@@UAEHIHPAXPAUAFX_CMDHANDLERINFO@@@Z 5f72b8f4 f   MFC42D:MFC42D.DLL
 0001:0002a8fa       ??0CFormView@@IAE@PBD@Z    5f72b8fa f   MFC42D:MFC42D.DLL
 0001:0002a900       ??0CFormView@@IAE@I@Z      5f72b900 f   MFC42D:MFC42D.DLL
 0001:0002a906       ??1CScrollView@@UAE@XZ     5f72b906 f   MFC42D:MFC42D.DLL
 0001:0002a90c       ?OnInitialUpdate@CFormView@@UAEXXZ 5f72b90c f   MFC42D:MFC42D.DLL
 0001:0002a912       ??1CWaitCursor@@QAE@XZ     5f72b912 f   MFC42D:MFC42D.DLL
 0001:0002a918       ??0CWaitCursor@@QAE@XZ     5f72b918 f   MFC42D:MFC42D.DLL
 0001:0002a91e       ?UpdateData@CWnd@@QAEHH@Z  5f72b91e f   MFC42D:MFC42D.DLL
 0001:0002a924       ?AfxSetWindowText@@YGXPAUHWND__@@PBD@Z 5f72b924 f   MFC42D:MFC42D.DLL
 0001:0002a92a       ?PrepareEditCtrl@CDataExchange@@QAEPAUHWND__@@H@Z 5f72b92a f   MFC42D:MFC42D.DLL
 0001:0002a930       ?DDX_Text@@YGXPAVCDataExchange@@HAAH@Z 5f72b930 f   MFC42D:MFC42D.DLL
 0001:0002a936       ?DDX_Text@@YGXPAVCDataExchange@@HAAE@Z 5f72b936 f   MFC42D:MFC42D.DLL
 0001:0002a93c       ?DDX_Text@@YGXPAVCDataExchange@@HAAI@Z 5f72b93c f   MFC42D:MFC42D.DLL
 0001:0002a942       ?DDX_Text@@YGXPAVCDataExchange@@HAAJ@Z 5f72b942 f   MFC42D:MFC42D.DLL
 0001:0002a948       ?DDX_Text@@YGXPAVCDataExchange@@HAAK@Z 5f72b948 f   MFC42D:MFC42D.DLL
 0001:0002a94e       ?AfxFailMaxChars@@YGXPAVCDataExchange@@H@Z 5f72b94e f   MFC42D:MFC42D.DLL
 0001:0002a954       ?GetAllocLength@CString@@QBEHXZ 5f72b954 f   MFC42D:MFC42D.DLL
 0001:0002a95a       ?PrepareCtrl@CDataExchange@@QAEPAUHWND__@@H@Z 5f72b95a f   MFC42D:MFC42D.DLL
 0001:0002a960       ?DDX_LBIndex@@YGXPAVCDataExchange@@HAAH@Z 5f72b960 f   MFC42D:MFC42D.DLL
 0001:0002a966       ?DDX_CBIndex@@YGXPAVCDataExchange@@HAAH@Z 5f72b966 f   MFC42D:MFC42D.DLL
 0001:0002a96c       ?DDX_Scroll@@YGXPAVCDataExchange@@HAAH@Z 5f72b96c f   MFC42D:MFC42D.DLL
 0001:0002a972       ?AfxFailRadio@@YGXPAVCDataExchange@@@Z 5f72b972 f   MFC42D:MFC42D.DLL
 0001:0002a978       ?DDX_Radio@@YGXPAVCDataExchange@@HAAH@Z 5f72b978 f   MFC42D:MFC42D.DLL
 0001:0002a97e       ?AssertValid@CFormView@@UBEXXZ 5f72b97e f   MFC42D:MFC42D.DLL
 0001:0002a984       ?Dump@CFormView@@UBEXAAVCDumpContext@@@Z 5f72b984 f   MFC42D:MFC42D.DLL
 0001:0002a98a       ?OnMove@CWnd@@IAEXHH@Z     5f72b98a f   MFC42D:MFC42D.DLL
 0001:0002a990       ??6CDumpContext@@QAEAAV0@M@Z 5f72b990 f   MFC42D:MFC42D.DLL
 0001:0002a996       ??6CDumpContext@@QAEAAV0@N@Z 5f72b996 f   MFC42D:MFC42D.DLL
 0001:0002a99c       ?AfxTextFloatFormat@@YGXPAVCDataExchange@@HPAXNH@Z 5f72b99c f   MFC42D:MFC42D.DLL
 0001:0002a9a2       ?IsEmpty@CMapPtrToPtr@@QBEHXZ 5f72b9a2 f   MFC42D:MFC42D.DLL
 0001:0002a9a8       ?RemoveKey@CMapPtrToPtr@@QAEHPAX@Z 5f72b9a8 f   MFC42D:MFC42D.DLL
 0001:0002a9ae       ?RemoveAll@CMapPtrToPtr@@QAEXXZ 5f72b9ae f   MFC42D:MFC42D.DLL
 0001:0002a9b4       ?GetNextAssoc@CMapPtrToPtr@@QBEXAAPAU__POSITION@@AAPAX1@Z 5f72b9b4 f   MFC42D:MFC42D.DLL
 0001:0002a9ba       ?GetStartPosition@CMapPtrToPtr@@QBEPAU__POSITION@@XZ 5f72b9ba f   MFC42D:MFC42D.DLL
 0001:0002a9c0       ??0CString@@QAE@ABV0@@Z    5f72b9c0 f   MFC42D:MFC42D.DLL
 0001:0002a9c6       ??3CNoTrackObject@@SGXPAXPBDH@Z 5f72b9c6 f   MFC42D:MFC42D.DLL
 0001:0002a9cc       ??2CNoTrackObject@@SGPAXIPBDH@Z 5f72b9cc f   MFC42D:MFC42D.DLL
 0001:0002a9d2       ?AfxGetApp@@YGPAVCWinApp@@XZ 5f72b9d2 f   MFC42D:MFC42D.DLL
 0001:0002a9d8       ??6CDumpContext@@QAEAAV0@ABVCObject@@@Z 5f72b9d8 f   MFC42D:MFC42D.DLL
 0001:0002a9de       ?DDX_Text@@YGXPAVCDataExchange@@HAAF@Z 5f72b9de f   MFC42D:MFC42D.DLL
 0001:0002a9e4       ?DDX_Text@@YGXPAVCDataExchange@@HAAM@Z 5f72b9e4 f   MFC42D:MFC42D.DLL
 0001:0002a9ea       ?DDX_Text@@YGXPAVCDataExchange@@HAAN@Z 5f72b9ea f   MFC42D:MFC42D.DLL
 0001:0002a9f0       ?DDX_Text@@YGXPAVCDataExchange@@HAAVCString@@@Z 5f72b9f0 f   MFC42D:MFC42D.DLL
 0001:0002a9f6       ?DDX_Text@@YGXPAVCDataExchange@@HPADH@Z 5f72b9f6 f   MFC42D:MFC42D.DLL
 0001:0002a9fc       ?DDX_Slider@@YGXPAVCDataExchange@@HAAH@Z 5f72b9fc f   MFC42D:MFC42D.DLL
 0001:0002aa02       ?Format@COleDateTime@@QBE?AVCString@@KK@Z 5f72ba02 f   MFCO42D:MFCO42D.DLL
 0001:0002aa08       ?GetStatus@COleDateTime@@QBE?AW4DateTimeStatus@1@XZ 5f72ba08 f   MFCO42D:MFCO42D.DLL
 0001:0002aa0e       ??4COleDateTime@@QAEABV0@ABV0@@Z 5f72ba0e f   MFCO42D:MFCO42D.DLL
 0001:0002aa14       ??0COleDateTime@@QAE@HHHHHH@Z 5f72ba14 f   MFCO42D:MFCO42D.DLL
 0001:0002aa1a       ?SetStatus@COleDateTime@@QAEXW4DateTimeStatus@1@@Z 5f72ba1a f   MFCO42D:MFCO42D.DLL
 0001:0002aa20       ??0COleDateTime@@QAE@XZ    5f72ba20 f   MFCO42D:MFCO42D.DLL
 0001:0002aa26       ?GetSecond@COleDateTime@@QBEHXZ 5f72ba26 f   MFCO42D:MFCO42D.DLL
 0001:0002aa2c       ?GetMinute@COleDateTime@@QBEHXZ 5f72ba2c f   MFCO42D:MFCO42D.DLL
 0001:0002aa32       ?GetHour@COleDateTime@@QBEHXZ 5f72ba32 f   MFCO42D:MFCO42D.DLL
 0001:0002aa38       ?GetDay@COleDateTime@@QBEHXZ 5f72ba38 f   MFCO42D:MFCO42D.DLL
 0001:0002aa3e       ?GetMonth@COleDateTime@@QBEHXZ 5f72ba3e f   MFCO42D:MFCO42D.DLL
 0001:0002aa44       ?GetYear@COleDateTime@@QBEHXZ 5f72ba44 f   MFCO42D:MFCO42D.DLL
 0001:0002aa4a       ??8COleDateTime@@QBEHABV0@@Z 5f72ba4a f   MFCO42D:MFCO42D.DLL
 0001:0002aa50       ??6@YGAAVCDumpContext@@AAV0@VCOleDateTime@@@Z 5f72ba50 f   MFCO42D:MFCO42D.DLL
 0001:0002aa56       ??0COleDateTime@@QAE@ABV0@@Z 5f72ba56 f   MFCO42D:MFCO42D.DLL
 0001:0002aa5c       ??1COleVariant@@QAE@XZ     5f72ba5c f   MFCO42D:MFCO42D.DLL
 0001:0002aa62       ??6@YGAAVCDumpContext@@AAV0@VCOleVariant@@@Z 5f72ba62 f   MFCO42D:MFCO42D.DLL
 0001:0002aa68       ??0COleVariant@@QAE@ABV0@@Z 5f72ba68 f   MFCO42D:MFCO42D.DLL
 0001:0002aa6e       ??0COleVariant@@QAE@JG@Z   5f72ba6e f   MFCO42D:MFCO42D.DLL
 0001:0002aa74       ?Clear@COleVariant@@QAEXXZ 5f72ba74 f   MFCO42D:MFCO42D.DLL
 0001:0002aa7a       ??0COleVariant@@QAE@XZ     5f72ba7a f   MFCO42D:MFCO42D.DLL
 0001:0002aa80       ??0COleVariant@@QAE@PBDG@Z 5f72ba80 f   MFCO42D:MFCO42D.DLL
 0001:0002aa86       ??4COleVariant@@QAEABV0@J@Z 5f72ba86 f   MFCO42D:MFCO42D.DLL
 0001:0002aa8c       ??4COleDateTime@@QAEABV0@ABUtagVARIANT@@@Z 5f72ba8c f   MFCO42D:MFCO42D.DLL
 0001:0002aa92       ??BCOleVariant@@QAEPAUtagVARIANT@@XZ 5f72ba92 f   MFCO42D:MFCO42D.DLL
 0001:0002aa98       ??0COleDateTime@@QAE@N@Z   5f72ba98 f   MFCO42D:MFCO42D.DLL
 0001:0002aa9e       ??0COleVariant@@QAE@FG@Z   5f72ba9e f   MFCO42D:MFCO42D.DLL
 0001:0002aaa4       ??0COleVariant@@QAE@ABUtagVARIANT@@@Z 5f72baa4 f   MFCO42D:MFCO42D.DLL
 0001:0002aaaa       ??4COleVariant@@QAEABV0@QBD@Z 5f72baaa f   MFCO42D:MFCO42D.DLL
 0001:0002aab0       ?SetStatus@COleCurrency@@QAEXW4CurrencyStatus@1@@Z 5f72bab0 f   MFCO42D:MFCO42D.DLL
 0001:0002aab6       ?GetStatus@COleCurrency@@QBE?AW4CurrencyStatus@1@XZ 5f72bab6 f   MFCO42D:MFCO42D.DLL
 0001:0002aabc       ??0COleCurrency@@QAE@XZ    5f72babc f   MFCO42D:MFCO42D.DLL
 0001:0002aac2       ??4COleCurrency@@QAEABV0@ABV0@@Z 5f72bac2 f   MFCO42D:MFCO42D.DLL
 0001:0002aac8       ??9COleDateTime@@QBEHABV0@@Z 5f72bac8 f   MFCO42D:MFCO42D.DLL
 0001:0002aace       ??9COleCurrency@@QBEHABV0@@Z 5f72bace f   MFCO42D:MFCO42D.DLL
 0001:0002aad4       ??4COleVariant@@QAEABV0@ABVCOleDateTime@@@Z 5f72bad4 f   MFCO42D:MFCO42D.DLL
 0001:0002aada       ??4COleVariant@@QAEABV0@N@Z 5f72bada f   MFCO42D:MFCO42D.DLL
 0001:0002aae0       ??4COleVariant@@QAEABV0@M@Z 5f72bae0 f   MFCO42D:MFCO42D.DLL
 0001:0002aae6       ??4COleVariant@@QAEABV0@ABVCOleCurrency@@@Z 5f72bae6 f   MFCO42D:MFCO42D.DLL
 0001:0002aaec       ??4COleVariant@@QAEABV0@F@Z 5f72baec f   MFCO42D:MFCO42D.DLL
 0001:0002aaf2       ??4COleVariant@@QAEABV0@E@Z 5f72baf2 f   MFCO42D:MFCO42D.DLL
 0001:0002aaf8       ??4COleVariant@@QAEABV0@ABVCLongBinary@@@Z 5f72baf8 f   MFCO42D:MFCO42D.DLL
 0001:0002aafe       ??4COleVariant@@QAEABV0@ABVCByteArray@@@Z 5f72bafe f   MFCO42D:MFCO42D.DLL
 0001:0002ab04       ??6@YGAAVCDumpContext@@AAV0@VCOleCurrency@@@Z 5f72bb04 f   MFCO42D:MFCO42D.DLL
 0001:0002ab0a       ??0COleCurrency@@QAE@ABV0@@Z 5f72bb0a f   MFCO42D:MFCO42D.DLL
 0001:0002ab10       ??4COleVariant@@QAEABV0@ABV0@@Z 5f72bb10 f   MFCO42D:MFCO42D.DLL
 0001:0002ab16       ??8COleVariant@@QBEHABUtagVARIANT@@@Z 5f72bb16 f   MFCO42D:MFCO42D.DLL
 0001:0002ab1c       ?DDX_Text@@YGXPAVCDataExchange@@HAAVCOleCurrency@@@Z 5f72bb1c f   MFCO42D:MFCO42D.DLL
 0001:0002ab22       ?DDX_Text@@YGXPAVCDataExchange@@HAAVCOleDateTime@@@Z 5f72bb22 f   MFCO42D:MFCO42D.DLL
 0001:0002ab28       ___CxxFrameHandler         5f72bb28 f   msvcrtd:MSVCRTD.dll
 0001:0002ab30       ??_L@YGXPAXIHP6EX0@Z1@Z    5f72bb30 f   msvcrtd:ehvecctr.obj
 0001:0002abd0       ??_M@YGXPAXIHP6EX0@Z@Z     5f72bbd0 f   msvcrtd:ehvecdtr.obj
 0001:0002ac80       ?__ArrayUnwind@@YGXPAXIHP6EX0@Z@Z 5f72bc80 f   msvcrtd:ehvecdtr.obj
 0001:0002ad30       ??0type_info@@AAE@ABV0@@Z  5f72bd30 f   msvcrtd:ti_inst.obj
 0001:0002ad50       ??_Gtype_info@@UAEPAXI@Z   5f72bd50 f i msvcrtd:ti_inst.obj
 0001:0002ad50       ??_Etype_info@@UAEPAXI@Z   5f72bd50 f i msvcrtd:ti_inst.obj
 0001:0002ad80       ??4type_info@@AAEAAV0@ABV0@@Z 5f72bd80 f   msvcrtd:ti_inst.obj
 0001:0002ad90       __CxxThrowException@8      5f72bd90 f   msvcrtd:MSVCRTD.dll
 0001:0002ad96       __mbsnbicmp                5f72bd96 f   msvcrtd:MSVCRTD.dll
 0001:0002ad9c       __mbsinc                   5f72bd9c f   msvcrtd:MSVCRTD.dll
 0001:0002ada2       _memset                    5f72bda2 f   msvcrtd:MSVCRTD.dll
 0001:0002ada8       _memcpy                    5f72bda8 f   msvcrtd:MSVCRTD.dll
 0001:0002adae       __mbsstr                   5f72bdae f   msvcrtd:MSVCRTD.dll
 0001:0002adb4       _abs                       5f72bdb4 f   msvcrtd:MSVCRTD.dll
 0001:0002adc0       __onexit                   5f72bdc0 f   msvcrtd:atonexit.obj
 0001:0002ae00       _atexit                    5f72be00 f   msvcrtd:atonexit.obj
 0001:0002ae18       _labs                      5f72be18 f   msvcrtd:MSVCRTD.dll
 0001:0002ae1e       _memcmp                    5f72be1e f   msvcrtd:MSVCRTD.dll
 0001:0002ae24       __purecall                 5f72be24 f   msvcrtd:MSVCRTD.dll
 0001:0002ae2a       __CrtDbgReport             5f72be2a f   msvcrtd:MSVCRTD.dll
 0001:0002ae30       __vsnprintf                5f72be30 f   msvcrtd:MSVCRTD.dll
 0001:0002ae40       __CRT_INIT@12              5f72be40 f   msvcrtd:crtdll.obj
 0001:0002af50       __DllMainCRTStartup@12     5f72bf50 f   msvcrtd:crtdll.obj
 0001:0002b044       __except_handler3          5f72c044 f   msvcrtd:MSVCRTD.dll
 0001:0002b04a       ?terminate@@YAXXZ          5f72c04a f   msvcrtd:MSVCRTD.dll
 0001:0002b050       ??1type_info@@UAE@XZ       5f72c050 f   msvcrtd:MSVCRTD.dll
 0001:0002b056       ___dllonexit               5f72c056 f   msvcrtd:MSVCRTD.dll
 0001:0002b05c       __free_dbg                 5f72c05c f   msvcrtd:MSVCRTD.dll
 0001:0002b062       __initterm                 5f72c062 f   msvcrtd:MSVCRTD.dll
 0001:0002b068       __malloc_dbg               5f72c068 f   msvcrtd:MSVCRTD.dll
 0001:0002b06e       _FreeLibrary@4             5f72c06e f   kernel32:KERNEL32.dll
 0001:0002b074       _GetModuleHandleA@4        5f72c074 f   kernel32:KERNEL32.dll
 0001:0002b07a       _LocalFree@4               5f72c07a f   kernel32:KERNEL32.dll
 0001:0002b080       _LocalAlloc@8              5f72c080 f   kernel32:KERNEL32.dll
 0001:0002b086       _LoadLibraryA@4            5f72c086 f   kernel32:KERNEL32.dll
 0001:0002b08c       _lstrcmpA@8                5f72c08c f   kernel32:KERNEL32.dll
 0001:0002b092       _lstrcpynA@12              5f72c092 f   kernel32:KERNEL32.dll
 0001:0002b098       _lstrlenA@4                5f72c098 f   kernel32:KERNEL32.dll
 0001:0002b09e       _lstrcpyA@8                5f72c09e f   kernel32:KERNEL32.dll
 0001:0002b0a4       _GlobalUnlock@4            5f72c0a4 f   kernel32:KERNEL32.dll
 0001:0002b0aa       _GlobalLock@4              5f72c0aa f   kernel32:KERNEL32.dll
 0001:0002b0b0       _GlobalAlloc@8             5f72c0b0 f   kernel32:KERNEL32.dll
 0001:0002b0b6       _GlobalReAlloc@12          5f72c0b6 f   kernel32:KERNEL32.dll
 0001:0002b0bc       _GlobalFree@4              5f72c0bc f   kernel32:KERNEL32.dll
 0001:0002b0c2       _GlobalSize@4              5f72c0c2 f   kernel32:KERNEL32.dll
 0001:0002b0c8       _OutputDebugStringA@4      5f72c0c8 f   kernel32:KERNEL32.dll
 0001:0002b0ce       _wsprintfA                 5f72c0ce f   user32:USER32.dll
 0001:0002b0d4       _EnableWindow@8            5f72c0d4 f   user32:USER32.dll
 0001:0002b0da       _GetDesktopWindow@0        5f72c0da f   user32:USER32.dll
 0001:0002b0e0       _GetWindowTextA@12         5f72c0e0 f   user32:USER32.dll
 0001:0002b0e6       _GetWindowTextLengthA@4    5f72c0e6 f   user32:USER32.dll
 0001:0002b0ec       _SendMessageA@16           5f72c0ec f   user32:USER32.dll
 0001:0002b0f2       _GetWindowLongA@8          5f72c0f2 f   user32:USER32.dll
 0001:0002b0f8       __imp_load__CoGetClassObject@20 5f72c0f8     ole32:ole32.dll
 0001:0002b104       __tailMerge_ole32          5f72c104     ole32:ole32.dll
 0001:0002b112       _CoGetClassObject@20       5f72c112     ole32:ole32.dll
 0001:0002b118       __imp_load__CoInitialize@4 5f72c118     ole32:ole32.dll
 0001:0002b124       _CoInitialize@4            5f72c124     ole32:ole32.dll
 0001:0002b12a       __imp_load__CoUninitialize@0 5f72c12a     ole32:ole32.dll
 0001:0002b136       _CoUninitialize@0          5f72c136     ole32:ole32.dll
 0001:0002b13c       __imp_load__SysFreeString@4 5f72c13c     oleaut32:OLEAUT32.dll
 0001:0002b148       __tailMerge_OLEAUT32       5f72c148     oleaut32:OLEAUT32.dll
 0001:0002b156       _SysFreeString@4           5f72c156     oleaut32:OLEAUT32.dll
 0001:0002b15c       __imp_load__SQLError@32    5f72c15c     odbc32:ODBC32.dll
 0001:0002b168       __tailMerge_ODBC32         5f72c168     odbc32:ODBC32.dll
 0001:0002b176       _SQLError@32               5f72c176     odbc32:ODBC32.dll
 0001:0002b17c       __imp_load__SQLFreeStmt@8  5f72c17c     odbc32:ODBC32.dll
 0001:0002b188       _SQLFreeStmt@8             5f72c188     odbc32:ODBC32.dll
 0001:0002b18e       __imp_load__SQLCancel@4    5f72c18e     odbc32:ODBC32.dll
 0001:0002b19a       _SQLCancel@4               5f72c19a     odbc32:ODBC32.dll
 0001:0002b1a0       __imp_load__SQLMoreResults@4 5f72c1a0     odbc32:ODBC32.dll
 0001:0002b1ac       _SQLMoreResults@4          5f72c1ac     odbc32:ODBC32.dll
 0001:0002b1b2       __imp_load__SQLFetch@4     5f72c1b2     odbc32:ODBC32.dll
 0001:0002b1be       _SQLFetch@4                5f72c1be     odbc32:ODBC32.dll
 0001:0002b1c4       __imp_load__SQLNumResultCols@8 5f72c1c4     odbc32:ODBC32.dll
 0001:0002b1d0       _SQLNumResultCols@8        5f72c1d0     odbc32:ODBC32.dll
 0001:0002b1d6       __imp_load__SQLExecDirect@12 5f72c1d6     odbc32:ODBC32.dll
 0001:0002b1e2       _SQLExecDirect@12          5f72c1e2     odbc32:ODBC32.dll
 0001:0002b1e8       __imp_load__SQLAllocStmt@8 5f72c1e8     odbc32:ODBC32.dll
 0001:0002b1f4       _SQLAllocStmt@8            5f72c1f4     odbc32:ODBC32.dll
 0001:0002b1fa       __imp_load__SQLFreeConnect@4 5f72c1fa     odbc32:ODBC32.dll
 0001:0002b206       _SQLFreeConnect@4          5f72c206     odbc32:ODBC32.dll
 0001:0002b20c       __imp_load__SQLDisconnect@4 5f72c20c     odbc32:ODBC32.dll
 0001:0002b218       _SQLDisconnect@4           5f72c218     odbc32:ODBC32.dll
 0001:0002b21e       __imp_load__SQLFreeEnv@4   5f72c21e     odbc32:ODBC32.dll
 0001:0002b22a       _SQLFreeEnv@4              5f72c22a     odbc32:ODBC32.dll
 0001:0002b230       __imp_load__SQLSetStmtOption@12 5f72c230     odbc32:ODBC32.dll
 0001:0002b23c       _SQLSetStmtOption@12       5f72c23c     odbc32:ODBC32.dll
 0001:0002b242       __imp_load__SQLGetInfo@20  5f72c242     odbc32:ODBC32.dll
 0001:0002b24e       _SQLGetInfo@20             5f72c24e     odbc32:ODBC32.dll
 0001:0002b254       __imp_load__SQLSetConnectOption@12 5f72c254     odbc32:ODBC32.dll
 0001:0002b260       _SQLSetConnectOption@12    5f72c260     odbc32:ODBC32.dll
 0001:0002b266       __imp_load__SQLTransact@12 5f72c266     odbc32:ODBC32.dll
 0001:0002b272       _SQLTransact@12            5f72c272     odbc32:ODBC32.dll
 0001:0002b278       __imp_load__SQLAllocConnect@8 5f72c278     odbc32:ODBC32.dll
 0001:0002b284       _SQLAllocConnect@8         5f72c284     odbc32:ODBC32.dll
 0001:0002b28a       __imp_load__SQLAllocEnv@4  5f72c28a     odbc32:ODBC32.dll
 0001:0002b296       _SQLAllocEnv@4             5f72c296     odbc32:ODBC32.dll
 0001:0002b29c       __imp_load__SQLDriverConnect@32 5f72c29c     odbc32:ODBC32.dll
 0001:0002b2a8       _SQLDriverConnect@32       5f72c2a8     odbc32:ODBC32.dll
 0001:0002b2ae       __imp_load__SQLGetData@24  5f72c2ae     odbc32:ODBC32.dll
 0001:0002b2ba       _SQLGetData@24             5f72c2ba     odbc32:ODBC32.dll
 0001:0002b2c0       __imp_load__SQLSetPos@16   5f72c2c0     odbc32:ODBC32.dll
 0001:0002b2cc       _SQLSetPos@16              5f72c2cc     odbc32:ODBC32.dll
 0001:0002b2d2       __imp_load__SQLExecute@4   5f72c2d2     odbc32:ODBC32.dll
 0001:0002b2de       _SQLExecute@4              5f72c2de     odbc32:ODBC32.dll
 0001:0002b2e4       __imp_load__SQLGetStmtOption@12 5f72c2e4     odbc32:ODBC32.dll
 0001:0002b2f0       _SQLGetStmtOption@12       5f72c2f0     odbc32:ODBC32.dll
 0001:0002b2f6       __imp_load__SQLPrepare@12  5f72c2f6     odbc32:ODBC32.dll
 0001:0002b302       _SQLPrepare@12             5f72c302     odbc32:ODBC32.dll
 0001:0002b308       __imp_load__SQLGetFunctions@12 5f72c308     odbc32:ODBC32.dll
 0001:0002b314       _SQLGetFunctions@12        5f72c314     odbc32:ODBC32.dll
 0001:0002b31a       __imp_load__SQLDescribeCol@36 5f72c31a     odbc32:ODBC32.dll
 0001:0002b326       _SQLDescribeCol@36         5f72c326     odbc32:ODBC32.dll
 0001:0002b32c       __imp_load__SQLExtendedFetch@20 5f72c32c     odbc32:ODBC32.dll
 0001:0002b338       _SQLExtendedFetch@20       5f72c338     odbc32:ODBC32.dll
 0001:0002b33e       __imp_load__SQLGetCursorName@16 5f72c33e     odbc32:ODBC32.dll
 0001:0002b34a       _SQLGetCursorName@16       5f72c34a     odbc32:ODBC32.dll
 0001:0002b350       __imp_load__SQLRowCount@8  5f72c350     odbc32:ODBC32.dll
 0001:0002b35c       _SQLRowCount@8             5f72c35c     odbc32:ODBC32.dll
 0001:0002b362       __imp_load__SQLPutData@12  5f72c362     odbc32:ODBC32.dll
 0001:0002b36e       _SQLPutData@12             5f72c36e     odbc32:ODBC32.dll
 0001:0002b374       __imp_load__SQLParamData@8 5f72c374     odbc32:ODBC32.dll
 0001:0002b380       _SQLParamData@8            5f72c380     odbc32:ODBC32.dll
 0001:0002b386       __imp_load__SQLBindCol@24  5f72c386     odbc32:ODBC32.dll
 0001:0002b392       _SQLBindCol@24             5f72c392     odbc32:ODBC32.dll
 0001:0002b398       __imp_load__SQLBindParameter@40 5f72c398     odbc32:ODBC32.dll
 0001:0002b3a4       _SQLBindParameter@40       5f72c3a4     odbc32:ODBC32.dll
 0001:0002b3aa       ___delayLoadHelper@8       5f72c3aa f   delayimp:delayhlp.obj
 0001:0002b5a3       ___FUnloadDelayLoadedDLL@4 5f72c5a3 f   delayimp:delayhlp.obj
 0001:0002b656       _GetProcAddress@8          5f72c656 f   kernel32:KERNEL32.dll
 0001:0002b65c       _InterlockedExchange@8     5f72c65c f   kernel32:KERNEL32.dll
 0001:0002b662       _RaiseException@16         5f72c662 f   kernel32:KERNEL32.dll
 0001:0002b668       _GetLastError@0            5f72c668 f   kernel32:KERNEL32.dll
 0001:0002b670       ?_GetBaseMessageMap@COleDBRecordView@@KGPBUAFX_MSGMAP@@XZ 5f72c670 f   viewoled.obj
 0001:0002b67a       ?GetMessageMap@COleDBRecordView@@MBEPBUAFX_MSGMAP@@XZ 5f72c67a f   viewoled.obj
 0001:0002b68a       ?OnInitialUpdate@COleDBRecordView@@UAEXXZ 5f72c68a f   viewoled.obj
 0001:0002b69d       ?OnMove@COleDBRecordView@@UAEHI@Z 5f72c69d f   viewoled.obj
 0001:0002b816       ?OnUpdateRecordFirst@COleDBRecordView@@IAEXPAVCCmdUI@@@Z 5f72c816 f   viewoled.obj
 0001:0002b83d       ?OnUpdateRecordPrev@COleDBRecordView@@IAEXPAVCCmdUI@@@Z 5f72c83d f   viewoled.obj
 0001:0002b864       ?OnUpdateRecordNext@COleDBRecordView@@IAEXPAVCCmdUI@@@Z 5f72c864 f   viewoled.obj
 0001:0002b88b       ?OnUpdateRecordLast@COleDBRecordView@@IAEXPAVCCmdUI@@@Z 5f72c88b f   viewoled.obj
 0001:0002b8c0       _RawDllMain@12             5f72c8c0 f   dlldb.obj
 0001:0002b97b       _DllMain@12                5f72c97b f   dlldb.obj
 0001:0002ba3a       ?AfxDbInitModule@@YGXXZ    5f72ca3a f   dlldb.obj
 0001:0002bb00       ?_GetBaseClass@CDBException@@KGPAUCRuntimeClass@@XZ 5f72cb00 f   dbcore.obj
 0001:0002bb0a       ?GetRuntimeClass@CDBException@@UBEPAUCRuntimeClass@@XZ 5f72cb0a f   dbcore.obj
 0001:0002bb1a       ?_GetBaseClass@CDatabase@@KGPAUCRuntimeClass@@XZ 5f72cb1a f   dbcore.obj
 0001:0002bb24       ?GetRuntimeClass@CDatabase@@UBEPAUCRuntimeClass@@XZ 5f72cb24 f   dbcore.obj
 0001:0002bb34       ?_GetBaseClass@CRecordset@@KGPAUCRuntimeClass@@XZ 5f72cb34 f   dbcore.obj
 0001:0002bb3e       ?GetRuntimeClass@CRecordset@@UBEPAUCRuntimeClass@@XZ 5f72cb3e f   dbcore.obj
 0001:0002bb90       ??1?$CProcessLocal@V_AFX_DB_STATE@@@@QAE@XZ 5f72cb90 f i dbcore.obj
 0001:0002bbb0       ??B?$CProcessLocal@V_AFX_DB_STATE@@@@QAEPAV_AFX_DB_STATE@@XZ 5f72cbb0 f i dbcore.obj
 0001:0002bbd0       ?GetData@?$CProcessLocal@V_AFX_DB_STATE@@@@QAEPAV_AFX_DB_STATE@@XZ 5f72cbd0 f i dbcore.obj
 0001:0002bc20       ?CreateObject@?$CProcessLocal@V_AFX_DB_STATE@@@@SGPAVCNoTrackObject@@XZ 5f72cc20 f i dbcore.obj
 0001:0002bc90       ??0_AFX_DB_STATE@@QAE@XZ   5f72cc90 f i dbcore.obj
 0001:0002bcb0       ??_E_AFX_DB_STATE@@UAEPAXI@Z 5f72ccb0 f i dbcore.obj
 0001:0002bcb0       ??_G_AFX_DB_STATE@@UAEPAXI@Z 5f72ccb0 f i dbcore.obj
 0001:0002bce0       ??0CNoTrackObject@@QAE@XZ  5f72cce0 f i dbcore.obj
 0001:0002bd00       ??1_AFX_DB_STATE@@UAE@XZ   5f72cd00 f i dbcore.obj
 0001:0002bd20       ?_GetBaseClass@CRecordView@@KGPAUCRuntimeClass@@XZ 5f72cd20 f   dbview.obj
 0001:0002bd2a       ?GetRuntimeClass@CRecordView@@UBEPAUCRuntimeClass@@XZ 5f72cd2a f   dbview.obj
 0001:0002bd40       ?_GetBaseClass@CLongBinary@@KGPAUCRuntimeClass@@XZ 5f72cd40 f   dblong.obj
 0001:0002bd4a       ?GetRuntimeClass@CLongBinary@@UBEPAUCRuntimeClass@@XZ 5f72cd4a f   dblong.obj
 0001:0002bd60       ?_GetBaseClass@COleDBRecordView@@KGPAUCRuntimeClass@@XZ 5f72cd60 f   viewoled.obj
 0001:0002bd6a       ?GetRuntimeClass@COleDBRecordView@@UBEPAUCRuntimeClass@@XZ 5f72cd6a f   viewoled.obj
 0001:0002bd80       ??B?$CComPtr@UIRowsetChange@@@ATL@@QBEPAUIRowsetChange@@XZ 5f72cd80 f i viewoled.obj
 0001:0002bd80       ??B?$CComPtr@UIRowset@@@ATL@@QBEPAUIRowset@@XZ 5f72cd80 f i viewoled.obj
 0001:0002bd90       ??C?$CComPtr@UIRowsetChange@@@ATL@@QBEPAV?$_NoAddRefReleaseOnCComPtr@UIRowsetChange@@@1@XZ 5f72cd90 f i viewoled.obj
 0001:0002bd90       ??C?$CComPtr@UIRowset@@@ATL@@QBEPAV?$_NoAddRefReleaseOnCComPtr@UIRowset@@@1@XZ 5f72cd90 f i viewoled.obj
 0001:0002c070       ??_ECDatabase@@UAEPAXI@Z   5f72d070 f i dlldb.obj
 0001:0002c0e0       ??_ECLongBinary@@UAEPAXI@Z 5f72d0e0 f i dlldb.obj
 0001:0002c150       ??_ECDaoWorkspace@@UAEPAXI@Z 5f72d150 f i dlldb.obj
 0001:0002c1c0       ??_ECDaoException@@UAEPAXI@Z 5f72d1c0 f i dlldb.obj
 0001:0002c230       ??_ECDaoDatabase@@UAEPAXI@Z 5f72d230 f i dlldb.obj
 0001:0002c2a0       ??_FCDaoDatabase@@QAEXXZ   5f72d2a0 f i dlldb.obj
 0001:0002c2c0       ??_ECDaoRecordset@@UAEPAXI@Z 5f72d2c0 f i dlldb.obj
 0001:0002c330       ??_FCDaoRecordset@@QAEXXZ  5f72d330 f i dlldb.obj
 0001:0002c350       ??B?$CTypedSimpleList@PAVCOleObjectFactory@@@@QAEPAVCOleObjectFactory@@XZ 5f72d350 f i dlldb.obj
 0001:0002c350       ??B?$CTypedSimpleList@PAUCRuntimeClass@@@@QAEPAUCRuntimeClass@@XZ 5f72d350 f i dlldb.obj
 0002:00000000       __imp__FreeLibrary@4       5f72f000     kernel32:KERNEL32.dll
 0002:00000004       __imp__GetModuleHandleA@4  5f72f004     kernel32:KERNEL32.dll
 0002:00000008       __imp__LocalFree@4         5f72f008     kernel32:KERNEL32.dll
 0002:0000000c       __imp__LocalAlloc@8        5f72f00c     kernel32:KERNEL32.dll
 0002:00000010       __imp__LoadLibraryA@4      5f72f010     kernel32:KERNEL32.dll
 0002:00000014       __imp__lstrcmpA@8          5f72f014     kernel32:KERNEL32.dll
 0002:00000018       __imp__lstrcpynA@12        5f72f018     kernel32:KERNEL32.dll
 0002:0000001c       __imp__lstrlenA@4          5f72f01c     kernel32:KERNEL32.dll
 0002:00000020       __imp__lstrcpyA@8          5f72f020     kernel32:KERNEL32.dll
 0002:00000024       __imp__GlobalUnlock@4      5f72f024     kernel32:KERNEL32.dll
 0002:00000028       __imp__GlobalLock@4        5f72f028     kernel32:KERNEL32.dll
 0002:0000002c       __imp__GlobalAlloc@8       5f72f02c     kernel32:KERNEL32.dll
 0002:00000030       __imp__GlobalReAlloc@12    5f72f030     kernel32:KERNEL32.dll
 0002:00000034       __imp__GlobalFree@4        5f72f034     kernel32:KERNEL32.dll
 0002:00000038       __imp__GlobalSize@4        5f72f038     kernel32:KERNEL32.dll
 0002:0000003c       __imp__OutputDebugStringA@4 5f72f03c     kernel32:KERNEL32.dll
 0002:00000040       __imp__GetProcAddress@8    5f72f040     kernel32:KERNEL32.dll
 0002:00000044       __imp__InterlockedExchange@8 5f72f044     kernel32:KERNEL32.dll
 0002:00000048       __imp__RaiseException@16   5f72f048     kernel32:KERNEL32.dll
 0002:0000004c       __imp__GetLastError@0      5f72f04c     kernel32:KERNEL32.dll
 0002:00000050       \177KERNEL32_NULL_THUNK_DATA 5f72f050     kernel32:KERNEL32.dll
 0002:00000054       __imp_??0CString@@QAE@XZ   5f72f054     MFC42D:MFC42D.DLL
 0002:00000058       __imp_??0CException@@QAE@XZ 5f72f058     MFC42D:MFC42D.DLL
 0002:0000005c       __imp_??H@YG?AVCString@@ABV0@PBD@Z 5f72f05c     MFC42D:MFC42D.DLL
 0002:00000060       __imp_??H@YG?AVCString@@PBDABV0@@Z 5f72f060     MFC42D:MFC42D.DLL
 0002:00000064       __imp_??1CException@@UAE@XZ 5f72f064     MFC42D:MFC42D.DLL
 0002:00000068       __imp_??4CString@@QAEABV0@ABV0@@Z 5f72f068     MFC42D:MFC42D.DLL
 0002:0000006c       __imp_?Right@CString@@QBE?AV1@H@Z 5f72f06c     MFC42D:MFC42D.DLL
 0002:00000070       __imp_?GetLength@CString@@QBEHXZ 5f72f070     MFC42D:MFC42D.DLL
 0002:00000074       __imp_??YCString@@QAEABV0@ABV0@@Z 5f72f074     MFC42D:MFC42D.DLL
 0002:00000078       __imp_?Left@CString@@QBE?AV1@H@Z 5f72f078     MFC42D:MFC42D.DLL
 0002:0000007c       __imp_?Find@CString@@QBEHD@Z 5f72f07c     MFC42D:MFC42D.DLL
 0002:00000080       __imp_??ACString@@QBEDH@Z  5f72f080     MFC42D:MFC42D.DLL
 0002:00000084       __imp_?IsEmpty@CString@@QBEHXZ 5f72f084     MFC42D:MFC42D.DLL
 0002:00000088       __imp_??YCString@@QAEABV0@PBD@Z 5f72f088     MFC42D:MFC42D.DLL
 0002:0000008c       __imp_??BCString@@QBEPBDXZ 5f72f08c     MFC42D:MFC42D.DLL
 0002:00000090       __imp_??4CString@@QAEABV0@PBE@Z 5f72f090     MFC42D:MFC42D.DLL
 0002:00000094       __imp_?AfxAssertValidObject@@YGXPBVCObject@@PBDH@Z 5f72f094     MFC42D:MFC42D.DLL
 0002:00000098       __imp_?AfxIsValidString@@YGHPBDH@Z 5f72f098     MFC42D:MFC42D.DLL
 0002:0000009c       __imp_??0CString@@QAE@PBD@Z 5f72f09c     MFC42D:MFC42D.DLL
 0002:000000a0       __imp_?Empty@CString@@QAEXXZ 5f72f0a0     MFC42D:MFC42D.DLL
 0002:000000a4       __imp_??1CObject@@UAE@XZ   5f72f0a4     MFC42D:MFC42D.DLL
 0002:000000a8       __imp_??0CPtrList@@QAE@H@Z 5f72f0a8     MFC42D:MFC42D.DLL
 0002:000000ac       __imp_??0CObject@@IAE@XZ   5f72f0ac     MFC42D:MFC42D.DLL
 0002:000000b0       __imp_??1CPtrList@@UAE@XZ  5f72f0b0     MFC42D:MFC42D.DLL
 0002:000000b4       __imp_??4CString@@QAEABV0@PBD@Z 5f72f0b4     MFC42D:MFC42D.DLL
 0002:000000b8       __imp_?IsKindOf@CObject@@QBEHPBUCRuntimeClass@@@Z 5f72f0b8     MFC42D:MFC42D.DLL
 0002:000000bc       __imp_?classCException@CException@@2UCRuntimeClass@@B 5f72f0bc     MFC42D:MFC42D.DLL
 0002:000000c0       __imp_?AfxUnlockGlobals@@YGXH@Z 5f72f0c0     MFC42D:MFC42D.DLL
 0002:000000c4       __imp_?GetHead@CPtrList@@QAEAAPAXXZ 5f72f0c4     MFC42D:MFC42D.DLL
 0002:000000c8       __imp_?IsEmpty@CPtrList@@QBEHXZ 5f72f0c8     MFC42D:MFC42D.DLL
 0002:000000cc       __imp_?AfxLockGlobals@@YGXH@Z 5f72f0cc     MFC42D:MFC42D.DLL
 0002:000000d0       __imp_?Delete@CException@@QAEXXZ 5f72f0d0     MFC42D:MFC42D.DLL
 0002:000000d4       __imp_?afxTraceFlags@@3IA  5f72f0d4     MFC42D:MFC42D.DLL
 0002:000000d8       __imp_?AfxThrowMemoryException@@YGXXZ 5f72f0d8     MFC42D:MFC42D.DLL
 0002:000000dc       __imp_?GetSafeOwner_@CWnd@@SGPAUHWND__@@PAU2@PAPAU2@@Z 5f72f0dc     MFC42D:MFC42D.DLL
 0002:000000e0       __imp_?GetDepth@CDumpContext@@QBEHXZ 5f72f0e0     MFC42D:MFC42D.DLL
 0002:000000e4       __imp_??6CDumpContext@@QAEAAV0@K@Z 5f72f0e4     MFC42D:MFC42D.DLL
 0002:000000e8       __imp_??6CDumpContext@@QAEAAV0@H@Z 5f72f0e8     MFC42D:MFC42D.DLL
 0002:000000ec       __imp_??6@YGAAVCDumpContext@@AAV0@ABVCString@@@Z 5f72f0ec     MFC42D:MFC42D.DLL
 0002:000000f0       __imp_??6CDumpContext@@QAEAAV0@PBX@Z 5f72f0f0     MFC42D:MFC42D.DLL
 0002:000000f4       __imp_??6CDumpContext@@QAEAAV0@PBD@Z 5f72f0f4     MFC42D:MFC42D.DLL
 0002:000000f8       __imp_??1CMapPtrToPtr@@UAE@XZ 5f72f0f8     MFC42D:MFC42D.DLL
 0002:000000fc       __imp_?AddHead@CPtrList@@QAEPAU__POSITION@@PAX@Z 5f72f0fc     MFC42D:MFC42D.DLL
 0002:00000100       __imp_?AfxIsValidAddress@@YGHPBXIH@Z 5f72f100     MFC42D:MFC42D.DLL
 0002:00000104       __imp_??0CMapPtrToPtr@@QAE@H@Z 5f72f104     MFC42D:MFC42D.DLL
 0002:00000108       __imp_?RemoveAt@CPtrList@@QAEXPAU__POSITION@@@Z 5f72f108     MFC42D:MFC42D.DLL
 0002:0000010c       __imp_?Find@CPtrList@@QBEPAU__POSITION@@PAXPAU2@@Z 5f72f10c     MFC42D:MFC42D.DLL
 0002:00000110       __imp_?Find@CString@@QBEHPBD@Z 5f72f110     MFC42D:MFC42D.DLL
 0002:00000114       __imp_??2@YAPAXIPBDH@Z     5f72f114     MFC42D:MFC42D.DLL
 0002:00000118       __imp_?GetBufferSetLength@CString@@QAEPADH@Z 5f72f118     MFC42D:MFC42D.DLL
 0002:0000011c       __imp_??9@YG_NABVCString@@0@Z 5f72f11c     MFC42D:MFC42D.DLL
 0002:00000120       __imp_??3CObject@@SGXPAXPBDH@Z 5f72f120     MFC42D:MFC42D.DLL
 0002:00000124       __imp_?ReleaseBuffer@CString@@QAEXH@Z 5f72f124     MFC42D:MFC42D.DLL
 0002:00000128       __imp_?GetBuffer@CString@@QAEPADH@Z 5f72f128     MFC42D:MFC42D.DLL
 0002:0000012c       __imp_??3@YAXPAXPBDH@Z     5f72f12c     MFC42D:MFC42D.DLL
 0002:00000130       __imp_?MakeUpper@CString@@QAEXXZ 5f72f130     MFC42D:MFC42D.DLL
 0002:00000134       __imp_?SetAt@CString@@QAEXHD@Z 5f72f134     MFC42D:MFC42D.DLL
 0002:00000138       __imp_?Lookup@CMapPtrToPtr@@QBEHPAXAAPAX@Z 5f72f138     MFC42D:MFC42D.DLL
 0002:0000013c       __imp_??8@YG_NABVCString@@PBD@Z 5f72f13c     MFC42D:MFC42D.DLL
 0002:00000140       __imp_??6CDumpContext@@QAEAAV0@PBVCObject@@@Z 5f72f140     MFC42D:MFC42D.DLL
 0002:00000144       __imp_??6CDumpContext@@QAEAAV0@J@Z 5f72f144     MFC42D:MFC42D.DLL
 0002:00000148       __imp_??6CDumpContext@@QAEAAV0@I@Z 5f72f148     MFC42D:MFC42D.DLL
 0002:0000014c       __imp_?classCObject@CObject@@2UCRuntimeClass@@B 5f72f14c     MFC42D:MFC42D.DLL
 0002:00000150       __imp_??1CProcessLocalObject@@QAE@XZ 5f72f150     MFC42D:MFC42D.DLL
 0002:00000154       __imp_?GetData@CProcessLocalObject@@QAEPAVCNoTrackObject@@P6GPAV2@XZ@Z 5f72f154     MFC42D:MFC42D.DLL
 0002:00000158       __imp_??3CNoTrackObject@@SGXPAX@Z 5f72f158     MFC42D:MFC42D.DLL
 0002:0000015c       __imp_??2CNoTrackObject@@SGPAXI@Z 5f72f15c     MFC42D:MFC42D.DLL
 0002:00000160       __imp_?GetData@CByteArray@@QAEPAEXZ 5f72f160     MFC42D:MFC42D.DLL
 0002:00000164       __imp_??YCString@@QAEABV0@D@Z 5f72f164     MFC42D:MFC42D.DLL
 0002:00000168       __imp_?SetAt@CMapPtrToPtr@@QAEXPAX0@Z 5f72f168     MFC42D:MFC42D.DLL
 0002:0000016c       __imp_?LockBuffer@CString@@QAEPADXZ 5f72f16c     MFC42D:MFC42D.DLL
 0002:00000170       __imp_??6CDumpContext@@QAEAAV0@E@Z 5f72f170     MFC42D:MFC42D.DLL
 0002:00000174       __imp_??0CByteArray@@QAE@XZ 5f72f174     MFC42D:MFC42D.DLL
 0002:00000178       __imp_?SetSize@CByteArray@@QAEXHH@Z 5f72f178     MFC42D:MFC42D.DLL
 0002:0000017c       __imp_??ACByteArray@@QAEAAEH@Z 5f72f17c     MFC42D:MFC42D.DLL
 0002:00000180       __imp_?GetSize@CByteArray@@QBEHXZ 5f72f180     MFC42D:MFC42D.DLL
 0002:00000184       __imp_??6@YGAAVCDumpContext@@AAV0@VCTime@@@Z 5f72f184     MFC42D:MFC42D.DLL
 0002:00000188       __imp_??0CTime@@QAE@XZ     5f72f188     MFC42D:MFC42D.DLL
 0002:0000018c       __imp_??9CTime@@QBEHV0@@Z  5f72f18c     MFC42D:MFC42D.DLL
 0002:00000190       __imp_??0CTime@@QAE@ABV0@@Z 5f72f190     MFC42D:MFC42D.DLL
 0002:00000194       __imp_??0CTime@@QAE@HHHHHHH@Z 5f72f194     MFC42D:MFC42D.DLL
 0002:00000198       __imp_??4CTime@@QAEABV0@ABV0@@Z 5f72f198     MFC42D:MFC42D.DLL
 0002:0000019c       __imp_??0CTime@@QAE@J@Z    5f72f19c     MFC42D:MFC42D.DLL
 0002:000001a0       __imp_?GetSecond@CTime@@QBEHXZ 5f72f1a0     MFC42D:MFC42D.DLL
 0002:000001a4       __imp_?GetMinute@CTime@@QBEHXZ 5f72f1a4     MFC42D:MFC42D.DLL
 0002:000001a8       __imp_?GetHour@CTime@@QBEHXZ 5f72f1a8     MFC42D:MFC42D.DLL
 0002:000001ac       __imp_?GetDay@CTime@@QBEHXZ 5f72f1ac     MFC42D:MFC42D.DLL
 0002:000001b0       __imp_?GetMonth@CTime@@QBEHXZ 5f72f1b0     MFC42D:MFC42D.DLL
 0002:000001b4       __imp_?GetYear@CTime@@QBEHXZ 5f72f1b4     MFC42D:MFC42D.DLL
 0002:000001b8       __imp_??6CDumpContext@@QAEAAV0@G@Z 5f72f1b8     MFC42D:MFC42D.DLL
 0002:000001bc       __imp_??8CTime@@QBEHV0@@Z  5f72f1bc     MFC42D:MFC42D.DLL
 0002:000001c0       __imp_??8@YG_NABVCString@@0@Z 5f72f1c0     MFC42D:MFC42D.DLL
 0002:000001c4       __imp_?Copy@CByteArray@@QAEXABV1@@Z 5f72f1c4     MFC42D:MFC42D.DLL
 0002:000001c8       __imp_?messageMap@CFormView@@1UAFX_MSGMAP@@B 5f72f1c8     MFC42D:MFC42D.DLL
 0002:000001cc       __imp_?OnEndPrintPreview@CView@@MAEXPAVCDC@@PAUCPrintInfo@@UtagPOINT@@PAVCPreviewView@@@Z 5f72f1cc     MFC42D:MFC42D.DLL
 0002:000001d0       __imp_?OnEndPrinting@CView@@MAEXPAVCDC@@PAUCPrintInfo@@@Z 5f72f1d0     MFC42D:MFC42D.DLL
 0002:000001d4       __imp_?OnPrint@CView@@MAEXPAVCDC@@PAUCPrintInfo@@@Z 5f72f1d4     MFC42D:MFC42D.DLL
 0002:000001d8       __imp_?OnBeginPrinting@CView@@MAEXPAVCDC@@PAUCPrintInfo@@@Z 5f72f1d8     MFC42D:MFC42D.DLL
 0002:000001dc       __imp_?OnPreparePrinting@CView@@MAEHPAUCPrintInfo@@@Z 5f72f1dc     MFC42D:MFC42D.DLL
 0002:000001e0       __imp_?OnDraw@CFormView@@MAEXPAVCDC@@@Z 5f72f1e0     MFC42D:MFC42D.DLL
 0002:000001e4       __imp_?Serialize@CObject@@UAEXAAVCArchive@@@Z 5f72f1e4     MFC42D:MFC42D.DLL
 0002:000001e8       __imp_??1CString@@QAE@XZ   5f72f1e8     MFC42D:MFC42D.DLL
 0002:000001ec       __imp_?OnActivateView@CFormView@@MAEXHPAVCView@@0@Z 5f72f1ec     MFC42D:MFC42D.DLL
 0002:000001f0       __imp_?OnPrepareDC@CScrollView@@UAEXPAVCDC@@PAUCPrintInfo@@@Z 5f72f1f0     MFC42D:MFC42D.DLL
 0002:000001f4       __imp_?OnDragScroll@CView@@UAEKKVCPoint@@@Z 5f72f1f4     MFC42D:MFC42D.DLL
 0002:000001f8       __imp_?OnDropEx@CView@@UAEKPAVCOleDataObject@@KKVCPoint@@@Z 5f72f1f8     MFC42D:MFC42D.DLL
 0002:000001fc       __imp_?OnDrop@CView@@UAEHPAVCOleDataObject@@KVCPoint@@@Z 5f72f1fc     MFC42D:MFC42D.DLL
 0002:00000200       __imp_?OnDragLeave@CView@@UAEXXZ 5f72f200     MFC42D:MFC42D.DLL
 0002:00000204       __imp_?OnDragOver@CView@@UAEKPAVCOleDataObject@@KVCPoint@@@Z 5f72f204     MFC42D:MFC42D.DLL
 0002:00000208       __imp_?OnDragEnter@CView@@UAEKPAVCOleDataObject@@KVCPoint@@@Z 5f72f208     MFC42D:MFC42D.DLL
 0002:0000020c       __imp_?OnScrollBy@CScrollView@@UAEHVCSize@@H@Z 5f72f20c     MFC42D:MFC42D.DLL
 0002:00000210       __imp_?OnScroll@CScrollView@@UAEHIIH@Z 5f72f210     MFC42D:MFC42D.DLL
 0002:00000214       __imp_?IsSelected@CView@@UBEHPBVCObject@@@Z 5f72f214     MFC42D:MFC42D.DLL
 0002:00000218       __imp_?SetOccDialogInfo@CFormView@@MAEHPAU_AFX_OCC_DIALOG_INFO@@@Z 5f72f218     MFC42D:MFC42D.DLL
 0002:0000021c       __imp_?IsFrameWnd@CWnd@@UBEHXZ 5f72f21c     MFC42D:MFC42D.DLL
 0002:00000220       __imp_?CheckAutoCenter@CWnd@@UAEHXZ 5f72f220     MFC42D:MFC42D.DLL
 0002:00000224       __imp_?OnChildNotify@CWnd@@MAEHIIJPAJ@Z 5f72f224     MFC42D:MFC42D.DLL
 0002:00000228       __imp_?PostNcDestroy@CView@@MAEXXZ 5f72f228     MFC42D:MFC42D.DLL
 0002:0000022c       __imp_?DefWindowProcA@CWnd@@MAEJIIJ@Z 5f72f22c     MFC42D:MFC42D.DLL
 0002:00000230       __imp_?OnWndMsg@CWnd@@MAEHIIJPAJ@Z 5f72f230     MFC42D:MFC42D.DLL
 0002:00000234       __imp_?WindowProc@CWnd@@MAEJIIJ@Z 5f72f234     MFC42D:MFC42D.DLL
 0002:00000238       __imp_?OnAmbientProperty@CWnd@@UAEHPAVCOleControlSite@@JPAUtagVARIANT@@@Z 5f72f238     MFC42D:MFC42D.DLL
 0002:0000023c       __imp_?PreTranslateMessage@CFormView@@MAEHPAUtagMSG@@@Z 5f72f23c     MFC42D:MFC42D.DLL
 0002:00000240       __imp_?EndModalState@CWnd@@UAEXXZ 5f72f240     MFC42D:MFC42D.DLL
 0002:00000244       __imp_?BeginModalState@CWnd@@UAEXXZ 5f72f244     MFC42D:MFC42D.DLL
 0002:00000248       __imp_?DoDataExchange@CWnd@@MAEXPAVCDataExchange@@@Z 5f72f248     MFC42D:MFC42D.DLL
 0002:0000024c       __imp_?GetSuperWndProcAddr@CWnd@@MAEPAP6GJPAUHWND__@@IIJ@ZXZ 5f72f24c     MFC42D:MFC42D.DLL
 0002:00000250       __imp_?OnNotify@CWnd@@MAEHIJPAJ@Z 5f72f250     MFC42D:MFC42D.DLL
 0002:00000254       __imp_?OnCommand@CWnd@@MAEHIJ@Z 5f72f254     MFC42D:MFC42D.DLL
 0002:00000258       __imp_?EndModalLoop@CWnd@@UAEXH@Z 5f72f258     MFC42D:MFC42D.DLL
 0002:0000025c       __imp_?ContinueModal@CWnd@@UAEHXZ 5f72f25c     MFC42D:MFC42D.DLL
 0002:00000260       __imp_?WinHelpA@CWnd@@UAEXKI@Z 5f72f260     MFC42D:MFC42D.DLL
 0002:00000264       __imp_?GetScrollBarCtrl@CView@@UBEPAVCScrollBar@@H@Z 5f72f264     MFC42D:MFC42D.DLL
 0002:00000268       __imp_?OnToolHitTest@CWnd@@UBEHVCPoint@@PAUtagTOOLINFOA@@@Z 5f72f268     MFC42D:MFC42D.DLL
 0002:0000026c       __imp_?CalcWindowRect@CScrollView@@UAEXPAUtagRECT@@I@Z 5f72f26c     MFC42D:MFC42D.DLL
 0002:00000270       __imp_?PreCreateWindow@CView@@MAEHAAUtagCREATESTRUCTA@@@Z 5f72f270     MFC42D:MFC42D.DLL
 0002:00000274       __imp_?DestroyWindow@CWnd@@UAEHXZ 5f72f274     MFC42D:MFC42D.DLL
 0002:00000278       __imp_?Create@CFormView@@MAEHPBD0KABUtagRECT@@PAVCWnd@@IPAUCCreateContext@@@Z 5f72f278     MFC42D:MFC42D.DLL
 0002:0000027c       __imp_?PreSubclassWindow@CWnd@@UAEXXZ 5f72f27c     MFC42D:MFC42D.DLL
 0002:00000280       __imp_?GetConnectionHook@CCmdTarget@@MAEPAUIConnectionPoint@@ABU_GUID@@@Z 5f72f280     MFC42D:MFC42D.DLL
 0002:00000284       __imp_?GetExtraConnectionPoints@CCmdTarget@@MAEHPAVCPtrArray@@@Z 5f72f284     MFC42D:MFC42D.DLL
 0002:00000288       __imp_?GetInterfaceHook@CCmdTarget@@UAEPAUIUnknown@@PBX@Z 5f72f288     MFC42D:MFC42D.DLL
 0002:0000028c       __imp_?AfxGetModuleState@@YGPAVAFX_MODULE_STATE@@XZ 5f72f28c     MFC42D:MFC42D.DLL
 0002:00000290       __imp_?GetEventSinkMap@CCmdTarget@@MBEPBUAFX_EVENTSINKMAP@@XZ 5f72f290     MFC42D:MFC42D.DLL
 0002:00000294       __imp_?GetInterfaceMap@CCmdTarget@@MBEPBUAFX_INTERFACEMAP@@XZ 5f72f294     MFC42D:MFC42D.DLL
 0002:00000298       __imp_?GetConnectionMap@CCmdTarget@@MBEPBUAFX_CONNECTIONMAP@@XZ 5f72f298     MFC42D:MFC42D.DLL
 0002:0000029c       __imp_?GetDispatchMap@CCmdTarget@@MBEPBUAFX_DISPMAP@@XZ 5f72f29c     MFC42D:MFC42D.DLL
 0002:000002a0       __imp_?GetCommandMap@CCmdTarget@@MBEPBUAFX_OLECMDMAP@@XZ 5f72f2a0     MFC42D:MFC42D.DLL
 0002:000002a4       __imp_?GetTypeLib@CCmdTarget@@UAEJKPAPAUITypeLib@@@Z 5f72f2a4     MFC42D:MFC42D.DLL
 0002:000002a8       __imp_?GetTypeLibCache@CCmdTarget@@UAEPAVCTypeLibCache@@XZ 5f72f2a8     MFC42D:MFC42D.DLL
 0002:000002ac       __imp_?GetTypeInfoCount@CCmdTarget@@UAEIXZ 5f72f2ac     MFC42D:MFC42D.DLL
 0002:000002b0       __imp_?GetDispatchIID@CCmdTarget@@UAEHPAU_GUID@@@Z 5f72f2b0     MFC42D:MFC42D.DLL
 0002:000002b4       __imp_?IsInvokeAllowed@CCmdTarget@@UAEHJ@Z 5f72f2b4     MFC42D:MFC42D.DLL
 0002:000002b8       __imp_?OnFinalRelease@CWnd@@UAEXXZ 5f72f2b8     MFC42D:MFC42D.DLL
 0002:000002bc       __imp_?OnCmdMsg@CView@@UAEHIHPAXPAUAFX_CMDHANDLERINFO@@@Z 5f72f2bc     MFC42D:MFC42D.DLL
 0002:000002c0       __imp_??0CFormView@@IAE@PBD@Z 5f72f2c0     MFC42D:MFC42D.DLL
 0002:000002c4       __imp_??0CFormView@@IAE@I@Z 5f72f2c4     MFC42D:MFC42D.DLL
 0002:000002c8       __imp_??1CScrollView@@UAE@XZ 5f72f2c8     MFC42D:MFC42D.DLL
 0002:000002cc       __imp_?OnInitialUpdate@CFormView@@UAEXXZ 5f72f2cc     MFC42D:MFC42D.DLL
 0002:000002d0       __imp_??1CWaitCursor@@QAE@XZ 5f72f2d0     MFC42D:MFC42D.DLL
 0002:000002d4       __imp_??0CWaitCursor@@QAE@XZ 5f72f2d4     MFC42D:MFC42D.DLL
 0002:000002d8       __imp_?UpdateData@CWnd@@QAEHH@Z 5f72f2d8     MFC42D:MFC42D.DLL
 0002:000002dc       __imp_?AfxSetWindowText@@YGXPAUHWND__@@PBD@Z 5f72f2dc     MFC42D:MFC42D.DLL
 0002:000002e0       __imp_?PrepareEditCtrl@CDataExchange@@QAEPAUHWND__@@H@Z 5f72f2e0     MFC42D:MFC42D.DLL
 0002:000002e4       __imp_?DDX_Text@@YGXPAVCDataExchange@@HAAH@Z 5f72f2e4     MFC42D:MFC42D.DLL
 0002:000002e8       __imp_?DDX_Text@@YGXPAVCDataExchange@@HAAE@Z 5f72f2e8     MFC42D:MFC42D.DLL
 0002:000002ec       __imp_?DDX_Text@@YGXPAVCDataExchange@@HAAI@Z 5f72f2ec     MFC42D:MFC42D.DLL
 0002:000002f0       __imp_?DDX_Text@@YGXPAVCDataExchange@@HAAJ@Z 5f72f2f0     MFC42D:MFC42D.DLL
 0002:000002f4       __imp_?DDX_Text@@YGXPAVCDataExchange@@HAAK@Z 5f72f2f4     MFC42D:MFC42D.DLL
 0002:000002f8       __imp_?AfxFailMaxChars@@YGXPAVCDataExchange@@H@Z 5f72f2f8     MFC42D:MFC42D.DLL
 0002:000002fc       __imp_?_afxDBCS@@3HB       5f72f2fc     MFC42D:MFC42D.DLL
 0002:00000300       __imp_?GetAllocLength@CString@@QBEHXZ 5f72f300     MFC42D:MFC42D.DLL
 0002:00000304       __imp_?PrepareCtrl@CDataExchange@@QAEPAUHWND__@@H@Z 5f72f304     MFC42D:MFC42D.DLL
 0002:00000308       __imp_?DDX_LBIndex@@YGXPAVCDataExchange@@HAAH@Z 5f72f308     MFC42D:MFC42D.DLL
 0002:0000030c       __imp_?DDX_CBIndex@@YGXPAVCDataExchange@@HAAH@Z 5f72f30c     MFC42D:MFC42D.DLL
 0002:00000310       __imp_?DDX_Scroll@@YGXPAVCDataExchange@@HAAH@Z 5f72f310     MFC42D:MFC42D.DLL
 0002:00000314       __imp_?AfxFailRadio@@YGXPAVCDataExchange@@@Z 5f72f314     MFC42D:MFC42D.DLL
 0002:00000318       __imp_?DDX_Radio@@YGXPAVCDataExchange@@HAAH@Z 5f72f318     MFC42D:MFC42D.DLL
 0002:0000031c       __imp_?AssertValid@CFormView@@UBEXXZ 5f72f31c     MFC42D:MFC42D.DLL
 0002:00000320       __imp_?Dump@CFormView@@UBEXAAVCDumpContext@@@Z 5f72f320     MFC42D:MFC42D.DLL
 0002:00000324       __imp_?OnMove@CWnd@@IAEXHH@Z 5f72f324     MFC42D:MFC42D.DLL
 0002:00000328       __imp_?classCFormView@CFormView@@2UCRuntimeClass@@B 5f72f328     MFC42D:MFC42D.DLL
 0002:0000032c       __imp_??6CDumpContext@@QAEAAV0@M@Z 5f72f32c     MFC42D:MFC42D.DLL
 0002:00000330       __imp_??6CDumpContext@@QAEAAV0@N@Z 5f72f330     MFC42D:MFC42D.DLL
 0002:00000334       __imp_?AfxTextFloatFormat@@YGXPAVCDataExchange@@HPAXNH@Z 5f72f334     MFC42D:MFC42D.DLL
 0002:00000338       __imp_?IsEmpty@CMapPtrToPtr@@QBEHXZ 5f72f338     MFC42D:MFC42D.DLL
 0002:0000033c       __imp_?RemoveKey@CMapPtrToPtr@@QAEHPAX@Z 5f72f33c     MFC42D:MFC42D.DLL
 0002:00000340       __imp_?RemoveAll@CMapPtrToPtr@@QAEXXZ 5f72f340     MFC42D:MFC42D.DLL
 0002:00000344       __imp_?GetNextAssoc@CMapPtrToPtr@@QBEXAAPAU__POSITION@@AAPAX1@Z 5f72f344     MFC42D:MFC42D.DLL
 0002:00000348       __imp_?GetStartPosition@CMapPtrToPtr@@QBEPAU__POSITION@@XZ 5f72f348     MFC42D:MFC42D.DLL
 0002:0000034c       __imp_??0CString@@QAE@ABV0@@Z 5f72f34c     MFC42D:MFC42D.DLL
 0002:00000350       __imp_??3CNoTrackObject@@SGXPAXPBDH@Z 5f72f350     MFC42D:MFC42D.DLL
 0002:00000354       __imp_??2CNoTrackObject@@SGPAXIPBDH@Z 5f72f354     MFC42D:MFC42D.DLL
 0002:00000358       __imp_?AfxGetApp@@YGPAVCWinApp@@XZ 5f72f358     MFC42D:MFC42D.DLL
 0002:0000035c       __imp_??6CDumpContext@@QAEAAV0@ABVCObject@@@Z 5f72f35c     MFC42D:MFC42D.DLL
 0002:00000360       __imp_?DDX_Text@@YGXPAVCDataExchange@@HAAF@Z 5f72f360     MFC42D:MFC42D.DLL
 0002:00000364       __imp_?DDX_Text@@YGXPAVCDataExchange@@HAAM@Z 5f72f364     MFC42D:MFC42D.DLL
 0002:00000368       __imp_?DDX_Text@@YGXPAVCDataExchange@@HAAN@Z 5f72f368     MFC42D:MFC42D.DLL
 0002:0000036c       __imp_?DDX_Text@@YGXPAVCDataExchange@@HAAVCString@@@Z 5f72f36c     MFC42D:MFC42D.DLL
 0002:00000370       __imp_?DDX_Text@@YGXPAVCDataExchange@@HPADH@Z 5f72f370     MFC42D:MFC42D.DLL
 0002:00000374       __imp_?DDX_Slider@@YGXPAVCDataExchange@@HAAH@Z 5f72f374     MFC42D:MFC42D.DLL
 0002:00000378       __imp_?AssertValid@CObject@@UBEXXZ 5f72f378     MFC42D:MFC42D.DLL
 0002:0000037c       __imp_?Dump@CObject@@UBEXAAVCDumpContext@@@Z 5f72f37c     MFC42D:MFC42D.DLL
 0002:00000380       __imp_?ReportError@CException@@UAEHII@Z 5f72f380     MFC42D:MFC42D.DLL
 0002:00000384       __imp_??2CObject@@SGPAXIPBDH@Z 5f72f384     MFC42D:MFC42D.DLL
 0002:00000388       __imp_?LoadStringA@CString@@QAEHI@Z 5f72f388     MFC42D:MFC42D.DLL
 0002:0000038c       __imp_?AfxTrace@@YAXPBDZZ  5f72f38c     MFC42D:MFC42D.DLL
 0002:00000390       __imp_??3CException@@SGXPAXPBDH@Z 5f72f390     MFC42D:MFC42D.DLL
 0002:00000394       __imp_??3CException@@SGXPAX@Z 5f72f394     MFC42D:MFC42D.DLL
 0002:00000398       __imp_??2@YAPAXI@Z         5f72f398     MFC42D:MFC42D.DLL
 0002:0000039c       __imp_??3@YAXPAX@Z         5f72f39c     MFC42D:MFC42D.DLL
 0002:000003a0       __imp_?AfxGetAppModuleState@@YGPAVAFX_MODULE_STATE@@XZ 5f72f3a0     MFC42D:MFC42D.DLL
 0002:000003a4       __imp_??3CObject@@SGXPAX@Z 5f72f3a4     MFC42D:MFC42D.DLL
 0002:000003a8       __imp_?AfxInitExtensionModule@@YGHAAUAFX_EXTENSION_MODULE@@PAUHINSTANCE__@@@Z 5f72f3a8     MFC42D:MFC42D.DLL
 0002:000003ac       __imp_?AfxAssertFailedLine@@YGHPBDH@Z 5f72f3ac     MFC42D:MFC42D.DLL
 0002:000003b0       __imp_??2CObject@@SGPAXI@Z 5f72f3b0     MFC42D:MFC42D.DLL
 0002:000003b4       __imp_??0CDynLinkLibrary@@QAE@AAUAFX_EXTENSION_MODULE@@H@Z 5f72f3b4     MFC42D:MFC42D.DLL
 0002:000003b8       __imp_?AfxTermExtensionModule@@YGXAAUAFX_EXTENSION_MODULE@@H@Z 5f72f3b8     MFC42D:MFC42D.DLL
 0002:000003bc       __imp_?AfxTermThread@@YGXPAUHINSTANCE__@@@Z 5f72f3bc     MFC42D:MFC42D.DLL
 0002:000003c0       __imp_?OnActivateFrame@CFormView@@MAEXIPAVCFrameWnd@@@Z 5f72f3c0     MFC42D:MFC42D.DLL
 0002:000003c4       __imp_?OnUpdate@CView@@MAEXPAV1@JPAVCObject@@@Z 5f72f3c4     MFC42D:MFC42D.DLL
 0002:000003c8       __imp_?OnCreateAggregates@CCmdTarget@@UAEHXZ 5f72f3c8     MFC42D:MFC42D.DLL
 0002:000003cc       \177MFC42D_NULL_THUNK_DATA 5f72f3cc     MFC42D:MFC42D.DLL
 0002:000003d0       __imp_??0COleDateTime@@QAE@HHHHHH@Z 5f72f3d0     MFCO42D:MFCO42D.DLL
 0002:000003d4       __imp_??4COleVariant@@QAEABV0@J@Z 5f72f3d4     MFCO42D:MFCO42D.DLL
 0002:000003d8       __imp_??4COleDateTime@@QAEABV0@ABUtagVARIANT@@@Z 5f72f3d8     MFCO42D:MFCO42D.DLL
 0002:000003dc       __imp_??BCOleVariant@@QAEPAUtagVARIANT@@XZ 5f72f3dc     MFCO42D:MFCO42D.DLL
 0002:000003e0       __imp_??0COleDateTime@@QAE@N@Z 5f72f3e0     MFCO42D:MFCO42D.DLL
 0002:000003e4       __imp_??0COleVariant@@QAE@FG@Z 5f72f3e4     MFCO42D:MFCO42D.DLL
 0002:000003e8       __imp_??0COleVariant@@QAE@ABUtagVARIANT@@@Z 5f72f3e8     MFCO42D:MFCO42D.DLL
 0002:000003ec       __imp_??4COleVariant@@QAEABV0@QBD@Z 5f72f3ec     MFCO42D:MFCO42D.DLL
 0002:000003f0       __imp_?SetStatus@COleCurrency@@QAEXW4CurrencyStatus@1@@Z 5f72f3f0     MFCO42D:MFCO42D.DLL
 0002:000003f4       __imp_?GetStatus@COleCurrency@@QBE?AW4CurrencyStatus@1@XZ 5f72f3f4     MFCO42D:MFCO42D.DLL
 0002:000003f8       __imp_??0COleCurrency@@QAE@XZ 5f72f3f8     MFCO42D:MFCO42D.DLL
 0002:000003fc       __imp_??4COleCurrency@@QAEABV0@ABV0@@Z 5f72f3fc     MFCO42D:MFCO42D.DLL
 0002:00000400       __imp_??9COleDateTime@@QBEHABV0@@Z 5f72f400     MFCO42D:MFCO42D.DLL
 0002:00000404       __imp_??9COleCurrency@@QBEHABV0@@Z 5f72f404     MFCO42D:MFCO42D.DLL
 0002:00000408       __imp_??4COleVariant@@QAEABV0@ABVCOleDateTime@@@Z 5f72f408     MFCO42D:MFCO42D.DLL
 0002:0000040c       __imp_??4COleVariant@@QAEABV0@N@Z 5f72f40c     MFCO42D:MFCO42D.DLL
 0002:00000410       __imp_??4COleVariant@@QAEABV0@M@Z 5f72f410     MFCO42D:MFCO42D.DLL
 0002:00000414       __imp_??4COleVariant@@QAEABV0@ABVCOleCurrency@@@Z 5f72f414     MFCO42D:MFCO42D.DLL
 0002:00000418       __imp_??4COleVariant@@QAEABV0@F@Z 5f72f418     MFCO42D:MFCO42D.DLL
 0002:0000041c       __imp_??4COleVariant@@QAEABV0@E@Z 5f72f41c     MFCO42D:MFCO42D.DLL
 0002:00000420       __imp_??4COleVariant@@QAEABV0@ABVCLongBinary@@@Z 5f72f420     MFCO42D:MFCO42D.DLL
 0002:00000424       __imp_??4COleVariant@@QAEABV0@ABVCByteArray@@@Z 5f72f424     MFCO42D:MFCO42D.DLL
 0002:00000428       __imp_??6@YGAAVCDumpContext@@AAV0@VCOleCurrency@@@Z 5f72f428     MFCO42D:MFCO42D.DLL
 0002:0000042c       __imp_??0COleCurrency@@QAE@ABV0@@Z 5f72f42c     MFCO42D:MFCO42D.DLL
 0002:00000430       __imp_??4COleVariant@@QAEABV0@ABV0@@Z 5f72f430     MFCO42D:MFCO42D.DLL
 0002:00000434       __imp_??8COleVariant@@QBEHABUtagVARIANT@@@Z 5f72f434     MFCO42D:MFCO42D.DLL
 0002:00000438       __imp_?DDX_Text@@YGXPAVCDataExchange@@HAAVCOleCurrency@@@Z 5f72f438     MFCO42D:MFCO42D.DLL
 0002:0000043c       __imp_?DDX_Text@@YGXPAVCDataExchange@@HAAVCOleDateTime@@@Z 5f72f43c     MFCO42D:MFCO42D.DLL
 0002:00000440       __imp_?Format@COleDateTime@@QBE?AVCString@@KK@Z 5f72f440     MFCO42D:MFCO42D.DLL
 0002:00000444       __imp_?SetStatus@COleDateTime@@QAEXW4DateTimeStatus@1@@Z 5f72f444     MFCO42D:MFCO42D.DLL
 0002:00000448       __imp_?GetStatus@COleDateTime@@QBE?AW4DateTimeStatus@1@XZ 5f72f448     MFCO42D:MFCO42D.DLL
 0002:0000044c       __imp_?GetSecond@COleDateTime@@QBEHXZ 5f72f44c     MFCO42D:MFCO42D.DLL
 0002:00000450       __imp_?GetMinute@COleDateTime@@QBEHXZ 5f72f450     MFCO42D:MFCO42D.DLL
 0002:00000454       __imp_??0COleDateTime@@QAE@XZ 5f72f454     MFCO42D:MFCO42D.DLL
 0002:00000458       __imp_?GetDay@COleDateTime@@QBEHXZ 5f72f458     MFCO42D:MFCO42D.DLL
 0002:0000045c       __imp_??4COleDateTime@@QAEABV0@ABV0@@Z 5f72f45c     MFCO42D:MFCO42D.DLL
 0002:00000460       __imp_?GetHour@COleDateTime@@QBEHXZ 5f72f460     MFCO42D:MFCO42D.DLL
 0002:00000464       __imp_?GetMonth@COleDateTime@@QBEHXZ 5f72f464     MFCO42D:MFCO42D.DLL
 0002:00000468       __imp_?GetYear@COleDateTime@@QBEHXZ 5f72f468     MFCO42D:MFCO42D.DLL
 0002:0000046c       __imp_??8COleDateTime@@QBEHABV0@@Z 5f72f46c     MFCO42D:MFCO42D.DLL
 0002:00000470       __imp_??0COleVariant@@QAE@PBDG@Z 5f72f470     MFCO42D:MFCO42D.DLL
 0002:00000474       __imp_??6@YGAAVCDumpContext@@AAV0@VCOleDateTime@@@Z 5f72f474     MFCO42D:MFCO42D.DLL
 0002:00000478       __imp_??1COleVariant@@QAE@XZ 5f72f478     MFCO42D:MFCO42D.DLL
 0002:0000047c       __imp_??6@YGAAVCDumpContext@@AAV0@VCOleVariant@@@Z 5f72f47c     MFCO42D:MFCO42D.DLL
 0002:00000480       __imp_??0COleVariant@@QAE@ABV0@@Z 5f72f480     MFCO42D:MFCO42D.DLL
 0002:00000484       __imp_??0COleVariant@@QAE@JG@Z 5f72f484     MFCO42D:MFCO42D.DLL
 0002:00000488       __imp_??0COleVariant@@QAE@XZ 5f72f488     MFCO42D:MFCO42D.DLL
 0002:0000048c       __imp_??0COleDateTime@@QAE@ABV0@@Z 5f72f48c     MFCO42D:MFCO42D.DLL
 0002:00000490       __imp_?Clear@COleVariant@@QAEXXZ 5f72f490     MFCO42D:MFCO42D.DLL
 0002:00000494       \177MFCO42D_NULL_THUNK_DATA 5f72f494     MFCO42D:MFCO42D.DLL
 0002:00000498       __imp_??1type_info@@UAE@XZ 5f72f498     msvcrtd:MSVCRTD.dll
 0002:0000049c       __imp____dllonexit         5f72f49c     msvcrtd:MSVCRTD.dll
 0002:000004a0       __imp___free_dbg           5f72f4a0     msvcrtd:MSVCRTD.dll
 0002:000004a4       __imp___onexit             5f72f4a4     msvcrtd:MSVCRTD.dll
 0002:000004a8       __imp_?terminate@@YAXXZ    5f72f4a8     msvcrtd:MSVCRTD.dll
 0002:000004ac       __imp___except_handler3    5f72f4ac     msvcrtd:MSVCRTD.dll
 0002:000004b0       __imp___vsnprintf          5f72f4b0     msvcrtd:MSVCRTD.dll
 0002:000004b4       __imp___adjust_fdiv        5f72f4b4     msvcrtd:MSVCRTD.dll
 0002:000004b8       __imp___mbctype            5f72f4b8     msvcrtd:MSVCRTD.dll
 0002:000004bc       __imp___purecall           5f72f4bc     msvcrtd:MSVCRTD.dll
 0002:000004c0       __imp__memcmp              5f72f4c0     msvcrtd:MSVCRTD.dll
 0002:000004c4       __imp__labs                5f72f4c4     msvcrtd:MSVCRTD.dll
 0002:000004c8       __imp__memset              5f72f4c8     msvcrtd:MSVCRTD.dll
 0002:000004cc       __imp___mbsstr             5f72f4cc     msvcrtd:MSVCRTD.dll
 0002:000004d0       __imp__memcpy              5f72f4d0     msvcrtd:MSVCRTD.dll
 0002:000004d4       __imp___CxxThrowException@8 5f72f4d4     msvcrtd:MSVCRTD.dll
 0002:000004d8       __imp___mbsinc             5f72f4d8     msvcrtd:MSVCRTD.dll
 0002:000004dc       __imp___mbsnbicmp          5f72f4dc     msvcrtd:MSVCRTD.dll
 0002:000004e0       __imp___initterm           5f72f4e0     msvcrtd:MSVCRTD.dll
 0002:000004e4       __imp____CxxFrameHandler   5f72f4e4     msvcrtd:MSVCRTD.dll
 0002:000004e8       __imp___malloc_dbg         5f72f4e8     msvcrtd:MSVCRTD.dll
 0002:000004ec       __imp__abs                 5f72f4ec     msvcrtd:MSVCRTD.dll
 0002:000004f0       __imp___CrtDbgReport       5f72f4f0     msvcrtd:MSVCRTD.dll
 0002:000004f4       \177MSVCRTD_NULL_THUNK_DATA 5f72f4f4     msvcrtd:MSVCRTD.dll
 0002:000004f8       __imp__SendMessageA@16     5f72f4f8     user32:USER32.dll
 0002:000004fc       __imp__GetWindowLongA@8    5f72f4fc     user32:USER32.dll
 0002:00000500       __imp__GetWindowTextA@12   5f72f500     user32:USER32.dll
 0002:00000504       __imp__GetDesktopWindow@0  5f72f504     user32:USER32.dll
 0002:00000508       __imp__EnableWindow@8      5f72f508     user32:USER32.dll
 0002:0000050c       __imp__wsprintfA           5f72f50c     user32:USER32.dll
 0002:00000510       __imp__GetWindowTextLengthA@4 5f72f510     user32:USER32.dll
 0002:00000514       \177USER32_NULL_THUNK_DATA 5f72f514     user32:USER32.dll
 0002:00000540       _IID_IDocHostUIHandlerDispatch 5f72f540     dlldb.obj
 0002:00000550       _IID_IInternalConnection   5f72f550     dlldb.obj
 0002:00000560       _IID_IAxWinAmbientDispatch 5f72f560     dlldb.obj
 0002:00000570       _IID_IAxWinHostWindow      5f72f570     dlldb.obj
 0002:00000580       _IID_IRegistrar            5f72f580     dlldb.obj
 0002:00000590       _CLSID_Registrar           5f72f590     dlldb.obj
 0002:000005a0       _LIBID_ATLLib              5f72f5a0     dlldb.obj
 0002:000005b0       ??_C@_0M@EAGE@MFCO42D?4DLL?$AA@ 5f72f5b0     dlldb.obj
 0002:000005bc       ??_C@_0L@LDKI@MFC42D?4DLL?$AA@ 5f72f5bc     dlldb.obj
 0002:000005c8       ?classCRecordset@CRecordset@@2UCRuntimeClass@@B 5f72f5c8     dbcore.obj
 0002:000005e0       ??_C@_0L@FKJL@CRecordset?$AA@ 5f72f5e0     dbcore.obj
 0002:000005f0       ?classCDatabase@CDatabase@@2UCRuntimeClass@@B 5f72f5f0     dbcore.obj
 0002:00000608       ??_C@_09CDJB@CDatabase?$AA@ 5f72f608     dbcore.obj
 0002:00000618       ?classCDBException@CDBException@@2UCRuntimeClass@@B 5f72f618     dbcore.obj
 0002:00000630       ??_C@_0N@GGEG@CDBException?$AA@ 5f72f630     dbcore.obj
 0002:00000640       ?_afxODBCDLL@@3QBDB        5f72f640     dbcore.obj
 0002:0000064c       ?_afxDriverNotCapable@@3QBDB 5f72f64c     dbcore.obj
 0002:00000658       ?_afxOutOfSequence@@3QBDB  5f72f658     dbcore.obj
 0002:00000664       ?_afxInfoRange@@3QBDB      5f72f664     dbcore.obj
 0002:00000670       ?_afxDataTruncated@@3QBDB  5f72f670     dbcore.obj
 0002:0000067c       ?_afxRowFetch@@3QBDB       5f72f67c     dbcore.obj
 0002:00000688       ?_afxForUpdate@@3QBDB      5f72f688     dbcore.obj
 0002:00000698       ?_afxOrderBy@@3QBDB        5f72f698     dbcore.obj
 0002:000006a4       ?_afxWhere@@3QBDB          5f72f6a4     dbcore.obj
 0002:000006ac       ?_afxFrom@@3QBDB           5f72f6ac     dbcore.obj
 0002:000006b4       ?_afxSelect@@3QBDB         5f72f6b4     dbcore.obj
 0002:000006bc       ?_afxParamCall@@3QBDB      5f72f6bc     dbcore.obj
 0002:000006c0       ?_afxCall@@3QBDB           5f72f6c0     dbcore.obj
 0002:000006c8       ?_afxLiteralSeparator@@3DB 5f72f6c8     dbcore.obj
 0002:000006cc       ?_afxComma@@3QBDB          5f72f6cc     dbcore.obj
 0002:000006d0       ?_afxODBCTrail@@3QBDB      5f72f6d0     dbcore.obj
 0002:000006d8       ??_C@_03HHKO@?$CFs?6?$AA@  5f72f6d8     dbcore.obj
 0002:000006e0       ??_7CDBException@@6B@      5f72f6e0     dbcore.obj
 0002:00000700       ??_C@_06LPPO@State?3?$AA@  5f72f700     dbcore.obj
 0002:00000708       ??_C@_01BJG@?6?$AA@        5f72f708     dbcore.obj
 0002:0000070c       ??_C@_0BE@DKOK@?0Native?3?$CFld?0Origin?3?$AA@ 5f72f70c     dbcore.obj
 0002:00000720       ??_C@_05NOEI@00000?$AA@    5f72f720     dbcore.obj
 0002:0000072c       ??_7CDatabase@@6B@         5f72f72c     dbcore.obj
 0002:0000075c       ??_C@_05LDGB@?$DLDSN?$DN?$AA@ 5f72f75c     dbcore.obj
 0002:00000764       ??_C@_02DILL@?$CFs?$AA@    5f72f764     dbcore.obj
 0002:00000768       ??_C@_0DB@JAJD@Error?3?5Missing?5?8ODBC?8?5prefix?5on?5@ 5f72f768     dbcore.obj
 0002:0000079c       ??_C@_0DJ@GKAP@Error?3?5SQLFreeEnv?5failure?5ignore@ 5f72f79c     dbcore.obj
 0002:000007d8       ??_C@_0EG@KPGE@Error?3?5exception?5by?5CDatabase?3?3C@ 5f72f7d8     dbcore.obj
 0002:00000820       ??_C@_0CC@OCAA@Warning?3?5ODBC?5Success?5With?5Info?0@ 5f72f820     dbcore.obj
 0002:00000844       ??_C@_0DB@KFIB@Warning?3?5Failure?5setting?5read?5on@ 5f72f844     dbcore.obj
 0002:00000878       ??_C@_0CJ@ICAI@Warning?3?5Failure?5setting?5login?5t@ 5f72f878     dbcore.obj
 0002:000008a4       ??_C@_0N@PKHK@odbccall?4txt?$AA@ 5f72f8a4     dbcore.obj
 0002:000008b4       ??_C@_0EK@BBMC@Error?3?5No?5default?5window?5?$CIAfxGet@ 5f72f8b4     dbcore.obj
 0002:00000900       ??_C@_0P@NHLG@?0?5Version?3?5?$CFs?6?$AA@ 5f72f900     dbcore.obj
 0002:00000910       ??_C@_09FDEN@DBMS?3?5?$CFs?6?$AA@ 5f72f910     dbcore.obj
 0002:0000091c       ??_C@_0CD@KCJE@Warning?3?5data?5source?5is?5readonly@ 5f72f91c     dbcore.obj
 0002:00000940       ??_C@_01PCJP@Y?$AA@        5f72f940     dbcore.obj
 0002:00000944       ??_C@_0BI@MNAB@?6?7henvAllConnections?5?$DN?5?$AA@ 5f72f944     dbcore.obj
 0002:0000095c       ??_C@_0BA@LDLC@?6?7nAllocated?5?$DN?5?$AA@ 5f72f95c     dbcore.obj
 0002:0000096c       ??_C@_0L@OKHO@?6with?5env?3?$AA@ 5f72f96c     dbcore.obj
 0002:00000978       ??_C@_0BF@DMHA@?6m_dwQueryTimeout?5?$DN?5?$AA@ 5f72f978     dbcore.obj
 0002:00000990       ??_C@_0BF@BECC@?6m_dwLoginTimeout?5?$DN?5?$AA@ 5f72f990     dbcore.obj
 0002:000009a8       ??_C@_0BK@IHG@?6m_bTransactionPending?5?$DN?5?$AA@ 5f72f9a8     dbcore.obj
 0002:000009c4       ??_C@_0BE@HNE@?6m_bTransactions?5?$DN?5?$AA@ 5f72f9c4     dbcore.obj
 0002:000009d8       ??_C@_0BB@FGMM@?6m_bUpdatable?5?$DN?5?$AA@ 5f72f9d8     dbcore.obj
 0002:000009ec       ??_C@_0BB@MLGK@?6m_strConnect?5?$DN?5?$AA@ 5f72f9ec     dbcore.obj
 0002:00000a00       ??_C@_09DBDF@m_hdbc?5?$DN?5?$AA@ 5f72fa00     dbcore.obj
 0002:00000a10       ??_7CRecordset@@6B@        5f72fa10     dbcore.obj
 0002:00000a78       ??_C@_0CM@IFBK@Error?3?5Exception?5ignored?5in?5?$HOCRe@ 5f72fa78     dbcore.obj
 0002:00000aa4       ??_C@_0CI@FBKI@?6to?5Close?5or?5memory?5leaks?5will?5r@ 5f72faa4     dbcore.obj
 0002:00000acc       ??_C@_0CP@EMLF@?6Use?5of?5multi?5row?5fetch?5requires@ 5f72facc     dbcore.obj
 0002:00000afc       ??_C@_0DD@JAID@?6WARNING?3?5Close?5called?5implicitl@ 5f72fafc     dbcore.obj
 0002:00000b30       ??_C@_0EB@JOFO@WARNING?3?5CRecordset?5not?5found?5in@ 5f72fb30     dbcore.obj
 0002:00000b74       ??_C@_0DB@LKMN@Error?3?5SQLNumResultCols?5failed?5d@ 5f72fb74     dbcore.obj
 0002:00000ba8       ??_C@_0CC@LBHG@Warning?3?5ODBC?5Success?5With?5Info?0@ 5f72fba8     dbcore.obj
 0002:00000bcc       ??_C@_0CC@PFCL@Error?3?5fetching?5row?5from?5server?4@ 5f72fbcc     dbcore.obj
 0002:00000bf0       ??_C@_0DA@PPCC@Error?3?5field?5data?5truncated?5duri@ 5f72fbf0     dbcore.obj
 0002:00000c20       ??_C@_0CG@LDBG@Error?3?5GetBookmark?5operation?5fai@ 5f72fc20     dbcore.obj
 0002:00000c48       ??_C@_0DM@NDCP@Error?3?5attempt?5to?5lock?5record?5fa@ 5f72fc48     dbcore.obj
 0002:00000c84       ??_C@_0CP@DMCL@Error?3?5Edit?5attempt?5failed?5?9?5not@ 5f72fc84     dbcore.obj
 0002:00000cb4       ??_C@_0DI@HNOF@Error?3?5must?5enter?5Edit?5or?5AddNew@ 5f72fcb4     dbcore.obj
 0002:00000cec       ??_C@_0EA@HBMB@Error?3?5attempted?5to?5delete?5while@ 5f72fcec     dbcore.obj
 0002:00000d2c       ??_C@_0CH@IBHN@Error?3?5attempt?5FlushResultSet?5fa@ 5f72fd2c     dbcore.obj
 0002:00000d54       ??_C@_0CA@OHDE@Error?3?5Requery?5attempt?5failed?4?6?$AA@ 5f72fd54     dbcore.obj
 0002:00000d74       ??_C@_00A@?$AA@            5f72fd74     dbcore.obj
 0002:00000d78       ??_C@_0DC@BJBD@Warning?3?5Setting?5forwardOnly?5rec@ 5f72fd78     dbcore.obj
 0002:00000dac       ??_C@_0DA@LMIK@Error?3?5CDatabase?5create?5for?5CRec@ 5f72fdac     dbcore.obj
 0002:00000ddc       ??_C@_0DH@FPLF@Error?3?5ODBC?5failure?5checking?5for@ 5f72fddc     dbcore.obj
 0002:00000e14       ??_C@_0CH@KFOF@?7Marking?5CRecordset?5as?5not?5updat@ 5f72fe14     dbcore.obj
 0002:00000e3c       ??_C@_0CJ@BALP@Warning?3?5Concurrency?5changed?5by?5@ 5f72fe3c     dbcore.obj
 0002:00000e68       ??_C@_0DE@DFFH@Error?3?5ODBC?5failure?5on?5SQLPrepar@ 5f72fe68     dbcore.obj
 0002:00000e9c       ??_C@_0DE@LDDI@Error?3?5ODBC?5failure?5setting?5reco@ 5f72fe9c     dbcore.obj
 0002:00000ed0       ??_C@_0CH@JGDM@Warning?3?5Setting?5recordset?5read?5@ 5f72fed0     dbcore.obj
 0002:00000ef8       ??_C@_0DJ@GKLE@Warning?3?5Driver?5does?5not?5support@ 5f72fef8     dbcore.obj
 0002:00000f34       ??_C@_0BI@EIOA@for?5use?5with?5SQLFetch?4?6?$AA@ 5f72ff34     dbcore.obj
 0002:00000f4c       ??_C@_0DI@PHNH@and?1or?5cursor?5library?5not?5loaded@ 5f72ff4c     dbcore.obj
 0002:00000f84       ??_C@_0DD@KIDP@Warning?3?5SQLExtendedFetch?5not?5su@ 5f72ff84     dbcore.obj
 0002:00000fb8       ??_C@_0EC@ENHP@Error?3?5ODBC?5failure?5determining?5@ 5f72ffb8     dbcore.obj
 0002:00000ffc       ??_C@_0CN@MMNF@Error?3?5ODBC?5failure?5getting?5fiel@ 5f72fffc     dbcore.obj
 0002:0000102c       ??_C@_0BO@OJF@Error?3?5Can?8t?5get?5field?5info?4?6?$AA@ 5f73002c     dbcore.obj
 0002:0000104c       ??_C@_0CH@FBFK@Error?3?5Can?8t?5enable?5bookmark?5sup@ 5f73004c     dbcore.obj
 0002:00001074       ??_C@_0DE@LOJN@Error?3?5ODBC?5failure?5setting?5reco@ 5f730074     dbcore.obj
 0002:000010a8       ??_C@_0DO@CDMH@Warning?3?5locking?5not?5supported?0?5@ 5f7300a8     dbcore.obj
 0002:000010e8       ??_C@_0DG@DPND@Error?3?5ODBC?5failure?5checking?5rec@ 5f7300e8     dbcore.obj
 0002:00001120       ??_C@_0DG@DIEO@Warning?3?5SQL?5contains?5join?0?5reco@ 5f730120     dbcore.obj
 0002:00001158       ??_C@_0DL@MOFF@Warning?3?5SQL?5contains?5?8?5UNION?5?8?0@ 5f730158     dbcore.obj
 0002:00001194       ??_C@_07CBOJ@?5UNION?5?$AA@ 5f730194     dbcore.obj
 0002:0000119c       ??_C@_0DO@EPAM@Warning?3?5SQL?5contains?5?8?5GROUP?5BY@ 5f73019c     dbcore.obj
 0002:000011dc       ??_C@_0L@GEHL@?5GROUP?5BY?5?$AA@ 5f7301dc     dbcore.obj
 0002:000011e8       ??_C@_0DF@PAPE@Warning?3?5Missing?5?8?5FROM?5?8?0?5recor@ 5f7301e8     dbcore.obj
 0002:00001220       ??_C@_06FHM@?5JOIN?5?$AA@  5f730220     dbcore.obj
 0002:00001228       ??_C@_0CG@JONH@Error?3?5attempted?5to?5move?5before?5@ 5f730228     dbcore.obj
 0002:00001250       ??_C@_0CE@ELBP@Error?3?5attempted?5to?5move?5past?5EO@ 5f730250     dbcore.obj
 0002:00001274       ??_C@_0DJ@JCEJ@Error?3?5attempted?5to?5position?5cur@ 5f730274     dbcore.obj
 0002:000012b0       ??_C@_0DH@HGN@Error?3?5forward?9only?5recordsets?5o@ 5f7302b0     dbcore.obj
 0002:000012e8       ??_C@_0CO@HBII@Error?3?5no?5field?5names?5?9?5at?5least@ 5f7302e8     dbcore.obj
 0002:00001318       ??_C@_01KMAE@?0?$AA@       5f730318     dbcore.obj
 0002:0000131c       ??_C@_0EJ@LAA@Warning?3?5Setting?5recordset?5read?5@ 5f73031c     dbcore.obj
 0002:00001368       ??_C@_0CC@NBNH@?7Will?5use?5positioned?5update?5SQL?4@ 5f730368     dbcore.obj
 0002:0000138c       ??_C@_0EB@HMHM@Warning?3?5Can?8t?5use?5SQLSetPos?5due@ 5f73038c     dbcore.obj
 0002:000013d0       ??_C@_0CB@NKLD@Error?3?5failure?5updating?5record?4?6@ 5f7303d0     dbcore.obj
 0002:000013f4       ??_C@_0CO@KNLC@Error?3?5failure?5to?5allocate?5updat@ 5f7303f4     dbcore.obj
 0002:00001424       ??_C@_0BD@CPP@?5WHERE?5CURRENT?5OF?5?$AA@ 5f730424     dbcore.obj
 0002:00001438       ??_C@_05DNFI@?5SET?5?$AA@  5f730438     dbcore.obj
 0002:00001440       ??_C@_07EKDD@UPDATE?5?$AA@ 5f730440     dbcore.obj
 0002:00001448       ??_C@_09CGAE@?5VALUES?5?$CI?$AA@ 5f730448     dbcore.obj
 0002:00001454       ??_C@_02NDAK@?5?$CI?$AA@   5f730454     dbcore.obj
 0002:00001458       ??_C@_0N@KHCN@INSERT?5INTO?5?$AA@ 5f730458     dbcore.obj
 0002:00001468       ??_C@_0N@MCBO@DELETE?5FROM?5?$AA@ 5f730468     dbcore.obj
 0002:00001478       ??_C@_0DN@EOJO@Warning?3?5?$CFu?5rows?5affected?5by?5upd@ 5f730478     dbcore.obj
 0002:000014b8       ??_C@_0DK@OEHO@Error?3?5failure?5handling?5long?5bin@ 5f7304b8     dbcore.obj
 0002:000014f4       ??_C@_0ED@MCNJ@Error?3?5attempting?5to?5update?5reco@ 5f7304f4     dbcore.obj
 0002:00001538       ??_C@_0DD@IDOM@Error?3?5attempted?5to?5update?5a?5rea@ 5f730538     dbcore.obj
 0002:0000156c       ??_C@_0DM@OKHE@Error?3?5attempted?5to?5add?5a?5record@ 5f73056c     dbcore.obj
 0002:000015a8       ??_C@_0CH@NCA@?7Data?5already?5fetched?5for?5this?5f@ 5f7305a8     dbcore.obj
 0002:000015d0       ??_C@_0DE@MBPN@Error?3?5GetFieldValue?5operation?5f@ 5f7305d0     dbcore.obj
 0002:00001604       ??_C@_0CO@IONN@Warning?3?5ODBC?5Success?5With?5Info?5@ 5f730604     dbcore.obj
 0002:00001634       ??_C@_0BA@BGHA@with?5database?3?5?$AA@ 5f730634     dbcore.obj
 0002:00001644       ??_C@_0BC@MKGN@with?5no?5database?6?$AA@ 5f730644     dbcore.obj
 0002:00001658       ??_C@_0CP@HPBB@?6Dump?5values?5for?5each?5field?5in?5c@ 5f730658     dbcore.obj
 0002:00001688       ??_C@_0BC@JNKN@?6m_hstmtUpdate?5?$DN?5?$AA@ 5f730688     dbcore.obj
 0002:0000169c       ??_C@_0BE@OFAF@?6m_strCursorName?5?$DN?5?$AA@ 5f73069c     dbcore.obj
 0002:000016b0       ??_C@_0BA@CDEP@?6m_nEditMode?5?$DN?5?$AA@ 5f7306b0     dbcore.obj
 0002:000016c0       ??_C@_0BA@GJB@?6m_bLockMode?5?$DN?5?$AA@ 5f7306c0     dbcore.obj
 0002:000016d0       ??_C@_0P@NFAJ@?6m_bDeleted?5?$DN?5?$AA@ 5f7306d0     dbcore.obj
 0002:000016e0       ??_C@_0L@IPIJ@?6m_bBOF?5?$DN?5?$AA@ 5f7306e0     dbcore.obj
 0002:000016ec       ??_C@_0L@GHOJ@?6m_bEOF?5?$DN?5?$AA@ 5f7306ec     dbcore.obj
 0002:000016f8       ??_C@_0O@DPF@?6m_nParams?5?$DN?5?$AA@ 5f7306f8     dbcore.obj
 0002:00001708       ??_C@_0BD@GPPK@?6m_nFieldsBound?5?$DN?5?$AA@ 5f730708     dbcore.obj
 0002:0000171c       ??_C@_0O@ECP@?6m_nFields?5?$DN?5?$AA@ 5f73071c     dbcore.obj
 0002:0000172c       ??_C@_0BC@IMFD@?6m_bAppendable?5?$DN?5?$AA@ 5f73072c     dbcore.obj
 0002:00001740       ??_C@_0BC@CBKM@?6m_bScrollable?5?$DN?5?$AA@ 5f730740     dbcore.obj
 0002:00001754       ??_C@_0M@CNKH@?6m_lOpen?5?$DN?5?$AA@ 5f730754     dbcore.obj
 0002:00001760       ??_C@_0BD@DHNL@?6m_bRecordsetDb?5?$DN?5?$AA@ 5f730760     dbcore.obj
 0002:00001774       ??_C@_0M@JKLH@?6m_hstmt?5?$DN?5?$AA@ 5f730774     dbcore.obj
 0002:00001780       ??_C@_0N@MDHJ@?6m_strSQL?5?$DN?5?$AA@ 5f730780     dbcore.obj
 0002:00001790       ??_C@_0P@KPIA@m_nOpenType?5?$DN?5?$AA@ 5f730790     dbcore.obj
 0002:000017a0       ??_C@_0DL@JHHP@Error?3?5SetSynchronousMode?5is?5obs@ 5f7307a0     dbcore.obj
 0002:000017dc       ??_C@_0CH@KFAI@E?3?28168?2vc98?2mfc?2mfc?2include?2afx@ 5f7307dc     dbcore.obj
 0002:00001808       ??_7_AFX_DB_STATE@@6B@     5f730808     dbcore.obj
 0002:00001810       ??_7CNoTrackObject@@6B@    5f730810     dbcore.obj
 0002:00001814       ??_C@_0CP@MBLH@Error?3?5field?5address?5?$CIcolumn?5?$CFu?$CJ@ 5f730814     dbrfx.obj
 0002:00001844       ??_C@_03FGJK@?5?$DN?5?$AA@ 5f730844     dbrfx.obj
 0002:00001848       ??_C@_0DA@EEGJ@Error?3?5buffer?5?$CIcolumn?5?$CFu?$CJ?5addres@ 5f730848     dbrfx.obj
 0002:00001878       ??_C@_0CO@CHAB@Warning?3?5string?5converted?5from?5S@ 5f730878     dbrfx.obj
 0002:000018a8       ??_C@_0DI@MFHF@Error?3?5CString?5buffer?5?$CIcolumn?5?$CFu@ 5f7308a8     dbrfx.obj
 0002:000018e0       ??_C@_0CP@KHPL@Warning?3?5CString?5converted?5from?5@ 5f7308e0     dbrfx.obj
 0002:00001910       ??_C@_0CL@KDPB@Warning?3?5int?5converted?5from?5SQL?5@ 5f730910     dbrfx.obj
 0002:0000193c       ??_C@_0CM@CDOP@Warning?3?5long?5converted?5from?5SQL@ 5f73093c     dbrfx.obj
 0002:00001968       ??_C@_0CM@DDAL@Warning?3?5BYTE?5converted?5from?5SQL@ 5f730968     dbrfx.obj
 0002:00001994       ??_C@_0CM@HOOD@Warning?3?5BOOL?5converted?5from?5SQL@ 5f730994     dbrfx.obj
 0002:000019c0       ??_C@_01PKAG@?3?$AA@       5f7309c0     dbrfx.obj
 0002:000019c4       ??_C@_0DC@MJOF@Warning?3?5CByteArray?5converted?5fr@ 5f7309c4     dbrfx.obj
 0002:000019f8       ??_C@_0CB@NGEA@Warning?3?5ignoring?5milliseconds?4?6@ 5f7309f8     dbrfx.obj
 0002:00001a1c       ??_C@_0DJ@MLFM@Warning?3?5date?5value?5out?5of?5range@ 5f730a1c     dbrfx.obj
 0002:00001a58       ??_C@_0CN@PMCD@Warning?3?5CTime?5converted?5from?5SQ@ 5f730a58     dbrfx.obj
 0002:00001a88       ??_C@_0N@OGBI@?4fraction?5?$DN?5?$AA@ 5f730a88     dbrfx.obj
 0002:00001a98       ??_C@_0L@BFHB@?4second?5?$DN?5?$AA@ 5f730a98     dbrfx.obj
 0002:00001aa4       ??_C@_0L@JFIG@?4minute?5?$DN?5?$AA@ 5f730aa4     dbrfx.obj
 0002:00001ab0       ??_C@_08PGJP@?4hour?5?$DN?5?$AA@ 5f730ab0     dbrfx.obj
 0002:00001abc       ??_C@_07JEIM@?4day?5?$DN?5?$AA@ 5f730abc     dbrfx.obj
 0002:00001ac4       ??_C@_09DKMF@?4month?5?$DN?5?$AA@ 5f730ac4     dbrfx.obj
 0002:00001ad0       ??_C@_08DFNB@?4year?5?$DN?5?$AA@ 5f730ad0     dbrfx.obj
 0002:00001adc       ??_C@_0DI@PGDH@Warning?3?5TIMESTAMP_STRUCT?5conver@ 5f730adc     dbrfx.obj
 0002:00001b14       ??_C@_0DE@HMIF@Warning?3?5COleDateTime?5converted?5@ 5f730b14     dbrfx.obj
 0002:00001b48       ??_C@_0M@JABG@State?301004?$AA@ 5f730b48     dbrfx.obj
 0002:00001b58       ?classCRecordView@CRecordView@@2UCRuntimeClass@@B 5f730b58     dbview.obj
 0002:00001b70       ??_C@_0M@EAFL@CRecordView?$AA@ 5f730b70     dbview.obj
 0002:00001b80       ?messageMap@CRecordView@@1UAFX_MSGMAP@@B 5f730b80     dbview.obj
 0002:00001b88       ?_messageEntries@CRecordView@@0QBUAFX_MSGMAP_ENTRY@@B 5f730b88     dbview.obj
 0002:00001c64       ??_7CRecordView@@6B@       5f730c64     dbview.obj
 0002:00001d7c       ??_C@_0CE@BOGL@Warning?3?5no?5listbox?5item?5selecte@ 5f730d7c     dbview.obj
 0002:00001da0       ??_C@_0CF@IFBC@Warning?3?5no?5combobox?5item?5select@ 5f730da0     dbview.obj
 0002:00001dc8       ??_C@_0DI@IJGE@Warning?3?5dialog?5data?5checkbox?5va@ 5f730dc8     dbview.obj
 0002:00001e00       ??_C@_0DK@CIE@Warning?3?5field?5NULL?5and?5checkbox@ 5f730e00     dbview.obj
 0002:00001e3c       ??_C@_0EA@FKPN@Warning?3?5checkbox?5value?5indeterm@ 5f730e3c     dbview.obj
 0002:00001e7c       ??_C@_0BE@JDG@?6m_bOnLastRecord?5?$DN?5?$AA@ 5f730e7c     dbview.obj
 0002:00001e90       ??_C@_0BE@GCEL@m_bOnFirstRecord?5?$DN?5?$AA@ 5f730e90     dbview.obj
 0002:00001eb8       ??_C@_0CN@LIHI@Warning?3?5float?5converted?5from?5SQ@ 5f730eb8     dbflt.obj
 0002:00001ee8       ??_C@_0CO@JONC@Warning?3?5double?5converted?5from?5S@ 5f730ee8     dbflt.obj
 0002:00001f18       ?classCLongBinary@CLongBinary@@2UCRuntimeClass@@B 5f730f18     dblong.obj
 0002:00001f30       ??_C@_0M@DJA@CLongBinary?$AA@ 5f730f30     dblong.obj
 0002:00001f40       ??_7CLongBinary@@6B@       5f730f40     dblong.obj
 0002:00001f54       ??_C@_0BD@HHCG@?6m_dwDataLength?5?$DN?5?$AA@ 5f730f54     dblong.obj
 0002:00001f68       ??_C@_0L@DGJD@m_hData?5?$DN?5?$AA@ 5f730f68     dblong.obj
 0002:00001f78       ??_7CDBVariant@@6B@        5f730f78     dbvar.obj
 0002:00001f80       ?classCDaoRecordset@CDaoRecordset@@2UCRuntimeClass@@B 5f730f80     daocore.obj
 0002:00001f98       ??_C@_0O@JOIL@CDaoRecordset?$AA@ 5f730f98     daocore.obj
 0002:00001fa8       ?classCDaoQueryDef@CDaoQueryDef@@2UCRuntimeClass@@B 5f730fa8     daocore.obj
 0002:00001fc0       ??_C@_0N@NGH@CDaoQueryDef?$AA@ 5f730fc0     daocore.obj
 0002:00001fd0       ?classCDaoTableDef@CDaoTableDef@@2UCRuntimeClass@@B 5f730fd0     daocore.obj
 0002:00001fe8       ??_C@_0N@PHMG@CDaoTableDef?$AA@ 5f730fe8     daocore.obj
 0002:00001ff8       ?classCDaoDatabase@CDaoDatabase@@2UCRuntimeClass@@B 5f730ff8     daocore.obj
 0002:00002010       ??_C@_0N@DDLP@CDaoDatabase?$AA@ 5f731010     daocore.obj
 0002:00002020       ?classCDaoWorkspace@CDaoWorkspace@@2UCRuntimeClass@@B 5f731020     daocore.obj
 0002:00002038       ??_C@_0O@IEJG@CDaoWorkspace?$AA@ 5f731038     daocore.obj
 0002:00002048       ?classCDaoException@CDaoException@@2UCRuntimeClass@@B 5f731048     daocore.obj
 0002:00002060       ??_C@_0O@OIMH@CDaoException?$AA@ 5f731060     daocore.obj
 0002:00002070       ?_afxTable2@@3QBDB         5f731070     daocore.obj
 0002:00002078       ?_afxTransform2@@3QBDB     5f731078     daocore.obj
 0002:00002084       ?_afxOrderBy2@@3QBDB       5f731084     daocore.obj
 0002:00002090       ?_afxWhere2@@3QBDB         5f731090     daocore.obj
 0002:00002098       ?_afxFrom2@@3QBDB          5f731098     daocore.obj
 0002:000020a0       ?_afxSelect2@@3QBDB        5f7310a0     daocore.obj
 0002:000020a8       ?_afxParameters2@@3QBDB    5f7310a8     daocore.obj
 0002:000020b8       ??_7_AFX_DAO_STATE@@6B@    5f7310b8     daocore.obj
 0002:000020bc       ??_C@_0O@IIOC@?6?7scode?5?$DN?5?$CFX?6?$AA@ 5f7310bc     daocore.obj
 0002:000020cc       ??_C@_0BJ@PFJI@?6?7In?5file?5?$CFhs?5on?5line?5?$CFd?$AA@ 5f7310cc     daocore.obj
 0002:000020e8       ??_C@_05HNHB@?6?7?$CFhs?$AA@ 5f7310e8     daocore.obj
 0002:000020f0       ??_C@_0BC@DBPE@?6DAO?5Call?5Failed?4?$AA@ 5f7310f0     daocore.obj
 0002:00002104       ??_C@_0M@KDOI@scode?5?$DN?5?$CFX?6?$AA@ 5f731104     daocore.obj
 0002:00002110       ??_C@_0BJ@JBPF@?6In?5file?5?$CFhs?5on?5line?5?$CFd?6?$AA@ 5f731110     daocore.obj
 0002:0000212c       ??_C@_04FDOH@?6?$CFhs?$AA@ 5f73112c     daocore.obj
 0002:00002134       ??_C@_0BE@GAIL@?6DAO?5Call?5Failed?4?6?7?$AA@ 5f731134     daocore.obj
 0002:00002148       ??_C@_0BD@JMBE@?6m_lHelpContext?5?$DN?5?$AA@ 5f731148     daocore.obj
 0002:0000215c       ??_C@_0BC@FOHM@?6m_strHelpFile?5?$DN?5?$AA@ 5f73115c     daocore.obj
 0002:00002170       ??_C@_0BF@JHNL@?6m_strDescription?5?$DN?5?$AA@ 5f731170     daocore.obj
 0002:00002188       ??_C@_0BA@HMPD@?6m_strSource?5?$DN?5?$AA@ 5f731188     daocore.obj
 0002:00002198       ??_C@_0BB@CCFD@?6m_lErrorCode?5?$DN?5?$AA@ 5f731198     daocore.obj
 0002:000021ac       ??_C@_0BE@OGG@a?5CDaoErrorInfo?5at?5?$AA@ 5f7311ac     daocore.obj
 0002:000021c0       ??_C@_0BJ@HLFP@?6b?5?$DN?5m_bIsolateODBCTrans?$AA@ 5f7311c0     daocore.obj
 0002:000021dc       ??_C@_0BC@HDK@?6m_strUserName?5?$DN?5?$AA@ 5f7311dc     daocore.obj
 0002:000021f0       ??_C@_0O@FEGP@?6m_strName?5?$DN?5?$AA@ 5f7311f0     daocore.obj
 0002:00002200       ??_C@_0BI@EJIL@a?5CDaoWorkspaceInfo?5at?5?$AA@ 5f731200     daocore.obj
 0002:00002218       ??_C@_0BE@JLEN@?6m_nQueryTimeout?5?$DN?5?$AA@ 5f731218     daocore.obj
 0002:0000222c       ??_C@_0BG@ILBM@?6m_lCollatingOrder?5?$DN?5?$AA@ 5f73122c     daocore.obj
 0002:00002244       ??_C@_0BB@LEGM@?6m_strVersion?5?$DN?5?$AA@ 5f731244     daocore.obj
 0002:00002258       ??_C@_0BH@FIEC@a?5CDaoDatabaseInfo?5at?5?$AA@ 5f731258     daocore.obj
 0002:00002270       ??_C@_0BD@FJAC@?6m_lRecordCount?5?$DN?5?$AA@ 5f731270     daocore.obj
 0002:00002284       ??_C@_0BI@JMNH@?6m_strValidationText?5?$DN?5?$AA@ 5f731284     daocore.obj
 0002:0000229c       ??_C@_0BI@NDBL@?6m_strValidationRule?5?$DN?5?$AA@ 5f73129c     daocore.obj
 0002:000022b4       ??_C@_0BG@FOBO@?6m_strSrcTableName?5?$DN?5?$AA@ 5f7312b4     daocore.obj
 0002:000022cc       ??_C@_0BG@PCL@?6m_dateLastUpdated?5?$DN?5?$AA@ 5f7312cc     daocore.obj
 0002:000022e4       ??_C@_0BG@FOFB@?6m_dateDateCreated?5?$DN?5?$AA@ 5f7312e4     daocore.obj
 0002:000022fc       ??_C@_0BC@KBNC@?6m_lAttributes?5?$DN?5?$AA@ 5f7312fc     daocore.obj
 0002:00002310       ??_C@_0BH@JFIA@a?5CDaoTableDefInfo?5at?5?$AA@ 5f731310     daocore.obj
 0002:00002328       ??_C@_0BG@MHMB@?6m_strDefaultValue?5?$DN?5?$AA@ 5f731328     daocore.obj
 0002:00002340       ??_C@_0BF@HCFN@?6m_strSourceTable?5?$DN?5?$AA@ 5f731340     daocore.obj
 0002:00002358       ??_C@_0BF@NJHG@?6m_strSourceField?5?$DN?5?$AA@ 5f731358     daocore.obj
 0002:00002370       ??_C@_0BF@KILJ@?6m_strForeignName?5?$DN?5?$AA@ 5f731370     daocore.obj
 0002:00002388       ??_C@_0BH@BCFG@?6m_bAllowZeroLength?5?$DN?5?$AA@ 5f731388     daocore.obj
 0002:000023a0       ??_C@_0BA@OOHL@?6m_bRequired?5?$DN?5?$AA@ 5f7313a0     daocore.obj
 0002:000023b0       ??_C@_0BH@IMAL@?6m_nOrdinalPosition?5?$DN?5?$AA@ 5f7313b0     daocore.obj
 0002:000023c8       ??_C@_0M@EOEG@?6m_lSize?5?$DN?5?$AA@ 5f7313c8     daocore.obj
 0002:000023d4       ??_C@_0M@MJB@?6m_nType?5?$DN?5?$AA@ 5f7313d4     daocore.obj
 0002:000023e0       ??_C@_0BE@PODE@a?5CDaoFieldInfo?5at?5?$AA@ 5f7313e0     daocore.obj
 0002:000023f4       ??_C@_0BC@ILAA@?6m_bDescending?5?$DN?5?$AA@ 5f7313f4     daocore.obj
 0002:00002408       ??_C@_0BK@KCFC@?5a?5CDaoIndexFieldInfo?5at?5?$AA@ 5f731408     daocore.obj
 0002:00002428       ??_7CDaoIndexInfo@@6B@     5f731428     daocore.obj
 0002:00002430       ??_C@_0BF@LIJD@?6m_lDistinctCount?5?$DN?5?$AA@ 5f731430     daocore.obj
 0002:00002448       ??_C@_0P@DLHL@?6m_bForeign?5?$DN?5?$AA@ 5f731448     daocore.obj
 0002:00002458       ??_C@_0BD@MAED@?6m_bIgnoreNulls?5?$DN?5?$AA@ 5f731458     daocore.obj
 0002:0000246c       ??_C@_0BB@FFL@?6m_bClustered?5?$DN?5?$AA@ 5f73146c     daocore.obj
 0002:00002480       ??_C@_0O@NMC@?6m_bUnique?5?$DN?5?$AA@ 5f731480     daocore.obj
 0002:00002490       ??_C@_0P@FFEB@?6m_bPrimary?5?$DN?5?$AA@ 5f731490     daocore.obj
 0002:000024a0       ??_C@_0BE@OGHD@a?5CDaoIndexInfo?5at?5?$AA@ 5f7314a0     daocore.obj
 0002:000024b4       ??_C@_0BN@BEAM@?5a?5CDaoRelationFieldInfo?5at?5?$AA@ 5f7314b4     daocore.obj
 0002:000024d8       ??_7CDaoRelationInfo@@6B@  5f7314d8     daocore.obj
 0002:000024e0       ??_C@_0BG@NBH@?6m_strForeignTable?5?$DN?5?$AA@ 5f7314e0     daocore.obj
 0002:000024f8       ??_C@_0P@CHOL@?6m_strTable?5?$DN?5?$AA@ 5f7314f8     daocore.obj
 0002:00002508       ??_C@_0BH@ICPE@a?5CDaoRelationInfo?5at?5?$AA@ 5f731508     daocore.obj
 0002:00002520       ??_C@_0BD@BKGA@?6m_nODBCTimeout?5?$DN?5?$AA@ 5f731520     daocore.obj
 0002:00002534       ??_C@_0BG@JDEE@?6m_bReturnsRecords?5?$DN?5?$AA@ 5f731534     daocore.obj
 0002:0000254c       ??_C@_0BC@DDHJ@?6m_dateCreated?5?$DN?5?$AA@ 5f73154c     daocore.obj
 0002:00002560       ??_C@_0BH@OPB@a?5CDaoQueryDefInfo?5at?5?$AA@ 5f731560     daocore.obj
 0002:00002578       ??_C@_0P@MIHC@?6m_varValue?5?$DN?5?$AA@ 5f731578     daocore.obj
 0002:00002588       ??_C@_0BI@NAFD@a?5CDaoParameterInfo?5at?5?$AA@ 5f731588     daocore.obj
 0002:000025a4       ??_7CDaoException@@6B@     5f7315a4     daocore.obj
 0002:000025c0       ??_C@_0CC@NFIM@m_pDAOErrors?9?$DOget_Count?$CI?$CGnErrors@ 5f7315c0     daocore.obj
 0002:000025e4       ??_C@_0EB@MBDI@m_pDAOErrors?9?$DOget_Item?$CI?5COleVari@ 5f7315e4     daocore.obj
 0002:00002628       ??_C@_0DG@CEPE@pDaoState?9?$DOm_pDAODBEngine?9?$DOget_E@ 5f731628     daocore.obj
 0002:00002660       ??_C@_0DN@LLAK@m_pDAOError?9?$DOget_HelpContext?$CI?5?$CGm@ 5f731660     daocore.obj
 0002:000026a0       ??_C@_0CJ@LALL@m_pDAOError?9?$DOget_HelpFile?$CI?$CGV_BST@ 5f7316a0     daocore.obj
 0002:000026cc       ??_C@_0CM@BAFD@m_pDAOError?9?$DOget_Description?$CI?$CGV_@ 5f7316cc     daocore.obj
 0002:000026f8       ??_C@_0CH@NNNO@m_pDAOError?9?$DOget_Source?$CI?$CGV_BSTR?$CI@ 5f7316f8     daocore.obj
 0002:00002720       ??_C@_0DG@GHAH@m_pDAOError?9?$DOget_Number?$CI?5?$CGm_pErr@ 5f731720     daocore.obj
 0002:0000275c       ??_7CDaoErrorInfo@@6B@     5f73175c     daocore.obj
 0002:00002760       ??_C@_0BC@NJHN@Description?5?$DN?5?$CFs?6?$AA@ 5f731760     daocore.obj
 0002:00002774       ??_C@_0N@GFFD@Source?5?$DN?5?$CFs?6?$AA@ 5f731774     daocore.obj
 0002:00002784       ??_C@_0BC@CBKK@?6Error?5Code?5?$DN?5?$CFd?6?$AA@ 5f731784     daocore.obj
 0002:0000279c       ??_7CDaoWorkspace@@6B@     5f73179c     daocore.obj
 0002:000027c4       ??_C@_0IA@IMA@pDaoState?9?$DOm_pDAODBEngine?9?$DO_30_C@ 5f7317c4     daocore.obj
 0002:00002844       ??_C@_0CI@OLEJ@pDAOWorkspaces?9?$DOAppend?$CIm_pDAOWor@ 5f731844     daocore.obj
 0002:0000286c       ??_C@_0DL@KMOM@pDaoState?9?$DOm_pDAODBEngine?9?$DOget_W@ 5f73186c     daocore.obj
 0002:000028a8       ??_C@_0DC@BHKN@m_pDAOWorkspaces?9?$DOget_Item?$CIvar?0?5@ 5f7318a8     daocore.obj
 0002:000028dc       ??_C@_0DO@NCLP@pDaoState?9?$DOm_pDAODBEngine?9?$DOget_W@ 5f7318dc     daocore.obj
 0002:0000291c       ??_C@_0BJ@BAIF@m_pDAOWorkspace?9?$DOClose?$CI?$CJ?$AA@ 5f73191c     daocore.obj
 0002:00002938       ??_C@_0DG@EKI@pDaoState?9?$DOm_pDAODBEngine?9?$DOget_V@ 5f731938     daocore.obj
 0002:00002970       ??_C@_0DG@POMJ@pDaoState?9?$DOm_pDAODBEngine?9?$DOget_I@ 5f731970     daocore.obj
 0002:000029a8       ??_C@_0DF@FAOI@pDaoState?9?$DOm_pDAODBEngine?9?$DOput_I@ 5f7319a8     daocore.obj
 0002:000029e0       ??_C@_0DJ@GIII@pDaoState?9?$DOm_pDAODBEngine?9?$DOput_D@ 5f7319e0     daocore.obj
 0002:00002a1c       ??_C@_0DO@ONCK@pDaoState?9?$DOm_pDAODBEngine?9?$DOput_D@ 5f731a1c     daocore.obj
 0002:00002a5c       ??_C@_0DH@FIK@pDaoState?9?$DOm_pDAODBEngine?9?$DOget_L@ 5f731a5c     daocore.obj
 0002:00002a94       ??_C@_0DG@FCKN@pDaoState?9?$DOm_pDAODBEngine?9?$DOput_L@ 5f731a94     daocore.obj
 0002:00002acc       ??_C@_0CJ@PIID@m_pDAOWorkspace?9?$DOget_Name?$CI?$CGV_BST@ 5f731acc     daocore.obj
 0002:00002af8       ??_C@_0CN@LNMJ@m_pDAOWorkspace?9?$DOget_UserName?$CI?$CGV@ 5f731af8     daocore.obj
 0002:00002b28       ??_C@_0GC@MAIK@m_pDAOWorkspace?9?$DOput_IsolateODBC@ 5f731b28     daocore.obj
 0002:00002b8c       ??_C@_0DK@BNMM@m_pDAOWorkspace?9?$DOget_IsolateODBC@ 5f731b8c     daocore.obj
 0002:00002bc8       ??_C@_0PC@HCAP@pDaoState?9?$DOm_pDAODBEngine?9?$DOCompa@ 5f731bc8     daocore.obj
 0002:00002cbc       ??_C@_0DN@CKIJ@pDaoState?9?$DOm_pDAODBEngine?9?$DORepai@ 5f731cbc     daocore.obj
 0002:00002cfc       ??_C@_0DN@BCJE@pDaoState?9?$DOm_pDAODBEngine?9?$DOIdle?$CI@ 5f731cfc     daocore.obj
 0002:00002d3c       ??_C@_0CG@MKCN@m_pDAOWorkspaces?9?$DOget_Count?$CI?$CGnFi@ 5f731d3c     daocore.obj
 0002:00002d64       ??_C@_0EH@MIPG@m_pDAOWorkspaces?9?$DOget_Item?$CI?5COle@ 5f731d64     daocore.obj
 0002:00002dac       ??_C@_0EN@CDCO@m_pDAOWorkspaces?9?$DOget_Item?$CI?5COle@ 5f731dac     daocore.obj
 0002:00002dfc       ??_C@_0CF@NKKO@m_pDAODatabases?9?$DOget_Count?$CI?$CGnFie@ 5f731dfc     daocore.obj
 0002:00002e24       ??_C@_0EF@MAIH@m_pDAODatabases?9?$DOget_Item?$CI?5COleV@ 5f731e24     daocore.obj
 0002:00002e6c       ??_C@_0EL@BNEE@m_pDAODatabases?9?$DOget_Item?$CI?5COleV@ 5f731e6c     daocore.obj
 0002:00002eb8       ??_C@_0BO@IBKO@m_pDAOWorkspace?9?$DOBeginTrans?$CI?$CJ?$AA@ 5f731eb8     daocore.obj
 0002:00002ed8       ??_C@_0BO@ONLB@?$CIm_pDAOWorkspace?9?$DO?$CKpMethod?$CJ?$CI?$CJ?$AA@ 5f731ed8     daocore.obj
 0002:00002ef8       ??_C@_0CA@PBAE@m_pDAOWorkspace?9?$DOCommitTrans?$CI0?$CJ?$AA@ 5f731ef8     daocore.obj
 0002:00002f18       ??_C@_0BM@BBEN@m_pDAOWorkspace?9?$DORollback?$CI?$CJ?$AA@ 5f731f18     daocore.obj
 0002:00002f34       ??_C@_0CM@PHDL@pDAOWorkspace?9?$DOget_IsolateODBCTr@ 5f731f34     daocore.obj
 0002:00002f60       ??_C@_0CL@LFDC@pDAOWorkspace?9?$DOget_UserName?$CI?$CGV_B@ 5f731f60     daocore.obj
 0002:00002f8c       ??_C@_0CH@NIA@pDAOWorkspace?9?$DOget_Name?$CI?$CGV_BSTR?$CI@ 5f731f8c     daocore.obj
 0002:00002fb4       ??_C@_0DB@FMO@m_pDAOWorkspace?9?$DOget_Databases?$CI?$CG@ 5f731fb4     daocore.obj
 0002:00002fe8       ??_C@_0CK@GLDA@pDAODatabase?9?$DOget_Connect?$CI?5?$CGV_BS@ 5f731fe8     daocore.obj
 0002:00003014       ??_C@_0DJ@LMDF@pDAODatabase?9?$DOget_QueryTimeout?$CI?5@ 5f732014     daocore.obj
 0002:00003050       ??_C@_0DN@CAFO@pDAODatabase?9?$DOget_CollatingOrder@ 5f732050     daocore.obj
 0002:00003090       ??_C@_0CK@LGL@pDAODatabase?9?$DOget_Version?$CI?5?$CGV_BS@ 5f732090     daocore.obj
 0002:000030bc       ??_C@_0CH@GLGK@pDAODatabase?9?$DOget_Transactions?$CI?$CG@ 5f7320bc     daocore.obj
 0002:000030e4       ??_C@_0CE@GDMB@pDAODatabase?9?$DOget_Updatable?$CI?$CGnBo@ 5f7320e4     daocore.obj
 0002:00003108       ??_C@_0CG@GEI@pDAODatabase?9?$DOget_Name?$CI?$CGV_BSTR?$CI?$CG@ 5f732108     daocore.obj
 0002:00003130       ??_C@_0O@KPOJ@?6m_nStatus?5?$DN?5?$AA@ 5f732130     daocore.obj
 0002:00003140       ??_C@_0L@OLPD@?6m_bNew?5?$DN?5?$AA@ 5f732140     daocore.obj
 0002:0000314c       ??_C@_0L@FNFF@m_bOpen?5?$DN?5?$AA@ 5f73214c     daocore.obj
 0002:0000315c       ??_7CDaoDatabase@@6B@      5f73215c     daocore.obj
 0002:00003180       ??_C@_0IC@FKK@m_pWorkspace?9?$DOm_pDAOWorkspace?9?$DOC@ 5f732180     daocore.obj
 0002:00003204       ??_C@_0LP@CIKN@m_pWorkspace?9?$DOm_pDAOWorkspace?9?$DOO@ 5f732204     daocore.obj
 0002:000032c4       ??_C@_0BI@NBCE@m_pDAODatabase?9?$DOClose?$CI?$CJ?$AA@ 5f7322c4     daocore.obj
 0002:000032dc       ??_C@_0CL@ELFI@m_pDAODatabase?9?$DOget_Updatable?$CI?$CGn@ 5f7322dc     daocore.obj
 0002:00003308       ??_C@_0DB@POJO@m_pDAODatabase?9?$DOget_Transactions@ 5f732308     daocore.obj
 0002:0000333c       ??_C@_0CI@FCO@m_pDAODatabase?9?$DOget_Name?$CI?$CGV_BSTR@ 5f73233c     daocore.obj
 0002:00003364       ??_C@_0CL@OIPD@m_pDAODatabase?9?$DOget_Connect?$CI?$CGV_B@ 5f732364     daocore.obj
 0002:00003390       ??_C@_0CL@LDKH@m_pDAODatabase?9?$DOget_Version?$CI?$CGV_B@ 5f732390     daocore.obj
 0002:000033bc       ??_C@_0DB@NKM@m_pDAODatabase?9?$DOget_QueryTimeout@ 5f7323bc     daocore.obj
 0002:000033f0       ??_C@_0CL@CMOO@m_pDAODatabase?9?$DOput_QueryTimeout@ 5f7323f0     daocore.obj
 0002:0000341c       ??_C@_0DH@EED@m_pDAODatabase?9?$DOget_RecordsAffec@ 5f73241c     daocore.obj
 0002:00003454       ??_C@_0CG@DPNF@m_pDAOTableDefs?9?$DODelete?$CIV_BSTR?$CI?$CG@ 5f732454     daocore.obj
 0002:0000347c       ??_C@_0CG@PEFD@m_pDAOQueryDefs?9?$DODelete?$CIV_BSTR?$CI?$CG@ 5f73247c     daocore.obj
 0002:000034a8       ??_7CDaoRelationFieldInfo@@6B@ 5f7324a8     daocore.obj
 0002:000034ac       ??_C@_0CG@KOHE@m_pDAORelations?9?$DOAppend?$CIpDAORela@ 5f7324ac     daocore.obj
 0002:000034d4       ??_C@_0BO@PKCL@pDAOFields?9?$DOAppend?$CIpDAOField?$CJ?$AA@ 5f7324d4     daocore.obj
 0002:000034f4       ??_C@_0CJ@GPBE@pDAOField?9?$DOput_ForeignName?$CIV_BST@ 5f7324f4     daocore.obj
 0002:00003520       ??_C@_0JB@FHMF@pDAORelation?9?$DOCreateField?$CI?5COleV@ 5f732520     daocore.obj
 0002:000035b4       ??_C@_0CG@INKG@pDAORelation?9?$DOget_Fields?$CI?$CGpDAOFi@ 5f7325b4     daocore.obj
 0002:000035dc       ??_C@_0NK@LJKP@m_pDAODatabase?9?$DOCreateRelation?$CI?5@ 5f7325dc     daocore.obj
 0002:000036b8       ??_C@_0CG@BJFH@m_pDAORelations?9?$DODelete?$CIV_BSTR?$CI?$CG@ 5f7326b8     daocore.obj
 0002:000036e0       ??_C@_0EE@KEMK@m_pDAODatabase?9?$DOExecute?$CI?5V_BSTR?$CI@ 5f7326e0     daocore.obj
 0002:00003724       ??_C@_0CF@JLMN@m_pDAOTableDefs?9?$DOget_Count?$CI?$CGnTab@ 5f732724     daocore.obj
 0002:0000374c       ??_C@_0EF@FBLA@m_pDAOTableDefs?9?$DOget_Item?$CI?5COleV@ 5f73274c     daocore.obj
 0002:00003794       ??_C@_0EL@KPGC@m_pDAOTableDefs?9?$DOget_Item?$CI?5COleV@ 5f732794     daocore.obj
 0002:000037e0       ??_C@_0CI@LDJE@m_pDAORelations?9?$DOget_Count?$CI?$CGnRel@ 5f7327e0     daocore.obj
 0002:00003808       ??_C@_0EF@IIIA@m_pDAORelations?9?$DOget_Item?$CI?5COleV@ 5f732808     daocore.obj
 0002:00003850       ??_C@_0EL@IHJB@m_pDAORelations?9?$DOget_Item?$CI?5COleV@ 5f732850     daocore.obj
 0002:0000389c       ??_C@_0CI@MEAB@m_pDAOQueryDefs?9?$DOget_Count?$CI?$CGnQue@ 5f73289c     daocore.obj
 0002:000038c4       ??_C@_0EF@NBOE@m_pDAOQueryDefs?9?$DOget_Item?$CI?5COleV@ 5f7328c4     daocore.obj
 0002:0000390c       ??_C@_0EL@IINM@m_pDAOQueryDefs?9?$DOget_Item?$CI?5COleV@ 5f73290c     daocore.obj
 0002:00003958       ??_C@_0DA@GLPP@m_pDAODatabase?9?$DOget_TableDefs?$CI?$CGm@ 5f732958     daocore.obj
 0002:00003988       ??_C@_0DN@PBMP@pDAOTableDef?9?$DOget_RecordCount?$CI?5?$CG@ 5f732988     daocore.obj
 0002:000039c8       ??_C@_0DB@KOFA@pDAOTableDef?9?$DOget_ValidationText@ 5f7329c8     daocore.obj
 0002:000039fc       ??_C@_0DB@HJKE@pDAOTableDef?9?$DOget_ValidationRule@ 5f7329fc     daocore.obj
 0002:00003a30       ??_C@_0CK@LEHN@pDAOTableDef?9?$DOget_Connect?$CI?5?$CGV_BS@ 5f732a30     daocore.obj
 0002:00003a5c       ??_C@_0DC@BFFJ@pDAOTableDef?9?$DOget_SourceTableNam@ 5f732a5c     daocore.obj
 0002:00003a90       ??_C@_0CE@FNDA@pDAOTableDef?9?$DOget_LastUpdated?$CI?$CGv@ 5f732a90     daocore.obj
 0002:00003ab4       ??_C@_0CE@NEPA@pDAOTableDef?9?$DOget_DateCreated?$CI?$CGv@ 5f732ab4     daocore.obj
 0002:00003ad8       ??_C@_0DL@DLNJ@pDAOTableDef?9?$DOget_Attributes?$CI?5?$CGt@ 5f732ad8     daocore.obj
 0002:00003b14       ??_C@_0CE@GAKL@pDAOTableDef?9?$DOget_Updatable?$CI?$CGnBo@ 5f732b14     daocore.obj
 0002:00003b38       ??_C@_0CG@GGLM@pDAOTableDef?9?$DOget_Name?$CI?$CGV_BSTR?$CI?$CG@ 5f732b38     daocore.obj
 0002:00003b60       ??_C@_0DA@JLIC@m_pDAODatabase?9?$DOget_Relations?$CI?$CGm@ 5f732b60     daocore.obj
 0002:00003b90       ??_C@_0CK@LAFA@pDAOField?9?$DOget_ForeignName?$CI?$CGV_BS@ 5f732b90     daocore.obj
 0002:00003bbc       ??_C@_0CD@BJOA@pDAOField?9?$DOget_Name?$CI?$CGV_BSTR?$CI?$CGvar@ 5f732bbc     daocore.obj
 0002:00003be0       ??_C@_0DN@MJFF@pDAOFields?9?$DOget_Item?$CI?5COleVarian@ 5f732be0     daocore.obj
 0002:00003c20       ??_C@_0BP@FFPK@pDAOFields?9?$DOget_Count?$CI?$CGnCount?$CJ?$AA@ 5f732c20     daocore.obj
 0002:00003c40       ??_C@_0DG@DMNE@pDAORelation?9?$DOget_Attributes?$CI?5?$CGr@ 5f732c40     daocore.obj
 0002:00003c78       ??_C@_0CP@PIMH@pDAORelation?9?$DOget_ForeignTable?$CI?5@ 5f732c78     daocore.obj
 0002:00003ca8       ??_C@_0CH@LDAN@pDAORelation?9?$DOget_Table?$CI?$CGV_BSTR?$CI@ 5f732ca8     daocore.obj
 0002:00003cd0       ??_C@_0CG@NDBG@pDAORelation?9?$DOget_Name?$CI?$CGV_BSTR?$CI?$CG@ 5f732cd0     daocore.obj
 0002:00003cf8       ??_C@_0DA@BPAN@m_pDAODatabase?9?$DOget_QueryDefs?$CI?$CGm@ 5f732cf8     daocore.obj
 0002:00003d28       ??_C@_0DE@DPOF@pDAOQueryDef?9?$DOget_Connect?$CI?$CGV_BST@ 5f732d28     daocore.obj
 0002:00003d5c       ??_C@_0CF@HFEL@pDAOQueryDef?9?$DOget_SQL?$CI?$CGV_BSTR?$CI?$CGv@ 5f732d5c     daocore.obj
 0002:00003d84       ??_C@_0CJ@KFGF@pDAOQueryDef?9?$DOget_ReturnsRecords@ 5f732d84     daocore.obj
 0002:00003db0       ??_C@_0CE@JGLG@pDAOQueryDef?9?$DOget_LastUpdated?$CI?$CGv@ 5f732db0     daocore.obj
 0002:00003dd4       ??_C@_0CE@BPHG@pDAOQueryDef?9?$DOget_DateCreated?$CI?$CGv@ 5f732dd4     daocore.obj
 0002:00003df8       ??_C@_0CE@KLCN@pDAOQueryDef?9?$DOget_Updatable?$CI?$CGnBo@ 5f732df8     daocore.obj
 0002:00003e1c       ??_C@_0CO@FAJF@pDAOQueryDef?9?$DOget_Type?$CI?$CGquerydef@ 5f732e1c     daocore.obj
 0002:00003e4c       ??_C@_0CG@DIGJ@pDAOQueryDef?9?$DOget_Name?$CI?$CGV_BSTR?$CI?$CG@ 5f732e4c     daocore.obj
 0002:00003e78       ??_7CDaoTableDef@@6B@      5f732e78     daocore.obj
 0002:00003ea0       ??_C@_0MC@IBMF@m_pDatabase?9?$DOm_pDAODatabase?9?$DOCre@ 5f732ea0     daocore.obj
 0002:00003f64       ??_C@_0CG@KMEO@pDAOTableDefs?9?$DOAppend?$CIm_pDAOTabl@ 5f732f64     daocore.obj
 0002:00003f8c       ??_C@_0DM@GNOH@m_pDatabase?9?$DOm_pDAODatabase?9?$DOget@ 5f732f8c     daocore.obj
 0002:00003fc8       ??_C@_0EK@DHEO@pDAOTableDefs?9?$DOget_Item?$CI?5COleVar@ 5f732fc8     daocore.obj
 0002:00004014       ??_C@_0CL@GMF@m_pDAOTableDef?9?$DOget_Updatable?$CI?$CGn@ 5f733014     daocore.obj
 0002:00004040       ??_C@_0CH@LFFO@m_pDAOTableDef?9?$DOput_Name?$CIV_BSTR?$CI@ 5f733040     daocore.obj
 0002:00004068       ??_C@_0CI@GFNK@m_pDAOTableDef?9?$DOget_Name?$CI?$CGV_BSTR@ 5f733068     daocore.obj
 0002:00004090       ??_C@_0DD@FHOC@m_pDAOTableDef?9?$DOput_SourceTableN@ 5f733090     daocore.obj
 0002:000040c4       ??_C@_0DE@CBJH@m_pDAOTableDef?9?$DOget_SourceTableN@ 5f7330c4     daocore.obj
 0002:000040f8       ??_C@_0CK@PHKK@m_pDAOTableDef?9?$DOput_Connect?$CIV_BS@ 5f7330f8     daocore.obj
 0002:00004124       ??_C@_0CL@KFGO@m_pDAOTableDef?9?$DOget_Connect?$CI?$CGV_B@ 5f733124     daocore.obj
 0002:00004150       ??_C@_0CM@DGAH@m_pDAOTableDef?9?$DOput_Attributes?$CIl@ 5f733150     daocore.obj
 0002:0000417c       ??_C@_0CN@EPFM@m_pDAOTableDef?9?$DOget_Attributes?$CI?$CG@ 5f73317c     daocore.obj
 0002:000041ac       ??_C@_0CK@CKHH@m_pDAOTableDef?9?$DOget_DateCreated?$CI@ 5f7331ac     daocore.obj
 0002:000041d8       ??_C@_0CK@ODEK@m_pDAOTableDef?9?$DOget_LastUpdated?$CI@ 5f7331d8     daocore.obj
 0002:00004204       ??_C@_0DC@EKFC@m_pDAOTableDef?9?$DOput_ValidationRu@ 5f733204     daocore.obj
 0002:00004238       ??_C@_0DD@LHDC@m_pDAOTableDef?9?$DOget_ValidationRu@ 5f733238     daocore.obj
 0002:0000426c       ??_C@_0DC@LOBP@m_pDAOTableDef?9?$DOput_ValidationTe@ 5f73326c     daocore.obj
 0002:000042a0       ??_C@_0DD@GAMG@m_pDAOTableDef?9?$DOget_ValidationTe@ 5f7332a0     daocore.obj
 0002:000042d4       ??_C@_0CP@NCFA@m_pDAOTableDef?9?$DOget_RecordCount?$CI@ 5f7332d4     daocore.obj
 0002:00004308       ??_7CDaoFieldInfo@@6B@     5f733308     daocore.obj
 0002:0000430c       ??_C@_0CA@KBPE@m_pDAOFields?9?$DOAppend?$CIpDAOField?$CJ?$AA@ 5f73330c     daocore.obj
 0002:0000432c       ??_C@_0JF@NDIH@m_pDAOTableDef?9?$DOCreateField?$CI?5COl@ 5f73332c     daocore.obj
 0002:000043c4       ??_C@_0CD@MPAH@m_pDAOFields?9?$DODelete?$CIV_BSTR?$CI?$CGvar@ 5f7333c4     daocore.obj
 0002:000043e8       ??_C@_0CB@GDE@m_pDAOIndexes?9?$DOAppend?$CIpDAOIndex?$CJ@ 5f7333e8     daocore.obj
 0002:0000440c       ??_C@_0FF@LAGC@m_pDAOTableDef?9?$DOCreateIndex?$CI?5COl@ 5f73340c     daocore.obj
 0002:00004464       ??_C@_0CE@GGDB@m_pDAOIndexes?9?$DODelete?$CIV_BSTR?$CI?$CGva@ 5f733464     daocore.obj
 0002:00004488       ??_C@_0CC@GCCM@m_pDAOFields?9?$DOget_Count?$CI?$CGnFields@ 5f733488     daocore.obj
 0002:000044ac       ??_C@_0DP@FPAO@m_pDAOFields?9?$DOget_Item?$CI?5COleVari@ 5f7334ac     daocore.obj
 0002:000044ec       ??_C@_0EF@MHNO@m_pDAOFields?9?$DOget_Item?$CI?5COleVari@ 5f7334ec     daocore.obj
 0002:00004534       ??_C@_0CE@LMII@m_pDAOIndexes?9?$DOget_Count?$CI?$CGnIndex@ 5f733534     daocore.obj
 0002:00004558       ??_C@_0EA@IAJA@m_pDAOIndexes?9?$DOget_Item?$CI?5COleVar@ 5f733558     daocore.obj
 0002:00004598       ??_C@_0EG@GOCN@m_pDAOIndexes?9?$DOget_Item?$CI?5COleVar@ 5f733598     daocore.obj
 0002:000045e0       ??_C@_0BO@KAIF@m_pDAOTableDef?9?$DORefreshLink?$CI?$CJ?$AA@ 5f7335e0     daocore.obj
 0002:00004600       ??_C@_0CK@MDGM@m_pDAOTableDef?9?$DOget_Fields?$CI?$CGm_pD@ 5f733600     daocore.obj
 0002:0000462c       ??_C@_0CM@GLNB@m_pDAOTableDef?9?$DOget_Indexes?$CI?$CGm_p@ 5f73362c     daocore.obj
 0002:0000465c       ??_7CDaoQueryDef@@6B@      5f73365c     daocore.obj
 0002:00004698       ??_C@_0GI@HNGJ@m_pDatabase?9?$DOm_pDAODatabase?9?$DOCre@ 5f733698     daocore.obj
 0002:00004700       ??_C@_0HN@FLN@m_pDatabase?9?$DOm_pDAODatabase?9?$DOCre@ 5f733700     daocore.obj
 0002:00004780       ??_C@_0CG@FLGB@pDAOQueryDefs?9?$DOAppend?$CIm_pDAOQuer@ 5f733780     daocore.obj
 0002:000047a8       ??_C@_0DM@IIMB@m_pDatabase?9?$DOm_pDAODatabase?9?$DOget@ 5f7337a8     daocore.obj
 0002:000047e4       ??_C@_0EO@KMBN@m_pDatabase?9?$DOm_pDAODatabase?9?$DOOpe@ 5f7337e4     daocore.obj
 0002:00004834       ??_C@_0HC@LEBM@m_pDatabase?9?$DOm_pDAODatabase?9?$DOCre@ 5f733834     daocore.obj
 0002:000048a8       ??_C@_0BI@GPHC@m_pDAOQueryDef?9?$DOClose?$CI?$CJ?$AA@ 5f7338a8     daocore.obj
 0002:000048c0       ??_C@_0CL@HEGE@m_pDAOQueryDef?9?$DOget_Updatable?$CI?$CGn@ 5f7338c0     daocore.obj
 0002:000048ec       ??_C@_0CI@DLAP@m_pDAOQueryDef?9?$DOget_Name?$CI?$CGV_BSTR@ 5f7338ec     daocore.obj
 0002:00004914       ??_C@_0CH@GAJF@m_pDAOQueryDef?9?$DOput_Name?$CIV_BSTR?$CI@ 5f733914     daocore.obj
 0002:0000493c       ??_C@_0CH@BDHB@m_pDAOQueryDef?9?$DOget_SQL?$CI?$CGV_BSTR?$CI@ 5f73393c     daocore.obj
 0002:00004964       ??_C@_0CG@HMBA@m_pDAOQueryDef?9?$DOput_SQL?$CIV_BSTR?$CI?$CG@ 5f733964     daocore.obj
 0002:0000498c       ??_C@_0CB@IFD@m_pDAOQueryDef?9?$DOget_Type?$CI?$CGnType?$CJ@ 5f73398c     daocore.obj
 0002:000049b0       ??_C@_0CK@ILJJ@m_pDAOQueryDef?9?$DOget_DateCreated?$CI@ 5f7339b0     daocore.obj
 0002:000049dc       ??_C@_0CK@ECKE@m_pDAOQueryDef?9?$DOget_LastUpdated?$CI@ 5f7339dc     daocore.obj
 0002:00004a08       ??_C@_0CL@NHMP@m_pDAOQueryDef?9?$DOget_Connect?$CI?$CGV_B@ 5f733a08     daocore.obj
 0002:00004a34       ??_C@_0CK@FGEE@m_pDAOQueryDef?9?$DOput_Connect?$CIV_BS@ 5f733a34     daocore.obj
 0002:00004a60       ??_C@_0CL@ODLC@m_pDAOQueryDef?9?$DOget_ODBCTimeout?$CI@ 5f733a60     daocore.obj
 0002:00004a8c       ??_C@_0CO@EFO@m_pDAOQueryDef?9?$DOput_ODBCTimeout?$CI@ 5f733a8c     daocore.obj
 0002:00004abc       ??_C@_0DF@JBJO@m_pDAOQueryDef?9?$DOget_ReturnsRecor@ 5f733abc     daocore.obj
 0002:00004af4       ??_C@_0FN@IFJL@m_pDAOQueryDef?9?$DOput_ReturnsRecor@ 5f733af4     daocore.obj
 0002:00004b54       ??_C@_0DH@IBAL@m_pDAOQueryDef?9?$DOget_RecordsAffec@ 5f733b54     daocore.obj
 0002:00004b8c       ??_C@_0DF@FIBD@m_pDAOQueryDef?9?$DOExecute?$CICOleVari@ 5f733b8c     daocore.obj
 0002:00004bc4       ??_C@_0BP@JAF@pDAOParameter?9?$DOget_Value?$CI?$CGvar?$CJ?$AA@ 5f733bc4     daocore.obj
 0002:00004be4       ??_C@_0EN@DKKA@m_pDAOParameters?9?$DOget_Item?$CI?5COle@ 5f733be4     daocore.obj
 0002:00004c34       ??_C@_0EH@EAEJ@m_pDAOParameters?9?$DOget_Item?$CI?5COle@ 5f733c34     daocore.obj
 0002:00004c7c       ??_C@_0CD@KIO@pDAOParameter?9?$DOput_Value?$CIvarValu@ 5f733c7c     daocore.obj
 0002:00004ca0       ??_C@_0CK@MAHP@m_pDAOParameters?9?$DOget_Count?$CI?$CGnPa@ 5f733ca0     daocore.obj
 0002:00004ccc       ??_C@_0CK@GCIC@m_pDAOQueryDef?9?$DOget_Fields?$CI?$CGm_pD@ 5f733ccc     daocore.obj
 0002:00004cf8       ??_C@_0DC@LDGL@m_pDAOQueryDef?9?$DOget_Parameters?$CI?$CG@ 5f733cf8     daocore.obj
 0002:00004d2c       ??_C@_0DB@JEPD@pDAOParameter?9?$DOget_Value?$CI?5?$CGparam@ 5f733d2c     daocore.obj
 0002:00004d60       ??_C@_0CN@IAMG@pDAOParameter?9?$DOget_Type?$CI?5?$CGparami@ 5f733d60     daocore.obj
 0002:00004d90       ??_C@_0CH@MNLB@pDAOParameter?9?$DOget_Name?$CI?$CGV_BSTR?$CI@ 5f733d90     daocore.obj
 0002:00004dbc       ??_7CDaoRecordset@@6B@     5f733dbc     daocore.obj
 0002:00004e3c       ??_C@_0IB@OLCO@m_pQueryDef?9?$DOm_pDAOQueryDef?9?$DO_30@ 5f733e3c     daocore.obj
 0002:00004ec0       ??_C@_0HN@DBDN@m_pTableDef?9?$DOm_pDAOTableDef?9?$DOOpe@ 5f733ec0     daocore.obj
 0002:00004f40       ??_C@_0BJ@NGAG@m_pDAORecordset?9?$DOClose?$CI?$CJ?$AA@ 5f733f40     daocore.obj
 0002:00004f5c       ??_C@_0CO@ENEN@m_pDAORecordset?9?$DORequery?$CI_afxOpt@ 5f733f5c     daocore.obj
 0002:00004f8c       ??_C@_0CC@EHJO@m_pDAORecordset?9?$DORequery?$CIvarDisp@ 5f733f8c     daocore.obj
 0002:00004fb0       ??_C@_0CA@OPCI@m_pDAORecordset?9?$DOget_BOF?$CI?$CGnBOF?$CJ?$AA@ 5f733fb0     daocore.obj
 0002:00004fd0       ??_C@_0CA@LKNJ@m_pDAORecordset?9?$DOget_EOF?$CI?$CGnEOF?$CJ?$AA@ 5f733fd0     daocore.obj
 0002:00004ff0       ??_C@_0CM@BOKG@m_pDAORecordset?9?$DOget_Updatable?$CI?$CG@ 5f733ff0     daocore.obj
 0002:0000501c       ??_C@_0DA@PJGA@m_pDAORecordset?9?$DOget_Restartable@ 5f73401c     daocore.obj
 0002:0000504c       ??_C@_0DC@DHEI@m_pDAORecordset?9?$DOget_Transaction@ 5f73404c     daocore.obj
 0002:00005080       ??_C@_0DC@BDFH@m_pDAORecordset?9?$DOget_Bookmarkabl@ 5f734080     daocore.obj
 0002:000050b4       ??_C@_0CJ@DDPM@m_pDAORecordset?9?$DOget_Name?$CI?$CGV_BST@ 5f7340b4     daocore.obj
 0002:000050e0       ??_C@_0CC@NAA@m_pDAORecordset?9?$DOget_Type?$CI?$CGnType@ 5f7340e0     daocore.obj
 0002:00005104       ??_C@_0CK@OCGL@m_pDAORecordset?9?$DOget_EditMode?$CI?$CGn@ 5f734104     daocore.obj
 0002:00005130       ??_C@_0CL@EJNE@m_pDAORecordset?9?$DOget_DateCreated@ 5f734130     daocore.obj
 0002:0000515c       ??_C@_0CL@IAOJ@m_pDAORecordset?9?$DOget_LastUpdated@ 5f73415c     daocore.obj
 0002:00005188       ??_C@_0CP@EDLK@m_pDAORecordset?9?$DOget_LastModifie@ 5f734188     daocore.obj
 0002:000051b8       ??_C@_0DD@KGH@m_pDAORecordset?9?$DOget_ValidationR@ 5f7341b8     daocore.obj
 0002:000051ec       ??_C@_0DD@POCK@m_pDAORecordset?9?$DOget_ValidationT@ 5f7341ec     daocore.obj
 0002:00005220       ??_C@_0CK@NNM@m_pDAORecordset?9?$DOget_Index?$CI?$CGV_BS@ 5f734220     daocore.obj
 0002:0000524c       ??_C@_0CJ@CEAC@m_pDAORecordset?9?$DOput_Index?$CIV_BST@ 5f73424c     daocore.obj
 0002:00005278       ??_C@_0DA@CFBI@m_pDAORecordset?9?$DOget_RecordCount@ 5f734278     daocore.obj
 0002:000052a8       ??_C@_0CL@BMFG@m_pDAORecordset?9?$DOget_Bookmark?$CI?$CGv@ 5f7342a8     daocore.obj
 0002:000052d4       ??_C@_0DD@MOL@m_pDAORecordset?9?$DOput_Bookmark?$CI?$CGv@ 5f7342d4     daocore.obj
 0002:00005308       ??_C@_0DC@GDMD@m_pDAORecordset?9?$DOget_AbsolutePos@ 5f734308     daocore.obj
 0002:0000533c       ??_C@_0DB@GLNO@m_pDAORecordset?9?$DOput_AbsolutePos@ 5f73433c     daocore.obj
 0002:00005370       ??_C@_0DB@LIAP@m_pDAORecordset?9?$DOget_PercentPosi@ 5f734370     daocore.obj
 0002:000053a4       ??_C@_0DA@MHMB@m_pDAORecordset?9?$DOput_PercentPosi@ 5f7343a4     daocore.obj
 0002:000053d4       ??_C@_0CM@OLNL@m_pDAORecordset?9?$DOMove?$CIlRows?0?5COl@ 5f7343d4     daocore.obj
 0002:00005400       ??_C@_0CA@IGPM@m_pDAORecordset?9?$DO_30_MoveLast?$CI?$CJ?$AA@ 5f734400     daocore.obj
 0002:00005420       ??_C@_0BN@OKBK@m_pDAORecordset?9?$DOMoveFirst?$CI?$CJ?$AA@ 5f734420     daocore.obj
 0002:00005440       ??_C@_0CA@PGPJ@m_pDAORecordset?9?$DOMovePrevious?$CI?$CJ?$AA@ 5f734440     daocore.obj
 0002:00005460       ??_C@_0BM@KCOP@m_pDAORecordset?9?$DOMoveNext?$CI?$CJ?$AA@ 5f734460     daocore.obj
 0002:0000547c       ??_C@_0CI@BDFN@m_pDAORecordset?9?$DOFindLast?$CIV_BSTR@ 5f73447c     daocore.obj
 0002:000054a4       ??_C@_0CJ@NOGD@m_pDAORecordset?9?$DOFindFirst?$CIV_BST@ 5f7344a4     daocore.obj
 0002:000054d0       ??_C@_0CM@CFIG@m_pDAORecordset?9?$DOFindPrevious?$CIV_@ 5f7344d0     daocore.obj
 0002:000054fc       ??_C@_0CI@IEGA@m_pDAORecordset?9?$DOFindNext?$CIV_BSTR@ 5f7344fc     daocore.obj
 0002:00005524       ??_C@_0BKF@GBHJ@m_pDAORecordset?9?$DOSeek?$CIV_BSTR?$CI?$CGva@ 5f734524     daocore.obj
 0002:000056cc       ??_C@_0PE@MNIL@m_pDAORecordset?9?$DOSeek?$CIV_BSTR?$CI?$CGva@ 5f7346cc     daocore.obj
 0002:000057c0       ??_C@_0CE@GKGD@m_pDAORecordset?9?$DO_30_CancelUpdat@ 5f7347c0     daocore.obj
 0002:000057e4       ??_C@_0FG@JILN@m_pDAORecordset?9?$DOput_LockEdits?$CI?5@ 5f7347e4     daocore.obj
 0002:0000583c       ??_C@_0CM@FJGM@m_pDAORecordset?9?$DOget_LockEdits?$CI?$CG@ 5f73483c     daocore.obj
 0002:00005868       ??_C@_0DF@NEPL@m_pDAORecordset?9?$DOput_CacheStart?$CI@ 5f734868     daocore.obj
 0002:000058a0       ??_C@_0CN@BBCI@m_pDAORecordset?9?$DOget_CacheStart?$CI@ 5f7348a0     daocore.obj
 0002:000058d0       ??_C@_0CG@GPJG@m_pDAORecordset?9?$DOput_CacheSize?$CIl@ 5f7348d0     daocore.obj
 0002:000058f8       ??_C@_0CH@FFJB@m_pDAORecordset?9?$DOget_CacheSize?$CI?$CG@ 5f7348f8     daocore.obj
 0002:00005920       ??_C@_0JP@FOGE@m_pDAORecordset?9?$DOFillCache?$CI?5pSiz@ 5f734920     daocore.obj
 0002:000059c0       ??_C@_0BK@MEND@m_pDAORecordset?9?$DOAddNew?$CI?$CJ?$AA@ 5f7349c0     daocore.obj
 0002:000059dc       ??_C@_0BI@CNBL@m_pDAORecordset?9?$DOEdit?$CI?$CJ?$AA@ 5f7349dc     daocore.obj
 0002:000059f4       ??_C@_0BO@JCIA@m_pDAORecordset?9?$DO_30_Update?$CI?$CJ?$AA@ 5f7349f4     daocore.obj
 0002:00005a14       ??_C@_0BK@DPAI@m_pDAORecordset?9?$DODelete?$CI?$CJ?$AA@ 5f734a14     daocore.obj
 0002:00005a30       ??_C@_0EK@CMJC@m_pDAORecordset?9?$DOget_Collect?$CI?5CO@ 5f734a30     daocore.obj
 0002:00005a7c       ??_C@_0EE@NBLG@m_pDAORecordset?9?$DOget_Collect?$CI?5CO@ 5f734a7c     daocore.obj
 0002:00005ac0       ??_C@_0EJ@FHEM@m_pDAORecordset?9?$DOput_Collect?$CI?5CO@ 5f734ac0     daocore.obj
 0002:00005b0c       ??_C@_0ED@ENAG@m_pDAORecordset?9?$DOput_Collect?$CI?5CO@ 5f734b0c     daocore.obj
 0002:00005b50       ??_C@_0CL@KAMP@m_pDAORecordset?9?$DOget_Fields?$CI?$CGm_p@ 5f734b50     daocore.obj
 0002:00005b7c       ??_C@_0DJ@FHAD@m_pTableDef?9?$DOm_pDAOTableDef?9?$DOget@ 5f734b7c     daocore.obj
 0002:00005bb8       ??_C@_01FAJB@?$DL?$AA@     5f734bb8     daocore.obj
 0002:00005bbc       ??_C@_0FI@LEEG@m_pDAORecordset?9?$DOQueryInterface?$CI@ 5f734bbc     daocore.obj
 0002:00005c14       ??_C@_0CI@ILFL@m_pDAORecordset?9?$DOget_NoMatch?$CI?$CGnN@ 5f734c14     daocore.obj
 0002:00005c3c       ??_C@_0CA@MLFB@?6m_bCheckCacheForDirtyFields?5?$DN?5?$AA@ 5f734c3c     daocore.obj
 0002:00005c5c       ??_C@_0BF@FEP@?6m_strRequerySort?5?$DN?5?$AA@ 5f734c5c     daocore.obj
 0002:00005c74       ??_C@_0BH@NPKA@?6m_strRequeryFilter?5?$DN?5?$AA@ 5f734c74     daocore.obj
 0002:00005c8c       ??_C@_0BE@OAFC@?6m_strRequerySQL?5?$DN?5?$AA@ 5f734c8c     daocore.obj
 0002:00005ca0       ??_C@_0O@JOGM@?6m_strSort?5?$DN?5?$AA@ 5f734ca0     daocore.obj
 0002:00005cb0       ??_C@_0BA@ICBM@?6m_strFilter?5?$DN?5?$AA@ 5f734cb0     daocore.obj
 0002:00005cc0       ??_C@_0P@CAKJ@?6m_nOptions?5?$DN?5?$AA@ 5f734cc0     daocore.obj
 0002:00005cd0       ??_C@_0BD@FPPO@?6m_nDefaultType?5?$DN?5?$AA@ 5f734cd0     daocore.obj
 0002:00005ce4       ??_C@_0BA@DPMC@?6m_nOpenType?5?$DN?5?$AA@ 5f734ce4     daocore.obj
 0002:00005cf4       ??_C@_0M@NMDE@?6m_bOpen?5?$DN?5?$AA@ 5f734cf4     daocore.obj
 0002:00005d00       ??_C@_0CN@LODG@pDAOField?9?$DOget_ValidationText?$CI?$CGV@ 5f734d00     daocore.obj
 0002:00005d30       ??_C@_0CN@EKHL@pDAOField?9?$DOget_ValidationRule?$CI?$CGV@ 5f734d30     daocore.obj
 0002:00005d60       ??_C@_0CK@NMNF@pDAOField?9?$DOget_SourceTable?$CI?$CGV_BS@ 5f734d60     daocore.obj
 0002:00005d8c       ??_C@_0CK@NMGJ@pDAOField?9?$DOget_SourceField?$CI?$CGV_BS@ 5f734d8c     daocore.obj
 0002:00005db8       ??_C@_0DN@PLFL@pDAOField?9?$DOget_CollatingOrder?$CI?5?$CG@ 5f734db8     daocore.obj
 0002:00005df8       ??_C@_0CH@BDEE@pDAOField?9?$DOget_AllowZeroLength?$CI?$CG@ 5f734df8     daocore.obj
 0002:00005e20       ??_C@_0CA@GJNH@pDAOField?9?$DOget_Required?$CI?$CGnBool?$CJ?$AA@ 5f734e20     daocore.obj
 0002:00005e40       ??_C@_0DP@GBEA@pDAOField?9?$DOget_OrdinalPosition?$CI?5@ 5f734e40     daocore.obj
 0002:00005e80       ??_C@_0DE@DLJC@pDAOField?9?$DOget_Attributes?$CI?$CGfield@ 5f734e80     daocore.obj
 0002:00005eb4       ??_C@_0CI@DFJD@pDAOField?9?$DOget_Size?$CI?$CGfieldinfo?4m@ 5f734eb4     daocore.obj
 0002:00005edc       ??_C@_0CI@LPDA@pDAOField?9?$DOget_Type?$CI?$CGfieldinfo?4m@ 5f734edc     daocore.obj
 0002:00005f04       ??_C@_0CM@OIHD@pDAOField?9?$DOput_ValidationText?$CIV_@ 5f734f04     daocore.obj
 0002:00005f30       ??_C@_0CM@KFNC@pDAOField?9?$DOput_ValidationRule?$CIV_@ 5f734f30     daocore.obj
 0002:00005f5c       ??_C@_0CN@ECE@pDAOField?9?$DOput_AllowZeroLength?$CIA@ 5f734f5c     daocore.obj
 0002:00005f8c       ??_C@_0CG@NDE@pDAOField?9?$DOput_Required?$CIAFX_DAO_@ 5f734f8c     daocore.obj
 0002:00005fb4       ??_C@_0DO@LDPI@pDAOField?9?$DOput_OrdinalPosition?$CI?5@ 5f734fb4     daocore.obj
 0002:00005ff4       ??_C@_0DD@KMNM@pDAOField?9?$DOput_Attributes?$CIfieldi@ 5f734ff4     daocore.obj
 0002:00006028       ??_C@_0CF@IAPF@?$CIpDAOField?9?$DO?$CKpMethod?$CJ?$CI?$CGV_BSTR?$CI?$CGv@ 5f735028     daocore.obj
 0002:00006050       ??_C@_0CC@GCFC@pDAOField?9?$DOget_DefaultValue?$CI?$CGvar@ 5f735050     daocore.obj
 0002:00006074       ??_C@_0CE@DCCL@?$CIpDAOField?9?$DO?$CKpMethod?$CJ?$CIV_BSTR?$CI?$CGva@ 5f735074     daocore.obj
 0002:00006098       ??_C@_0CB@DPPD@pDAOField?9?$DOput_DefaultValue?$CIvar?$CJ@ 5f735098     daocore.obj
 0002:000060bc       ??_C@_0DL@MFON@pDAOIndex?9?$DOget_DistinctCount?$CI?5?$CGi@ 5f7350bc     daocore.obj
 0002:000060f8       ??_C@_0BP@GBPC@pDAOIndex?9?$DOget_Foreign?$CI?$CGnBool?$CJ?$AA@ 5f7350f8     daocore.obj
 0002:00006118       ??_C@_0CA@LEOO@pDAOIndex?9?$DOget_Required?$CI?$CGnBool?$CJ?$AA@ 5f735118     daocore.obj
 0002:00006138       ??_C@_0CD@PNHL@pDAOIndex?9?$DOget_IgnoreNulls?$CI?$CGnBoo@ 5f735138     daocore.obj
 0002:0000615c       ??_C@_0CB@MCH@pDAOIndex?9?$DOget_Clustered?$CI?$CGnBool?$CJ@ 5f73515c     daocore.obj
 0002:00006180       ??_C@_0BO@HDBC@pDAOIndex?9?$DOget_Unique?$CI?$CGnBool?$CJ?$AA@ 5f735180     daocore.obj
 0002:000061a0       ??_C@_0BP@JAAH@pDAOIndex?9?$DOget_Primary?$CI?$CGnBool?$CJ?$AA@ 5f7351a0     daocore.obj
 0002:000061c0       ??_C@_0CD@MEGG@pDAOIndex?9?$DOget_Name?$CI?$CGV_BSTR?$CI?$CGvar@ 5f7351c0     daocore.obj
 0002:000061e4       ??_C@_0CG@NMKH@pDAOIndex?9?$DOput_Required?$CIAFX_DAO_@ 5f7351e4     daocore.obj
 0002:0000620c       ??_C@_0CJ@GEID@pDAOIndex?9?$DOput_IgnoreNulls?$CIAFX_D@ 5f73520c     daocore.obj
 0002:00006238       ??_C@_0CH@PIFK@pDAOIndex?9?$DOput_Clustered?$CIAFX_DAO@ 5f735238     daocore.obj
 0002:00006260       ??_C@_0CE@PPGA@pDAOIndex?9?$DOput_Unique?$CIAFX_DAO_TR@ 5f735260     daocore.obj
 0002:00006284       ??_C@_0CF@ONFI@pDAOIndex?9?$DOput_Primary?$CIAFX_DAO_T@ 5f735284     daocore.obj
 0002:000062ac       ??_C@_0EJ@HLNA@var?4pdispVal?9?$DOQueryInterface?$CI?5gu@ 5f7352ac     daocore.obj
 0002:000062f8       ??_C@_0BM@FLME@pDAOIndex?9?$DOget_Fields?$CI?$CGvar?$CJ?$AA@ 5f7352f8     daocore.obj
 0002:00006314       ??_C@_0CI@GIHF@pDAOField?9?$DOget_Attributes?$CI?$CGlAttr@ 5f735314     daocore.obj
 0002:0000633c       ??_C@_0DN@MHHF@var?4pdispVal?9?$DOQueryInterface?$CI?5gu@ 5f73533c     daocore.obj
 0002:0000637c       ??_C@_0DF@CLB@pDAOIndexFields?9?$DOget_Item?$CICOleVa@ 5f73537c     daocore.obj
 0002:000063b4       ??_C@_0CE@GNBF@pDAOIndexFields?9?$DOget_Count?$CI?$CGnCou@ 5f7353b4     daocore.obj
 0002:000063dc       ??_7CDaoIndexFieldInfo@@6B@ 5f7353dc     daocore.obj
 0002:000063e0       ??_C@_0CH@BPFN@pDAOField?9?$DOput_Attributes?$CIlAttri@ 5f7353e0     daocore.obj
 0002:00006408       ??_C@_0JA@MEIF@pDAOIndex?9?$DOCreateField?$CI?5COleVari@ 5f735408     daocore.obj
 0002:00006498       ??_C@_0BH@FGDO@ICDAORecordset?4GetRows?$AA@ 5f735498     daocore.obj
 0002:000064b0       ??_C@_0GH@DHEN@pCF2?9?$DOCreateInstanceLic?$CI?5NULL?0?5N@ 5f7354b0     daocore.obj
 0002:00006518       ??_C@_0GA@FMGC@?3?3CoGetClassObject?$CIclsidEngine?0?5@ 5f735518     daocore.obj
 0002:00006578       ??_C@_0CF@NAPJ@mjgcqcejfchcijecpdhckcdjqigdejfc@ 5f735578     daocore.obj
 0002:000065a0       ??_C@_0CF@CBFC@mbmabptebkjcdlgtjmskjwtsdhjbmkmw@ 5f7355a0     daocore.obj
 0002:000065c8       ??_C@_0BF@DC@?3?3CoInitialize?$CINULL?$CJ?$AA@ 5f7355c8     daocore.obj
 0002:000065e0       ?_afxDoublePseudoNull@@3NB 5f7355e0     daodfx.obj
 0002:000065e8       ?_afxFloatPseudoNull@@3MB  5f7355e8     daodfx.obj
 0002:000065ec       ??_C@_09CGOK@?5DateTime?$AA@ 5f7355ec     daodfx.obj
 0002:000065f8       ??_C@_0M@BGKI@?5IEEEDouble?$AA@ 5f7355f8     daodfx.obj
 0002:00006604       ??_C@_0M@GOBO@?5IEEESingle?$AA@ 5f735604     daodfx.obj
 0002:00006610       ??_C@_09GDCP@?5Currency?$AA@ 5f735610     daodfx.obj
 0002:0000661c       ??_C@_05BJMF@?5Long?$AA@   5f73561c     daodfx.obj
 0002:00006624       ??_C@_06KOJB@?5Short?$AA@  5f735624     daodfx.obj
 0002:0000662c       ??_C@_05IGCC@?5Byte?$AA@   5f73562c     daodfx.obj
 0002:00006634       ??_C@_04KDMA@?5Bit?$AA@    5f735634     daodfx.obj
 0002:0000663c       ??_C@_0M@MOAI@?5LongBinary?$AA@ 5f73563c     daodfx.obj
 0002:00006648       ??_C@_05BJHD@?5Text?$AA@   5f735648     daodfx.obj
 0002:00006650       ?messageMap@CDaoRecordView@@1UAFX_MSGMAP@@B 5f735650     daoview.obj
 0002:00006658       ?_messageEntries@CDaoRecordView@@0QBUAFX_MSGMAP_ENTRY@@B 5f735658     daoview.obj
 0002:00006730       ?classCDaoRecordView@CDaoRecordView@@2UCRuntimeClass@@B 5f735730     daoview.obj
 0002:00006748       ??_C@_0P@KPJP@CDaoRecordView?$AA@ 5f735748     daoview.obj
 0002:0000675c       ??_7CDaoRecordView@@6B@    5f73575c     daoview.obj
 0002:00006874       ??_C@_0DD@KKOA@Warning?3?5can?8t?5set?5checkbox?5valu@ 5f735874     daoview.obj
 0002:000068a8       ??_C@_0DD@LLGN@Warning?3?5can?8t?5set?5field?5NULL?5fo@ 5f7358a8     daoview.obj
 0002:000068dc       ??_C@_0BE@CLIM@m_varBookmarkLast?5?$DN?$AA@ 5f7358dc     daoview.obj
 0002:000068f0       ??_C@_0BF@EDLD@m_varBookmarkFirst?5?$DN?$AA@ 5f7358f0     daoview.obj
 0002:00006908       ??_C@_0BH@FBNH@m_varBookmarkCurrent?5?$DN?$AA@ 5f735908     daoview.obj
 0002:00006920       ??_C@_0M@LNMN@m_nStatus?5?$DN?$AA@ 5f735920     daoview.obj
 0002:00006930       ?classCOleDBRecordView@COleDBRecordView@@2UCRuntimeClass@@B 5f735930     viewoled.obj
 0002:00006948       ??_C@_0BB@HKOA@COleDBRecordView?$AA@ 5f735948     viewoled.obj
 0002:00006960       ?messageMap@COleDBRecordView@@1UAFX_MSGMAP@@B 5f735960     viewoled.obj
 0002:00006968       ?_messageEntries@COleDBRecordView@@0QBUAFX_MSGMAP_ENTRY@@B 5f735968     viewoled.obj
 0002:00006a40       ??_C@_0CB@CEAB@GetData?5failed?5?9?5HRESULT?5?$DN?50x?$CFX?6@ 5f735a40     viewoled.obj
 0002:00006a64       ??_C@_0BB@OJDA@m_pAccessor?5?$CB?$DN?50?$AA@ 5f735a64     viewoled.obj
 0002:00006a78       ??_C@_0CI@GKMH@E?3?28168?2vc98?2mfc?2atl?2include?2atl@ 5f735a78     viewoled.obj
 0002:00006aa0       ??_C@_0BA@EFBK@m_spRowset?5?$CB?$DN?50?$AA@ 5f735aa0     viewoled.obj
 0002:00006ab0       ??_C@_05BFMC@ATL?3?5?$AA@  5f735ab0     viewoled.obj
 0002:00006ab8       ??_C@_09PLJB@atlbase?4h?$AA@ 5f735ab8     viewoled.obj
 0002:00006ac4       ??_C@_0BI@CIAH@nBuf?5?$DM?5sizeof?$CIszBuffer?$CJ?$AA@ 5f735ac4     viewoled.obj
 0002:00006adc       ??_C@_0CP@HDHG@GetData?5from?5MoveLast?5failed?5?9?5H@ 5f735adc     viewoled.obj
 0002:00006b0c       ??_C@_0BF@GPJA@m_pAccessorInfo?5?$CB?$DN?50?$AA@ 5f735b0c     viewoled.obj
 0002:00006b24       ??_C@_0BJ@NICA@nAccessor?5?$DM?5m_nAccessors?$AA@ 5f735b24     viewoled.obj
 0002:00006b40       ??_C@_0M@DLL@m_hRow?5?$CB?$DN?50?$AA@ 5f735b40     viewoled.obj
 0002:00006b4c       ??_C@_0BH@DLBO@nAccessor?$DMm_nAccessors?$AA@ 5f735b4c     viewoled.obj
 0002:00006b64       ??_C@_04GBK@p?$CB?$DN0?$AA@ 5f735b64     viewoled.obj
 0002:00006ba0       ??_7type_info@@6B@         5f735ba0     msvcrtd:ti_inst.obj
 0002:00006ba4       ??_C@_08JKC@crtdll?4c?$AA@ 5f735ba4     msvcrtd:crtdll.obj
 0002:00006bb0       _IID_IClassFactory2        5f735bb0     uuid:ocidl_i_guid4.obj
 0002:00006bc0       _LIBID_CJETSQLHELP         5f735bc0     daouuid:daouuid.obj
 0002:00006bd0       _LIBID_CDAO                5f735bd0     daouuid:daouuid.obj
 0002:00006be0       _LIBID_CDAO25              5f735be0     daouuid:daouuid.obj
 0002:00006bf0       _BETA_LIBID_CDAO           5f735bf0     daouuid:daouuid.obj
 0002:00006c00       _BETA_LIBID_CDAO25         5f735c00     daouuid:daouuid.obj
 0002:00006c10       _IID_IDAOStdObject         5f735c10     daouuid:daouuid.obj
 0002:00006c20       _IID_IDAOStdCollection     5f735c20     daouuid:daouuid.obj
 0002:00006c30       _CLSID_CDAODBEngine        5f735c30     daouuid:daouuid.obj
 0002:00006c40       _CLSID_CDAOPrivDBEngine    5f735c40     daouuid:daouuid.obj
 0002:00006c50       _CLSID_CDAOConnection      5f735c50     daouuid:daouuid.obj
 0002:00006c60       _CLSID_CDAOTableDef        5f735c60     daouuid:daouuid.obj
 0002:00006c70       _CLSID_CDAOField           5f735c70     daouuid:daouuid.obj
 0002:00006c80       _CLSID_CDAOIndex           5f735c80     daouuid:daouuid.obj
 0002:00006c90       _CLSID_CDAOGroup           5f735c90     daouuid:daouuid.obj
 0002:00006ca0       _CLSID_CDAOUser            5f735ca0     daouuid:daouuid.obj
 0002:00006cb0       _CLSID_CDAOQueryDef        5f735cb0     daouuid:daouuid.obj
 0002:00006cc0       _CLSID_CDAORelation        5f735cc0     daouuid:daouuid.obj
 0002:00006cd0       _CLSID35_CDAODBEngine      5f735cd0     daouuid:daouuid.obj
 0002:00006ce0       _CLSID35_CDAOPrivDBEngine  5f735ce0     daouuid:daouuid.obj
 0002:00006cf0       _CLSID35_CDAOConnection    5f735cf0     daouuid:daouuid.obj
 0002:00006d00       _CLSID35_CDAOTableDef      5f735d00     daouuid:daouuid.obj
 0002:00006d10       _CLSID35_CDAOField         5f735d10     daouuid:daouuid.obj
 0002:00006d20       _CLSID35_CDAOIndex         5f735d20     daouuid:daouuid.obj
 0002:00006d30       _CLSID35_CDAOGroup         5f735d30     daouuid:daouuid.obj
 0002:00006d40       _CLSID35_CDAOUser          5f735d40     daouuid:daouuid.obj
 0002:00006d50       _CLSID35_CDAOQueryDef      5f735d50     daouuid:daouuid.obj
 0002:00006d60       _CLSID35_CDAORelation      5f735d60     daouuid:daouuid.obj
 0002:00006d70       _IID_IDAODBEngine          5f735d70     daouuid:daouuid.obj
 0002:00006d80       _IID_IDAODBEngineW         5f735d80     daouuid:daouuid.obj
 0002:00006d90       _IID_IDAOError             5f735d90     daouuid:daouuid.obj
 0002:00006da0       _IID_IDAOErrorW            5f735da0     daouuid:daouuid.obj
 0002:00006db0       _IID_IDAOErrors            5f735db0     daouuid:daouuid.obj
 0002:00006dc0       _IID_IDAOErrorsW           5f735dc0     daouuid:daouuid.obj
 0002:00006dd0       _IID_IDAOProperty          5f735dd0     daouuid:daouuid.obj
 0002:00006de0       _IID_IDAOPropertyW         5f735de0     daouuid:daouuid.obj
 0002:00006df0       _IID_IDAOProperties        5f735df0     daouuid:daouuid.obj
 0002:00006e00       _IID_IDAOPropertiesW       5f735e00     daouuid:daouuid.obj
 0002:00006e10       _IID_IDAORecordset         5f735e10     daouuid:daouuid.obj
 0002:00006e20       _IID_IDAORecordsetW        5f735e20     daouuid:daouuid.obj
 0002:00006e30       _IID_IDAORecordsets        5f735e30     daouuid:daouuid.obj
 0002:00006e40       _IID_IDAORecordsetsW       5f735e40     daouuid:daouuid.obj
 0002:00006e50       _IID_ICDAORecordset        5f735e50     daouuid:daouuid.obj
 0002:00006e60       _IID_IDAOWorkspace         5f735e60     daouuid:daouuid.obj
 0002:00006e70       _IID_IDAOWorkspaceW        5f735e70     daouuid:daouuid.obj
 0002:00006e80       _IID_IDAOWorkspaces        5f735e80     daouuid:daouuid.obj
 0002:00006e90       _IID_IDAOWorkspacesW       5f735e90     daouuid:daouuid.obj
 0002:00006ea0       _IID_IDAOConnection        5f735ea0     daouuid:daouuid.obj
 0002:00006eb0       _IID_IDAOConnectionW       5f735eb0     daouuid:daouuid.obj
 0002:00006ec0       _IID_IDAOConnections       5f735ec0     daouuid:daouuid.obj
 0002:00006ed0       _IID_IDAOConnectionsW      5f735ed0     daouuid:daouuid.obj
 0002:00006ee0       _IID_IDAOTableDef          5f735ee0     daouuid:daouuid.obj
 0002:00006ef0       _IID_IDAOTableDefW         5f735ef0     daouuid:daouuid.obj
 0002:00006f00       _IID_IDAOTableDefs         5f735f00     daouuid:daouuid.obj
 0002:00006f10       _IID_IDAOTableDefsW        5f735f10     daouuid:daouuid.obj
 0002:00006f20       _IID_IDAOField             5f735f20     daouuid:daouuid.obj
 0002:00006f30       _IID_IDAOFieldW            5f735f30     daouuid:daouuid.obj
 0002:00006f40       _IID_IDAOFields            5f735f40     daouuid:daouuid.obj
 0002:00006f50       _IID_IDAOFieldsW           5f735f50     daouuid:daouuid.obj
 0002:00006f60       _IID_IDAOIndex             5f735f60     daouuid:daouuid.obj
 0002:00006f70       _IID_IDAOIndexW            5f735f70     daouuid:daouuid.obj
 0002:00006f80       _IID_IDAOIndexes           5f735f80     daouuid:daouuid.obj
 0002:00006f90       _IID_IDAOIndexesW          5f735f90     daouuid:daouuid.obj
 0002:00006fa0       _IID_IDAOIndexFields       5f735fa0     daouuid:daouuid.obj
 0002:00006fb0       _IID_IDAOIndexFieldsW      5f735fb0     daouuid:daouuid.obj
 0002:00006fc0       _IID_IDAOGroup             5f735fc0     daouuid:daouuid.obj
 0002:00006fd0       _IID_IDAOGroupW            5f735fd0     daouuid:daouuid.obj
 0002:00006fe0       _IID_IDAOGroups            5f735fe0     daouuid:daouuid.obj
 0002:00006ff0       _IID_IDAOGroupsW           5f735ff0     daouuid:daouuid.obj
 0002:00007000       _IID_IDAOUser              5f736000     daouuid:daouuid.obj
 0002:00007010       _IID_IDAOUserW             5f736010     daouuid:daouuid.obj
 0002:00007020       _IID_IDAOUsers             5f736020     daouuid:daouuid.obj
 0002:00007030       _IID_IDAOUsersW            5f736030     daouuid:daouuid.obj
 0002:00007040       _IID_IDAODatabase          5f736040     daouuid:daouuid.obj
 0002:00007050       _IID_IDAODatabaseW         5f736050     daouuid:daouuid.obj
 0002:00007060       _IID_IDAODatabases         5f736060     daouuid:daouuid.obj
 0002:00007070       _IID_IDAODatabasesW        5f736070     daouuid:daouuid.obj
 0002:00007080       _IID_IDAOQueryDef          5f736080     daouuid:daouuid.obj
 0002:00007090       _IID_IDAOQueryDefW         5f736090     daouuid:daouuid.obj
 0002:000070a0       _IID_IDAOQueryDefs         5f7360a0     daouuid:daouuid.obj
 0002:000070b0       _IID_IDAOQueryDefsW        5f7360b0     daouuid:daouuid.obj
 0002:000070c0       _IID_IDAOParameter         5f7360c0     daouuid:daouuid.obj
 0002:000070d0       _IID_IDAOParameterW        5f7360d0     daouuid:daouuid.obj
 0002:000070e0       _IID_IDAOParameters        5f7360e0     daouuid:daouuid.obj
 0002:000070f0       _IID_IDAOParametersW       5f7360f0     daouuid:daouuid.obj
 0002:00007100       _IID_IDAORelation          5f736100     daouuid:daouuid.obj
 0002:00007110       _IID_IDAORelationW         5f736110     daouuid:daouuid.obj
 0002:00007120       _IID_IDAORelations         5f736120     daouuid:daouuid.obj
 0002:00007130       _IID_IDAORelationsW        5f736130     daouuid:daouuid.obj
 0002:00007140       _IID_IDAOContainer         5f736140     daouuid:daouuid.obj
 0002:00007150       _IID_IDAOContainerW        5f736150     daouuid:daouuid.obj
 0002:00007160       _IID_IDAOContainers        5f736160     daouuid:daouuid.obj
 0002:00007170       _IID_IDAOContainersW       5f736170     daouuid:daouuid.obj
 0002:00007180       _IID_IDAODocument          5f736180     daouuid:daouuid.obj
 0002:00007190       _IID_IDAODocumentW         5f736190     daouuid:daouuid.obj
 0002:000071a0       _IID_IDAODocuments         5f7361a0     daouuid:daouuid.obj
 0002:000071b0       _IID_IDAODocumentsW        5f7361b0     daouuid:daouuid.obj
 0002:000071c0       _IID_IDAOCollection        5f7361c0     daouuid:daouuid.obj
 0002:000071d0       _IID_IDAODynaCollection    5f7361d0     daouuid:daouuid.obj
 0002:000071e0       _IID_IDAOQueryCP           5f7361e0     daouuid:daouuid.obj
 0002:000071f0       _IID_IDAOQueryAS           5f7361f0     daouuid:daouuid.obj
 0002:00007200       _IID_ICDAOJETDBEngine      5f736200     daouuid:daouuid.obj
 0002:00007210       _IID_ICDAOJETError         5f736210     daouuid:daouuid.obj
 0002:00007220       _IID_ICDAOJETRecordset     5f736220     daouuid:daouuid.obj
 0002:00007230       _IID_ICDAOJETWorkspace     5f736230     daouuid:daouuid.obj
 0002:00007240       _IID_ICDAOJETField         5f736240     daouuid:daouuid.obj
 0002:00007250       _IID_ICDAOJETDatabase      5f736250     daouuid:daouuid.obj
 0002:00007260       _IID_IDAOSnapshot          5f736260     daouuid:daouuid.obj
 0002:00007270       _IID_IDAOTable             5f736270     daouuid:daouuid.obj
 0002:00007280       _IID_IDAODynaset           5f736280     daouuid:daouuid.obj
 0002:00007290       _IID_IDisconnect           5f736290     daouuid:daouuid.obj
 0002:000072a0       _IID_IDisconnectAll        5f7362a0     daouuid:daouuid.obj
 0002:000072b0       _IID_IDSCAdviseSink        5f7362b0     daouuid:daouuid.obj
 0002:000072c0       _IID_IDSCConnectionPoint   5f7362c0     daouuid:daouuid.obj
 0002:000072d0       _IID_IDBAdviseSink         5f7362d0     daouuid:daouuid.obj
 0002:000072e0       _IID_IDBConnectionPoint    5f7362e0     daouuid:daouuid.obj
 0002:000072f0       _LIBID30_CDAO              5f7362f0     daouuid:daouuid.obj
 0002:00007300       _LIBID30_CDAO25            5f736300     daouuid:daouuid.obj
 0002:00007310       _IID30_IDAOStdObject       5f736310     daouuid:daouuid.obj
 0002:00007320       _IID30_IDAOStdCollection   5f736320     daouuid:daouuid.obj
 0002:00007330       _CLSID30_CDAODBEngine      5f736330     daouuid:daouuid.obj
 0002:00007340       _IID30_IDAODBEngine        5f736340     daouuid:daouuid.obj
 0002:00007350       _IID30_IDAODBEngineW       5f736350     daouuid:daouuid.obj
 0002:00007360       _IID30_ICDAOJETDBEngine    5f736360     daouuid:daouuid.obj
 0002:00007370       _CLSID30_CDAOPrivDBEngine  5f736370     daouuid:daouuid.obj
 0002:00007380       _IID30_IDAOError           5f736380     daouuid:daouuid.obj
 0002:00007390       _IID30_IDAOErrorW          5f736390     daouuid:daouuid.obj
 0002:000073a0       _IID30_IDAOErrors          5f7363a0     daouuid:daouuid.obj
 0002:000073b0       _IID30_IDAOErrorsW         5f7363b0     daouuid:daouuid.obj
 0002:000073c0       _IID30_ICDAOJETError       5f7363c0     daouuid:daouuid.obj
 0002:000073d0       _IID30_IDAOProperty        5f7363d0     daouuid:daouuid.obj
 0002:000073e0       _IID30_IDAOPropertyW       5f7363e0     daouuid:daouuid.obj
 0002:000073f0       _IID30_IDAOProperties      5f7363f0     daouuid:daouuid.obj
 0002:00007400       _IID30_IDAOPropertiesW     5f736400     daouuid:daouuid.obj
 0002:00007410       _IID30_IDAORecordset       5f736410     daouuid:daouuid.obj
 0002:00007420       _IID30_IDAORecordsetW      5f736420     daouuid:daouuid.obj
 0002:00007430       _IID30_IDAORecordsets      5f736430     daouuid:daouuid.obj
 0002:00007440       _IID30_IDAORecordsetsW     5f736440     daouuid:daouuid.obj
 0002:00007450       _IID30_ICDAORecordset      5f736450     daouuid:daouuid.obj
 0002:00007460       _IID30_ICDAOJETRecordset   5f736460     daouuid:daouuid.obj
 0002:00007470       _IID30_IDAOSnapshot        5f736470     daouuid:daouuid.obj
 0002:00007480       _IID30_IDAOTable           5f736480     daouuid:daouuid.obj
 0002:00007490       _IID30_IDAODynaset         5f736490     daouuid:daouuid.obj
 0002:000074a0       _IID30_IDAOWorkspace       5f7364a0     daouuid:daouuid.obj
 0002:000074b0       _IID30_IDAOWorkspaceW      5f7364b0     daouuid:daouuid.obj
 0002:000074c0       _IID30_IDAOWorkspaces      5f7364c0     daouuid:daouuid.obj
 0002:000074d0       _IID30_IDAOWorkspacesW     5f7364d0     daouuid:daouuid.obj
 0002:000074e0       _IID30_ICDAOJETWorkspace   5f7364e0     daouuid:daouuid.obj
 0002:000074f0       _CLSID30_CDAOConnection    5f7364f0     daouuid:daouuid.obj
 0002:00007500       _IID30_IDAOConnection      5f736500     daouuid:daouuid.obj
 0002:00007510       _IID30_IDAOConnectionW     5f736510     daouuid:daouuid.obj
 0002:00007520       _IID30_IDAOConnections     5f736520     daouuid:daouuid.obj
 0002:00007530       _IID30_IDAOConnectionsW    5f736530     daouuid:daouuid.obj
 0002:00007540       _CLSID30_CDAOTableDef      5f736540     daouuid:daouuid.obj
 0002:00007550       _IID30_IDAOTableDef        5f736550     daouuid:daouuid.obj
 0002:00007560       _IID30_IDAOTableDefW       5f736560     daouuid:daouuid.obj
 0002:00007570       _IID30_IDAOTableDefs       5f736570     daouuid:daouuid.obj
 0002:00007580       _IID30_IDAOTableDefsW      5f736580     daouuid:daouuid.obj
 0002:00007590       _CLSID30_CDAOField         5f736590     daouuid:daouuid.obj
 0002:000075a0       _IID30_IDAOField           5f7365a0     daouuid:daouuid.obj
 0002:000075b0       _IID30_IDAOFieldW          5f7365b0     daouuid:daouuid.obj
 0002:000075c0       _IID30_IDAOFields          5f7365c0     daouuid:daouuid.obj
 0002:000075d0       _IID30_IDAOFieldsW         5f7365d0     daouuid:daouuid.obj
 0002:000075e0       _IID30_ICDAOJETField       5f7365e0     daouuid:daouuid.obj
 0002:000075f0       _CLSID30_CDAOIndex         5f7365f0     daouuid:daouuid.obj
 0002:00007600       _IID30_IDAOIndex           5f736600     daouuid:daouuid.obj
 0002:00007610       _IID30_IDAOIndexW          5f736610     daouuid:daouuid.obj
 0002:00007620       _IID30_IDAOIndexes         5f736620     daouuid:daouuid.obj
 0002:00007630       _IID30_IDAOIndexesW        5f736630     daouuid:daouuid.obj
 0002:00007640       _IID30_IDAOIndexFields     5f736640     daouuid:daouuid.obj
 0002:00007650       _IID30_IDAOIndexFieldsW    5f736650     daouuid:daouuid.obj
 0002:00007660       _CLSID30_CDAOGroup         5f736660     daouuid:daouuid.obj
 0002:00007670       _IID30_IDAOGroup           5f736670     daouuid:daouuid.obj
 0002:00007680       _IID30_IDAOGroupW          5f736680     daouuid:daouuid.obj
 0002:00007690       _IID30_IDAOGroups          5f736690     daouuid:daouuid.obj
 0002:000076a0       _IID30_IDAOGroupsW         5f7366a0     daouuid:daouuid.obj
 0002:000076b0       _CLSID30_CDAOUser          5f7366b0     daouuid:daouuid.obj
 0002:000076c0       _IID30_IDAOUser            5f7366c0     daouuid:daouuid.obj
 0002:000076d0       _IID30_IDAOUserW           5f7366d0     daouuid:daouuid.obj
 0002:000076e0       _IID30_IDAOUsers           5f7366e0     daouuid:daouuid.obj
 0002:000076f0       _IID30_IDAOUsersW          5f7366f0     daouuid:daouuid.obj
 0002:00007700       _IID30_IDAODatabase        5f736700     daouuid:daouuid.obj
 0002:00007710       _IID30_IDAODatabaseW       5f736710     daouuid:daouuid.obj
 0002:00007720       _IID30_IDAODatabases       5f736720     daouuid:daouuid.obj
 0002:00007730       _IID30_IDAODatabasesW      5f736730     daouuid:daouuid.obj
 0002:00007740       _IID30_ICDAOJETDatabase    5f736740     daouuid:daouuid.obj
 0002:00007750       _CLSID30_CDAOQueryDef      5f736750     daouuid:daouuid.obj
 0002:00007760       _IID30_IDAOQueryDef        5f736760     daouuid:daouuid.obj
 0002:00007770       _IID30_IDAOQueryDefW       5f736770     daouuid:daouuid.obj
 0002:00007780       _IID30_IDAOQueryDefs       5f736780     daouuid:daouuid.obj
 0002:00007790       _IID30_IDAOQueryDefsW      5f736790     daouuid:daouuid.obj
 0002:000077a0       _IID30_IDAOParameter       5f7367a0     daouuid:daouuid.obj
 0002:000077b0       _IID30_IDAOParameterW      5f7367b0     daouuid:daouuid.obj
 0002:000077c0       _IID30_IDAOParameters      5f7367c0     daouuid:daouuid.obj
 0002:000077d0       _IID30_IDAOParametersW     5f7367d0     daouuid:daouuid.obj
 0002:000077e0       _CLSID30_CDAORelation      5f7367e0     daouuid:daouuid.obj
 0002:000077f0       _IID30_IDAORelation        5f7367f0     daouuid:daouuid.obj
 0002:00007800       _IID30_IDAORelationW       5f736800     daouuid:daouuid.obj
 0002:00007810       _IID30_IDAORelations       5f736810     daouuid:daouuid.obj
 0002:00007820       _IID30_IDAORelationsW      5f736820     daouuid:daouuid.obj
 0002:00007830       _IID30_IDAOContainer       5f736830     daouuid:daouuid.obj
 0002:00007840       _IID30_IDAOContainerW      5f736840     daouuid:daouuid.obj
 0002:00007850       _IID30_IDAOContainers      5f736850     daouuid:daouuid.obj
 0002:00007860       _IID30_IDAOContainersW     5f736860     daouuid:daouuid.obj
 0002:00007870       _IID30_IDAODocument        5f736870     daouuid:daouuid.obj
 0002:00007880       _IID30_IDAODocumentW       5f736880     daouuid:daouuid.obj
 0002:00007890       _IID30_IDAODocuments       5f736890     daouuid:daouuid.obj
 0002:000078a0       _IID30_IDAODocumentsW      5f7368a0     daouuid:daouuid.obj
 0002:000078b0       _IID30_IDAOCollection      5f7368b0     daouuid:daouuid.obj
 0002:000078c0       _IID30_IDAODynaCollection  5f7368c0     daouuid:daouuid.obj
 0002:000078d0       _IID30_IDAOQueryCP         5f7368d0     daouuid:daouuid.obj
 0002:000078e0       _IID30_IDAOQueryAS         5f7368e0     daouuid:daouuid.obj
 0002:000078f0       _IID30_IDisconnect         5f7368f0     daouuid:daouuid.obj
 0002:00007900       _IID30_IDisconnectAll      5f736900     daouuid:daouuid.obj
 0002:00007910       _IID30_IDSCAdviseSink      5f736910     daouuid:daouuid.obj
 0002:00007920       _IID30_IDSCConnectionPoint 5f736920     daouuid:daouuid.obj
 0002:00007930       _IID30_IDBAdviseSink       5f736930     daouuid:daouuid.obj
 0002:00007940       _IID30_IDBConnectionPoint  5f736940     daouuid:daouuid.obj
 0002:00007950       __sz_ole32                 5f736950     ole32:ole32.dll
 0002:00007960       __sz_OLEAUT32              5f736960     oleaut32:OLEAUT32.dll
 0002:00007970       __sz_ODBC32                5f736970     odbc32:ODBC32.dll
 0002:00007980       ??_R1A@?0A@A@CObject@@8    5f736980     dbcore.obj
 0002:00007998       ??_R1A@?0A@A@CException@@8 5f736998     dbcore.obj
 0002:000079b0       ??_R1A@?0A@A@CDBException@@8 5f7369b0     dbcore.obj
 0002:000079c8       ??_R2CDBException@@8       5f7369c8     dbcore.obj
 0002:000079d8       ??_R3CDBException@@8       5f7369d8     dbcore.obj
 0002:000079e8       ??_R4CDBException@@6B@     5f7369e8     dbcore.obj
 0002:00007a00       ??_R1A@?0A@A@CDatabase@@8  5f736a00     dbcore.obj
 0002:00007a18       ??_R2CDatabase@@8          5f736a18     dbcore.obj
 0002:00007a28       ??_R3CDatabase@@8          5f736a28     dbcore.obj
 0002:00007a38       ??_R4CDatabase@@6B@        5f736a38     dbcore.obj
 0002:00007a50       ??_R1A@?0A@A@CRecordset@@8 5f736a50     dbcore.obj
 0002:00007a68       ??_R2CRecordset@@8         5f736a68     dbcore.obj
 0002:00007a78       ??_R3CRecordset@@8         5f736a78     dbcore.obj
 0002:00007a88       ??_R4CRecordset@@6B@       5f736a88     dbcore.obj
 0002:00007aa0       ??_R1A@?0A@A@CNoTrackObject@@8 5f736aa0     dbcore.obj
 0002:00007ab8       ??_R1A@?0A@A@_AFX_DB_STATE@@8 5f736ab8     dbcore.obj
 0002:00007ad0       ??_R2_AFX_DB_STATE@@8      5f736ad0     dbcore.obj
 0002:00007ae0       ??_R3_AFX_DB_STATE@@8      5f736ae0     dbcore.obj
 0002:00007af0       ??_R4_AFX_DB_STATE@@6B@    5f736af0     dbcore.obj
 0002:00007b04       ??_R2CNoTrackObject@@8     5f736b04     dbcore.obj
 0002:00007b10       ??_R3CNoTrackObject@@8     5f736b10     dbcore.obj
 0002:00007b20       ??_R4CNoTrackObject@@6B@   5f736b20     dbcore.obj
 0002:00007b38       ??_R1A@?0A@A@CCmdTarget@@8 5f736b38     dbview.obj
 0002:00007b50       ??_R1A@?0A@A@CWnd@@8       5f736b50     dbview.obj
 0002:00007b68       ??_R1A@?0A@A@CView@@8      5f736b68     dbview.obj
 0002:00007b80       ??_R1A@?0A@A@CScrollView@@8 5f736b80     dbview.obj
 0002:00007b98       ??_R1A@?0A@A@CFormView@@8  5f736b98     dbview.obj
 0002:00007bb0       ??_R1A@?0A@A@CRecordView@@8 5f736bb0     dbview.obj
 0002:00007bc8       ??_R2CRecordView@@8        5f736bc8     dbview.obj
 0002:00007be8       ??_R3CRecordView@@8        5f736be8     dbview.obj
 0002:00007bf8       ??_R4CRecordView@@6B@      5f736bf8     dbview.obj
 0002:00007c10       ??_R1A@?0A@A@CLongBinary@@8 5f736c10     dblong.obj
 0002:00007c28       ??_R2CLongBinary@@8        5f736c28     dblong.obj
 0002:00007c38       ??_R3CLongBinary@@8        5f736c38     dblong.obj
 0002:00007c48       ??_R4CLongBinary@@6B@      5f736c48     dblong.obj
 0002:00007c60       ??_R1A@?0A@A@CDBVariant@@8 5f736c60     dbvar.obj
 0002:00007c78       ??_R2CDBVariant@@8         5f736c78     dbvar.obj
 0002:00007c80       ??_R3CDBVariant@@8         5f736c80     dbvar.obj
 0002:00007c90       ??_R4CDBVariant@@6B@       5f736c90     dbvar.obj
 0002:00007ca8       ??_R1A@?0A@A@_AFX_DAO_STATE@@8 5f736ca8     daocore.obj
 0002:00007cc0       ??_R2_AFX_DAO_STATE@@8     5f736cc0     daocore.obj
 0002:00007cd0       ??_R3_AFX_DAO_STATE@@8     5f736cd0     daocore.obj
 0002:00007ce0       ??_R4_AFX_DAO_STATE@@6B@   5f736ce0     daocore.obj
 0002:00007cf8       ??_R1A@?0A@A@CDaoIndexInfo@@8 5f736cf8     daocore.obj
 0002:00007d10       ??_R2CDaoIndexInfo@@8      5f736d10     daocore.obj
 0002:00007d18       ??_R3CDaoIndexInfo@@8      5f736d18     daocore.obj
 0002:00007d28       ??_R4CDaoIndexInfo@@6B@    5f736d28     daocore.obj
 0002:00007d40       ??_R1A@?0A@A@CDaoRelationInfo@@8 5f736d40     daocore.obj
 0002:00007d58       ??_R2CDaoRelationInfo@@8   5f736d58     daocore.obj
 0002:00007d60       ??_R3CDaoRelationInfo@@8   5f736d60     daocore.obj
 0002:00007d70       ??_R4CDaoRelationInfo@@6B@ 5f736d70     daocore.obj
 0002:00007d88       ??_R1A@?0A@A@CDaoException@@8 5f736d88     daocore.obj
 0002:00007da0       ??_R2CDaoException@@8      5f736da0     daocore.obj
 0002:00007db0       ??_R3CDaoException@@8      5f736db0     daocore.obj
 0002:00007dc0       ??_R4CDaoException@@6B@    5f736dc0     daocore.obj
 0002:00007dd8       ??_R1A@?0A@A@CDaoErrorInfo@@8 5f736dd8     daocore.obj
 0002:00007df0       ??_R2CDaoErrorInfo@@8      5f736df0     daocore.obj
 0002:00007df8       ??_R3CDaoErrorInfo@@8      5f736df8     daocore.obj
 0002:00007e08       ??_R4CDaoErrorInfo@@6B@    5f736e08     daocore.obj
 0002:00007e20       ??_R1A@?0A@A@CDaoWorkspace@@8 5f736e20     daocore.obj
 0002:00007e38       ??_R2CDaoWorkspace@@8      5f736e38     daocore.obj
 0002:00007e48       ??_R3CDaoWorkspace@@8      5f736e48     daocore.obj
 0002:00007e58       ??_R4CDaoWorkspace@@6B@    5f736e58     daocore.obj
 0002:00007e70       ??_R1A@?0A@A@CDaoDatabase@@8 5f736e70     daocore.obj
 0002:00007e88       ??_R2CDaoDatabase@@8       5f736e88     daocore.obj
 0002:00007e98       ??_R3CDaoDatabase@@8       5f736e98     daocore.obj
 0002:00007ea8       ??_R4CDaoDatabase@@6B@     5f736ea8     daocore.obj
 0002:00007ec0       ??_R1A@?0A@A@CDaoRelationFieldInfo@@8 5f736ec0     daocore.obj
 0002:00007ed8       ??_R2CDaoRelationFieldInfo@@8 5f736ed8     daocore.obj
 0002:00007ee0       ??_R3CDaoRelationFieldInfo@@8 5f736ee0     daocore.obj
 0002:00007ef0       ??_R4CDaoRelationFieldInfo@@6B@ 5f736ef0     daocore.obj
 0002:00007f08       ??_R1A@?0A@A@CDaoTableDef@@8 5f736f08     daocore.obj
 0002:00007f20       ??_R2CDaoTableDef@@8       5f736f20     daocore.obj
 0002:00007f30       ??_R3CDaoTableDef@@8       5f736f30     daocore.obj
 0002:00007f40       ??_R4CDaoTableDef@@6B@     5f736f40     daocore.obj
 0002:00007f58       ??_R1A@?0A@A@CDaoFieldInfo@@8 5f736f58     daocore.obj
 0002:00007f70       ??_R2CDaoFieldInfo@@8      5f736f70     daocore.obj
 0002:00007f78       ??_R3CDaoFieldInfo@@8      5f736f78     daocore.obj
 0002:00007f88       ??_R4CDaoFieldInfo@@6B@    5f736f88     daocore.obj
 0002:00007fa0       ??_R1A@?0A@A@CDaoQueryDef@@8 5f736fa0     daocore.obj
 0002:00007fb8       ??_R2CDaoQueryDef@@8       5f736fb8     daocore.obj
 0002:00007fc8       ??_R3CDaoQueryDef@@8       5f736fc8     daocore.obj
 0002:00007fd8       ??_R4CDaoQueryDef@@6B@     5f736fd8     daocore.obj
 0002:00007ff0       ??_R1A@?0A@A@CDaoRecordset@@8 5f736ff0     daocore.obj
 0002:00008008       ??_R2CDaoRecordset@@8      5f737008     daocore.obj
 0002:00008018       ??_R3CDaoRecordset@@8      5f737018     daocore.obj
 0002:00008028       ??_R4CDaoRecordset@@6B@    5f737028     daocore.obj
 0002:00008040       ??_R1A@?0A@A@CDaoIndexFieldInfo@@8 5f737040     daocore.obj
 0002:00008058       ??_R2CDaoIndexFieldInfo@@8 5f737058     daocore.obj
 0002:00008060       ??_R3CDaoIndexFieldInfo@@8 5f737060     daocore.obj
 0002:00008070       ??_R4CDaoIndexFieldInfo@@6B@ 5f737070     daocore.obj
 0002:00008088       ??_R1A@?0A@A@CDaoRecordView@@8 5f737088     daoview.obj
 0002:000080a0       ??_R2CDaoRecordView@@8     5f7370a0     daoview.obj
 0002:000080c0       ??_R3CDaoRecordView@@8     5f7370c0     daoview.obj
 0002:000080d0       ??_R4CDaoRecordView@@6B@   5f7370d0     daoview.obj
 0002:000080e8       ??_R1A@?0A@A@type_info@@8  5f7370e8     msvcrtd:ti_inst.obj
 0002:00008100       ??_R2type_info@@8          5f737100     msvcrtd:ti_inst.obj
 0002:00008108       ??_R3type_info@@8          5f737108     msvcrtd:ti_inst.obj
 0002:00008118       ??_R4type_info@@6B@        5f737118     msvcrtd:ti_inst.obj
 0002:000081a8       __CT??_R0PAX@84            5f7371a8     dbcore.obj
 0002:000081c8       __CT??_R0PAVCObject@@@84   5f7371c8     dbcore.obj
 0002:000081e8       __CT??_R0PAVCException@@@84 5f7371e8     dbcore.obj
 0002:00008208       __CT??_R0PAVCDBException@@@84 5f737208     dbcore.obj
 0002:00008228       __CTA4PAVCDBException@@    5f737228     dbcore.obj
 0002:00008240       __TI4PAVCDBException@@     5f737240     dbcore.obj
 0002:0000af80       __CT??_R0PAVCDaoException@@@84 5f739f80     daocore.obj
 0002:0000afa0       __CTA4PAVCDaoException@@   5f739fa0     daocore.obj
 0002:0000afb8       __TI4PAVCDaoException@@    5f739fb8     daocore.obj
 0002:0000b408       __DELAY_IMPORT_DESCRIPTOR_ole32 5f73a408     ole32:ole32.dll
 0002:0000b428       __DELAY_IMPORT_DESCRIPTOR_OLEAUT32 5f73a428     oleaut32:OLEAUT32.dll
 0002:0000b448       __DELAY_IMPORT_DESCRIPTOR_ODBC32 5f73a448     odbc32:ODBC32.dll
 0002:0000b468       __NULL_DELAY_IMPORT_DESCRIPTOR 5f73a468     ole32:ole32.dll
 0002:0000b508       \177ODBC32_NULL_THUNK_DATA_DLN 5f73a508     odbc32:ODBC32.dll
 0002:0000b510       \177OLEAUT32_NULL_THUNK_DATA_DLN 5f73a510     oleaut32:OLEAUT32.dll
 0002:0000b520       \177ole32_NULL_THUNK_DATA_DLN 5f73a520     ole32:ole32.dll
 0002:0000b560       \177ole32_NULL_THUNK_DATA_DLB 5f73a560     ole32:ole32.dll
 0002:0000b570       \177OLEAUT32_NULL_THUNK_DATA_DLB 5f73a570     oleaut32:OLEAUT32.dll
 0002:0000b578       \177ODBC32_NULL_THUNK_DATA_DLB 5f73a578     odbc32:ODBC32.dll
 0002:0000b5f8       __IMPORT_DESCRIPTOR_MFC42D 5f73a5f8     MFC42D:MFC42D.DLL
 0002:0000b60c       __IMPORT_DESCRIPTOR_MFCO42D 5f73a60c     MFCO42D:MFCO42D.DLL
 0002:0000b620       __IMPORT_DESCRIPTOR_MSVCRTD 5f73a620     msvcrtd:MSVCRTD.dll
 0002:0000b634       __IMPORT_DESCRIPTOR_KERNEL32 5f73a634     kernel32:KERNEL32.dll
 0002:0000b648       __IMPORT_DESCRIPTOR_USER32 5f73a648     user32:USER32.dll
 0002:0000b65c       __NULL_IMPORT_DESCRIPTOR   5f73a65c     MFC42D:MFC42D.DLL
 0003:00000000       ___xc_a                    5f73c000     msvcrtd:cinitexe.obj
 0003:00000008       ___xc_z                    5f73c008     msvcrtd:cinitexe.obj
 0003:0000000c       ___xi_a                    5f73c00c     msvcrtd:cinitexe.obj
 0003:00000010       ___xi_z                    5f73c010     msvcrtd:cinitexe.obj
 0003:0000002c       __pRawDllMain              5f73c02c     dlldb.obj
 0003:00000030       ?_afxForceVectorDelete_mfcd@@3P6AXXZA 5f73c030     dlldb.obj
 0003:00000038       ?GUID_ATLVer30@ATL@@3U_GUID@@A 5f73c038     dlldb.obj
 0003:00000060       ??_R0PAX@8                 5f73c060     dbcore.obj
 0003:00000070       ??_R0PAVCObject@@@8        5f73c070     dbcore.obj
 0003:00000088       ??_R0PAVCException@@@8     5f73c088     dbcore.obj
 0003:000000a8       ??_R0PAVCDBException@@@8   5f73c0a8     dbcore.obj
 0003:000000c8       ??_R0?AVCObject@@@8        5f73c0c8     dbcore.obj
 0003:000000e0       ??_R0?AVCException@@@8     5f73c0e0     dbcore.obj
 0003:00000100       ??_R0?AVCDBException@@@8   5f73c100     dbcore.obj
 0003:00000120       ??_R0?AVCDatabase@@@8      5f73c120     dbcore.obj
 0003:00000138       ??_R0?AVCRecordset@@@8     5f73c138     dbcore.obj
 0003:00000158       ??_R0?AVCNoTrackObject@@@8 5f73c158     dbcore.obj
 0003:00000178       ??_R0?AV_AFX_DB_STATE@@@8  5f73c178     dbcore.obj
 0003:000001c8       ??_R0?AVCCmdTarget@@@8     5f73c1c8     dbview.obj
 0003:000001e8       ??_R0?AVCWnd@@@8           5f73c1e8     dbview.obj
 0003:00000200       ??_R0?AVCView@@@8          5f73c200     dbview.obj
 0003:00000218       ??_R0?AVCScrollView@@@8    5f73c218     dbview.obj
 0003:00000238       ??_R0?AVCFormView@@@8      5f73c238     dbview.obj
 0003:00000250       ??_R0?AVCRecordView@@@8    5f73c250     dbview.obj
 0003:00000288       ??_R0?AVCLongBinary@@@8    5f73c288     dblong.obj
 0003:000002b0       ??_R0?AVCDBVariant@@@8     5f73c2b0     dbvar.obj
 0003:000002e8       ?_afxNullVariant@@3UtagVARIANT@@A 5f73c2e8     daocore.obj
 0003:000002f8       ?_afxOptionalVariant@@3UtagVARIANT@@A 5f73c2f8     daocore.obj
 0003:00000308       ??_R0?AV_AFX_DAO_STATE@@@8 5f73c308     daocore.obj
 0003:00000328       ??_R0?AUCDaoIndexInfo@@@8  5f73c328     daocore.obj
 0003:00000348       ??_R0?AUCDaoRelationInfo@@@8 5f73c348     daocore.obj
 0003:00000368       ??_R0?AVCDaoException@@@8  5f73c368     daocore.obj
 0003:00000388       ??_R0?AUCDaoErrorInfo@@@8  5f73c388     daocore.obj
 0003:000003a8       ??_R0PAVCDaoException@@@8  5f73c3a8     daocore.obj
 0003:000003c8       ??_R0?AVCDaoWorkspace@@@8  5f73c3c8     daocore.obj
 0003:000003e8       ??_R0?AVCDaoDatabase@@@8   5f73c3e8     daocore.obj
 0003:00000408       ??_R0?AUCDaoRelationFieldInfo@@@8 5f73c408     daocore.obj
 0003:00000430       ??_R0?AVCDaoTableDef@@@8   5f73c430     daocore.obj
 0003:00000450       ??_R0?AUCDaoFieldInfo@@@8  5f73c450     daocore.obj
 0003:00000470       ??_R0?AVCDaoQueryDef@@@8   5f73c470     daocore.obj
 0003:00000490       ??_R0?AVCDaoRecordset@@@8  5f73c490     daocore.obj
 0003:000004b0       ??_R0?AUCDaoIndexFieldInfo@@@8 5f73c4b0     daocore.obj
 0003:00000508       ??_R0?AVCDaoRecordView@@@8 5f73c508     daoview.obj
 0003:00000540       ??_R0?AVtype_info@@@8      5f73c540     msvcrtd:ti_inst.obj
 0003:00000558       __imp__SQLGetInfo@20       5f73c558     odbc32:ODBC32.dll
 0003:0000055c       __imp__SQLSetConnectOption@12 5f73c55c     odbc32:ODBC32.dll
 0003:00000560       __imp__SQLBindCol@24       5f73c560     odbc32:ODBC32.dll
 0003:00000564       __imp__SQLParamData@8      5f73c564     odbc32:ODBC32.dll
 0003:00000568       __imp__SQLBindParameter@40 5f73c568     odbc32:ODBC32.dll
 0003:0000056c       __imp__SQLPutData@12       5f73c56c     odbc32:ODBC32.dll
 0003:00000570       __imp__SQLError@32         5f73c570     odbc32:ODBC32.dll
 0003:00000574       __imp__SQLFreeStmt@8       5f73c574     odbc32:ODBC32.dll
 0003:00000578       __imp__SQLCancel@4         5f73c578     odbc32:ODBC32.dll
 0003:0000057c       __imp__SQLMoreResults@4    5f73c57c     odbc32:ODBC32.dll
 0003:00000580       __imp__SQLFetch@4          5f73c580     odbc32:ODBC32.dll
 0003:00000584       __imp__SQLNumResultCols@8  5f73c584     odbc32:ODBC32.dll
 0003:00000588       __imp__SQLExecDirect@12    5f73c588     odbc32:ODBC32.dll
 0003:0000058c       __imp__SQLAllocStmt@8      5f73c58c     odbc32:ODBC32.dll
 0003:00000590       __imp__SQLFreeConnect@4    5f73c590     odbc32:ODBC32.dll
 0003:00000594       __imp__SQLDisconnect@4     5f73c594     odbc32:ODBC32.dll
 0003:00000598       __imp__SQLFreeEnv@4        5f73c598     odbc32:ODBC32.dll
 0003:0000059c       __imp__SQLSetStmtOption@12 5f73c59c     odbc32:ODBC32.dll
 0003:000005a0       __imp__SQLRowCount@8       5f73c5a0     odbc32:ODBC32.dll
 0003:000005a4       __imp__SQLExecute@4        5f73c5a4     odbc32:ODBC32.dll
 0003:000005a8       __imp__SQLTransact@12      5f73c5a8     odbc32:ODBC32.dll
 0003:000005ac       __imp__SQLAllocConnect@8   5f73c5ac     odbc32:ODBC32.dll
 0003:000005b0       __imp__SQLAllocEnv@4       5f73c5b0     odbc32:ODBC32.dll
 0003:000005b4       __imp__SQLDriverConnect@32 5f73c5b4     odbc32:ODBC32.dll
 0003:000005b8       __imp__SQLGetData@24       5f73c5b8     odbc32:ODBC32.dll
 0003:000005bc       __imp__SQLSetPos@16        5f73c5bc     odbc32:ODBC32.dll
 0003:000005c0       __imp__SQLGetStmtOption@12 5f73c5c0     odbc32:ODBC32.dll
 0003:000005c4       __imp__SQLPrepare@12       5f73c5c4     odbc32:ODBC32.dll
 0003:000005c8       __imp__SQLGetFunctions@12  5f73c5c8     odbc32:ODBC32.dll
 0003:000005cc       __imp__SQLDescribeCol@36   5f73c5cc     odbc32:ODBC32.dll
 0003:000005d0       __imp__SQLExtendedFetch@20 5f73c5d0     odbc32:ODBC32.dll
 0003:000005d4       __imp__SQLGetCursorName@16 5f73c5d4     odbc32:ODBC32.dll
 0003:000005d8       \177ODBC32_NULL_THUNK_DATA_DLA 5f73c5d8     odbc32:ODBC32.dll
 0003:000005dc       __imp__SysFreeString@4     5f73c5dc     oleaut32:OLEAUT32.dll
 0003:000005e0       \177OLEAUT32_NULL_THUNK_DATA_DLA 5f73c5e0     oleaut32:OLEAUT32.dll
 0003:000005e4       __imp__CoUninitialize@0    5f73c5e4     ole32:ole32.dll
 0003:000005e8       __imp__CoGetClassObject@20 5f73c5e8     ole32:ole32.dll
 0003:000005ec       __imp__CoInitialize@4      5f73c5ec     ole32:ole32.dll
 0003:000005f0       \177ole32_NULL_THUNK_DATA_DLA 5f73c5f0     ole32:ole32.dll
 0003:000005f8       ?ATL_CREATE_OBJECT@CComApartment@ATL@@2IA 5f73c5f8     dlldb.obj
 0003:00000600       ?m_libid@CComModule@ATL@@2U_GUID@@A 5f73c600     dlldb.obj
 0003:00000610       ?_pModule@ATL@@3PAVCComModule@1@A 5f73c610     dlldb.obj
 0003:0000062c       ?_afxDbState@@3V?$CProcessLocal@V_AFX_DB_STATE@@@@A 5f73c62c     dbcore.obj
 0003:00000630       ?bTraceSql@@3HA            5f73c630     dbcore.obj
 0003:00000638       __hmod__OLE32              5f73c638     ole32:ole32.dll
 0003:0000063c       __hmod__OLEAUT32           5f73c63c     oleaut32:OLEAUT32.dll
 0003:00000640       __hmod__ODBC32             5f73c640     odbc32:ODBC32.dll
 0003:00000644       ___puiHead                 5f73c644     delayimp:delayhlp.obj
 0003:00000648       ___pfnDliFailureHook       5f73c648     delayimp:delayhk1.obj
 0003:0000064c       ___pfnDliNotifyHook        5f73c64c     delayimp:delayhk2.obj
 0003:00000650       __adjust_fdiv              5f73c650     <common>
 0003:00000654       ___onexitend               5f73c654     <common>
 0003:00000658       ___onexitbegin             5f73c658     <common>

 entry point at        0001:0002af50

 Static symbols

 0001:00015629       ?_AfxDetermineDaoVersion@@YAEXZ 5f716629 f   daocore.obj
 0001:0002bb4e       _$E376                     5f72cb4e f   dbcore.obj
 0001:0002bb5d       _$E373                     5f72cb5d f   dbcore.obj
 0001:0002bb62       _$E375                     5f72cb62 f   dbcore.obj
 0001:0002bb74       _$E374                     5f72cb74 f   dbcore.obj
 0001:0002bde0       ?_AfxForceVectorDelete@@YAXXZ 5f72cde0 f   dlldb.obj
 0001:0002ad00       ?ArrayUnwindFilter@@YAHPAU_EXCEPTION_POINTERS@@@Z 5f72bd00 f   msvcrtd:ehvecdtr.obj
 0001:0002b633       ?OverlayIAT@@YGXPAU_IMAGE_THUNK_DATA32@@PBU1@@Z 5f72c633 f   delayimp:delayhlp.obj

 113 bytes saved through ICF

